:100000000C94A21E0C94D31E0C94D31E0C94D31EDD
:100010000C94D31E0C94D31E0C94D31E0C94D31E9C
:100020000C94D31E0C94D31E0C94D31E0C94D31E8C
:100030000C94D31E0C94D31E0C94D31E0C94D31E7C
:100040000C94D31E0C94BB7C0C94D31E0C94D31E26
:100050000C94D31E0C94D31E0C94B1D40C94B0FD0C
:100060000C94D31E0C94ED5B0C94E35B0C94D31EA8
:100070000C94D31E0C94D31E0C94D31E0C94D31E3C
:100080000C94AC530C94D31E0C94D31E0C94D31E1E
:100090000C94D31E0C94D31E0C94D31E0C94D31E1C
:1000A0000C94D31E0C94D31E0C947E530C94D31E2C
:1000B0000C94D31E0C94D31E0C94D31E0C9450534A
:1000C0000C94D31E0C94D31E0C94D31E0C94AA75BE
:1000D0000C9480750C94D31E0C94D31E0C94D31ED8
:1000E0000C94D31E6D1FB31FB91FE01FED1FF61F29
:1000F0000120E8270829E4290F2AD635D6352A2BEE
:10010000CD2BE428D635D635B72D642F9C2FD63588
:100110009A31D635D635EF32D635D6357E33B13332
:10012000D6352D34E934AB2FB32FD72FFB2F2F30FB
:10013000D230E630FF300C3119312D31205C265C95
:10014000385C485C505C7D5C545C7D5C585C5C5CFD
:100150007D5C605C645C685C705C7D5C7A5C2AE5FC
:100160004CE56CE591E5B6E56DE7DBE5FEE521E6FE
:1001700046E66BE690E6B5E6DAE66DE7FFE624E7ED
:1001800049E7DDE8E0E8E4E8E7E8EAE814E9EEE872
:10019000F1E8F5E8F8E8FBE8FFE802E905E914E929
:1001A00009E90CE90FE9DCF8DFF8CEF8D2F8D8F865
:1001B00016F9E3F8E7F8EDF8F1F8F5F8FBF8FFF8D1
:1001C00003F916F909F90DF911F9ABFCB0FCB5FC0E
:1001D000BFFCC9FC42FDD3FCDBFCE3FCEDFCF7FCFF
:1001E00001FD10FD1AFD42FD24FD2EFD38FD084ADB
:1001F000D73B3BCE016E84BCBFFDC12F3D6C74313B
:100200009ABD56833DDA3D00C77F11BED9E4BB4C91
:100210003E916BAAAABE000000803F05A84CCDB25B
:10022000D44EB93836A9020C50B9918688083CA63C
:10023000AAAA2ABE000000803F000C940FE90C948B
:10024000D8F80C940DF90C94F1F80C94F5E80C9492
:10025000CD2B0C94585C0C94E7E80C94DDE80C94DE
:10026000EDFC0C94F1E80C94F7FC0C94B31F0C9487
:1002700010FD0C94B1330C9409E90C94BFFC0C9460
:100280002A2B0C9405E90C94F5F80C94705C0C94F2
:10029000C9FC0C94D72F0C942AE50C94FEE50C9421
:1002A00038740C9401200C94E3F80C9442FD0C94E7
:1002B000B91F0C94B32F0C9421E60C947E330C944C
:1002C000FB2F0C94A1740C945C5C0C9419310C946D
:1002D00001FD0C940A740C94AB2F0C945B740C9479
:1002E000E0E80C94E4E80C94605C0C94E4290C9431
:1002F000ED1F0C94EAE80C942D310C94DFF80C946B
:10030000FF300C9438FD0C94EE740C94685C0C94E3
:10031000B0FC0C94545C0C94265C0D94B71C0C94AB
:100320009C2F0C947D5C0C94EF320C94ABFC0C94E1
:1003300046E60C941AFD0C94B6E50C94D2300C945D
:100340006CE50C94FBE80C946D1F0C940CE90C9478
:10035000485C0C94E8270C94D2F80C9491E50C942A
:10036000CEF80C94FBF80C947A5C0C94B5E60C94E3
:10037000642F0C94DCF80C9403F90C94D3FC0C94CB
:10038000DBFC0C9469740C94205C0C94EDF80C94D8
:1003900002E90C9424FD0C94D6350C94E6300C94B0
:1003A000DBE50D946D1C0C9416F90C9447740C94B9
:1003B0000F2A0C946DE70C949A310C9424E70C945A
:1003C00011F90C9490E60C94385C0C9449E70C9469
:1003D000505C0C94FFF80C942D340C944CE50C9468
:1003E000E4280C94B72D0C940C310C94EEE80C948A
:1003F000E3FC0C9409F90C94DAE60C94F8E80C94FC
:100400006BE60C942EFD0C942F300C94645C0C94D1
:1004100014E90C9408290C94FFE60C94E9340C942C
:10042000E01F0C94E7F80C94FFE80C94F61F0C9472
:10043000B5FC4E414E494E495459494E46CDCCCC5F
:100440003D0AD7233C17B7D13877CC2B329595E6A8
:10045000241FB14F0A000020410000C84200401C88
:100460004620BCBE4CCA1B0E5AAEC59D7400407AD5
:1004700010F35A00A0724E18090010A5D4E800002D
:10048000E87648170000E40B54020000CA9A3B00CB
:100490000000E1F505000080969800000040420F42
:1004A000000000A08601000000102700000000E806
:1004B00003000000006400000000000A00000000CB
:1004C000000100000000002C76D888DC674F08236C
:1004D000DFC1DFAE59E1B1B796E5E3E453C63AE6D2
:1004E00051997696E8E6C28426EB898C9B62ED40B2
:1004F0007C6FFCEFBC9C9F40F2BAA56FA5F4900501
:100500005A2AF75C936B6CF9676DC11BFCE0E40D34
:1005100047FEF520E6B500D0ED902E030094357728
:10052000050080841E080000204E0A000000C80C50
:10053000333333330F986E12831141EF8D211489B9
:100540003BE65516CFFEE6DB18D1844B381BF77C13
:100550001D901DA4BBE424203284725E228100C958
:10056000F124ECA1E53D274D323520500A4D3234BF
:1005700000526573756D650055492050617573654E
:10058000004E6F204D61746368203A004D33303364
:10059000452D31533635433455004D393939004DE9
:1005A0003530320A4D353030004D3330334530531D
:1005B000323135433855000A202A2A2A726563648D
:1005C00061742E646174615B305D203D0047323898
:1005D0000A4731204631303030205A313000556ED4
:1005E000737570706F72746564204F7074696F6E8C
:1005F0002053656C6563746564004D313930533543
:10060000350A4732380A4732390A4D3430300A4DFC
:10061000313034533231350A4732380A4D313039AE
:10062000533231350A4D34323053310A4731583163
:1006300030305931303046353030300A47315A3059
:100640000A4D3530300A4D31313720536574205A08
:10065000204F666673657400473120463130303074
:10066000205A302E30004732380A47312046313088
:100670003030205A302E30004D353030005A204F67
:100680006666736574203A202573004D353030005E
:100690005A204F6666736574203A202573004732EE
:1006A000385A0A473146313530305A302E300047FB
:1006B00032380A473146313530305A302E30004D0D
:1006C000383400473146313030305A302E30004710
:1006D00032380A473146313030305A302E30005AE5
:1006E000204F6666736574203A202573004D3530BF
:1006F00030004D383400426567696E537769746322
:1007000068007265636461742E61646472203D3DAB
:10071000007265636461742E646174615B305D2096
:100720003D3D0077616974776179203D3D000A2085
:100730002A2A2A4E6F7A7A6C6554656D70537461FB
:100740007475735B325D203D00434F4D4D554E49EE
:10075000434154494F4E0044525952554E00455260
:10076000524F525300494E464F004543484F0047B1
:10077000322F47332062616420706172616D65744D
:100780006572730A00536C6565702E2E2E005A2018
:1007900050726F62652050617374204265640A0074
:1007A0005A2050726F6265205061737420426564F4
:1007B00000486F6D652058592046697273740A00AD
:1007C000486F6D65205859204669727374004D3129
:1007D00031372050726F6265206661696C65642EE6
:1007E0000A4732380A0070726F62655F7265776916
:1007F0007065004469736D69737300473239205224
:1008000065747279696E670050726F62696E6720F5
:100810004661696C6564004D313137204265642062
:100820006C6576656C696E67206661696C65642EBF
:100830000A4730205A31300A4D333030205032359B
:1008400020533838300A4D33303020503530205363
:10085000300A4D3330302050323520533838300A8A
:100860004D333030205035302053300A4D33303046
:100870002050323520533838300A4D333030205034
:1008800035302053300A47342053310070726F6284
:10089000655F6661696C6564004D31313720426582
:1008A00064206C6576656C696E6720646F6E652E7A
:1008B00000205A3A200020593A200042656420580E
:1008C0003A20004D65736820706F696E7420636113
:1008D0006E6E6F74206265207265736F6C766564EE
:1008E0000A004D302F3120427265616B2043616CEC
:1008F0006C656400436F6E74696E7565004D302FD2
:100900003120427265616B2043616C6C6564004EFE
:100910006F204D6F76652E00456E642066696C65AC
:10092000206C6973740A00426567696E2066696CA1
:1009300065206C6973740A004469736D6973730090
:10094000526573756D696E6720534400286E6F2081
:1009500066696C65290043757272656E74206669FC
:100960006C653A20002E0A0044656C6574696F6EF0
:10097000206661696C65642C2046696C653A2000CC
:1009800046696C652064656C657465643A005072F4
:10099000696E742074696D653A20000A537461743D
:1009A000733A2046696C616D656E74207573656479
:1009B0003A20002C204C6F6E67657374206A6F625A
:1009C0003A2000546F74616C2074696D653A2000A0
:1009D00053746174733A20002C204661696C65641D
:1009E0003A20002C2046696E69736865643A2000DD
:1009F0005072696E74733A200053746174733A20B4
:100A000000436F6F6C696E672E2E2E00486561740F
:100A1000696E672E2E2E0045202553006F6B006FE8
:100A20006666006A0765075E07570749074445423F
:100A300055473A004D31313320530042656420431D
:100A40006F6F6C696E672E2E2E00426564204865BC
:100A50006174696E672E2E2E004348414D42455207
:100A60005F54454D5045524154555245004D4F54E9
:100A7000494F4E5F4D4F44455300544845524D41F8
:100A80004C5F50524F54454354494F4E00415554CA
:100A90004F5245504F52545F53445F535441545545
:100AA000530050524F4D50545F535550504F525475
:100AB00000454D455247454E43595F5041525345BD
:100AC0005200434153455F4C494748545F425249A5
:100AD0004748544E45535300544F47474C455F4C8D
:100AE000494748545300534F4654574152455F506D
:100AF0004F574552004255494C445F50455243457B
:100B00004E54004C4556454C494E475F4441544174
:100B1000005A5F50524F4245004155544F4C455684
:100B2000454C005052494E545F4A4F420050524F7C
:100B30004752455353004155544F5245504F52541C
:100B40005F54454D5000564F4C554D455452494306
:100B500000454550524F4D0042494E4152595F4663
:100B6000494C455F5452414E5346455200534552FD
:100B700049414C5F584F4E5F584F464600464952D8
:100B80004D574152455F4E414D453A4D61726C693A
:100B90006E20322E305F44573420544D334420357C
:100BA000534D44424220534F555243455F434F44B7
:100BB000455F55524C3A68747470733A2F2F6769C9
:100BC000746875622E636F6D2F496E73616E697400
:100BD000794175746F6D6174696F6E2F4D61726CC0
:100BE000696E2F747265652F437265616C697479E3
:100BF0005F4D61726C696E322E302E782050524FEC
:100C0000544F434F4C5F56455253494F4E3A312E45
:100C100030204D414348494E455F545950453A5460
:100C20004D3344204D617820455854525544455227
:100C30005F434F554E543A3120555549443A636508
:100C40006465326132662D343161322D3437343887
:100C50002D396231322D633535633632663336379E
:100C600066660A002F2F20003F4A206F7574206FA0
:100C7000662072616E67652028302E303120746FD7
:100C800020302E33290A0020466C6F773A2000501E
:100C9000726F7465637465642050696E0A00206F1A
:100CA0007574206F662072616E67650A0053657205
:100CB000766F20003A200020536572766F2000493D
:100CC0006E76616C69642065787472756465720A09
:100CD0000020643A0020693A0020703A0020643A0B
:100CE0000020693A0020703A0064697300656E0064
:100CF00043290A0061626C656420286D696E207466
:100D0000656D702000436F6C642065787472756443
:100D100065732061726520004F4646004F4E0046C5
:100D2000696C616D656E742072756E6F7574206488
:100D3000697374616E636520286D6D293A200046E1
:100D4000696C616D656E742072756E6F75742000CC
:100D50004D65736820706F696E742063616E6E6F8D
:100D600074206265207265736F6C7665640A004D4D
:100D700034323120696E636F727265637420706102
:100D800072616D657465722075736167650A004FE5
:100D9000666673657473204170706C6965640045A4
:100DA00072723A20546F6F206661722100546F6F27
:100DB000206661722066726F6D207265666572656D
:100DC0006E636520706F696E740A00454550524F1E
:100DD0004D204F4B0A004572726F72207772697412
:100DE000696E6720746F20454550524F4D210A00AF
:100DF000363726033C3D380E2E303E131A1C180899
:100E0000440AFF430809070001627573793A2070AC
:100E1000617573656420666F7220696E7075740AFF
:100E200000627573793A2070617573656420666F2E
:100E30007220757365720A00627573793A20707258
:100E40006F63657373696E670A007061757365001F
:100E50004D363030002066696C616D656E745F726E
:100E6000756E6F7574200066696C616D656E745F78
:100E700072756E6F757420540046696C616D656E95
:100E80007452756E6F757420540053544F50504512
:100E9000442E20005072696E7465722073746F70F6
:100EA0007065642064756520746F206572726F725E
:100EB000732E2046697820746865206572726F729F
:100EC00020616E6420757365204D39393920746F47
:100ED00020726573746172742E202854656D70657C
:100EE0007261747572652069732072657365742E02
:100EF0002053657420697420616674657220726580
:100F00007374617274696E67290A004E6F204368BA
:100F100065636B73756D2077697468206C696E65A5
:100F2000206E756D6265722C204C617374204C6963
:100F30006E653A20004E6F20436865636B73756D74
:100F40002077697468206C696E65206E756D6265C6
:100F5000722C204C617374204C696E653A200063DA
:100F60006865636B73756D206D69736D617463681B
:100F70002C204C617374204C696E653A20004C69DA
:100F80006E65204E756D626572206973206E6F7498
:100F9000204C617374204C696E65204E756D6265DE
:100FA000722B312C204C617374204C696E653A2091
:100FB000004D31313000776169740A004D313137AD
:100FC000004D3331005344207265616420657272B4
:100FD0006F720A00446F6E65207072696E74696E7C
:100FE000672066696C650A004B494C4C206361754B
:100FF00073656420627920746F6F206D756368205B
:10100000696E6163746976652074696D65202D2051
:1010100063757272656E7420636F6D6D616E643A94
:1010200020002020506C616E6E65724275666665A8
:101030007242797465733A20002046726565204DCE
:10104000656D6F72793A2000436F6D70696C6564ED
:101050003A204F637420323720323031390A002071
:101060004C61737420557064617465643A20323049
:1010700031392D31302D3035207C20417574686F29
:10108000723A2054696E794D616368696E65733395
:10109000440A00322E305F4457340A004D61726CAE
:1010A000696E0020536F66747761726520526573B4
:1010B00065740A00205761746368646F6720526525
:1010C0007365740A002042726F776E206F7574200A
:1010D00052657365740A002045787465726E616CA0
:1010E0002052657365740A00506F77657255700AF7
:1010F0000073746172740A006175746F25632E67E2
:10110000006572726F722077726974696E672074FD
:101110006F2066696C650A00446F6E6520736176A6
:10112000696E672066696C652E0A004D32390020B1
:101130005A3A0020593A0020583A00656E64737498
:101140006F7073206869743A20004732385859002C
:1011500024F4D43050C38E20C2A24017828B701169
:10116000127A910D816CD90AA861E108C758660707
:10117000615143061E4B5D05C145A7041A41110488
:10118000093D9803713931034036DB026533910222
:10119000D4305402802E1D02632CEE01752AC50145
:1011A000B028A001102781018F2564012B244B0159
:1011B000E0223401AC211F018D200D01801FFC00B5
:1011C000841EED00971DDF00B81CD200E61BC60090
:1011D000201BBC00641AB200B219A8000A19A000B2
:1011E0006A189900D117910040178B00B51684003A
:1011F00031167E00B31579003A157300C7146F00DD
:1012000058146A00EE1366008813630025135E000D
:10121000C7125B006C12570015125400C111510027
:1012200070114F0021114B00D61049008D1047005E
:101230004610440002104200C00F4000800F3E00E4
:10124000420F3C00060F3B00CB0E3800930E3700D8
:101250005C0E3500270E3400F30D3200C10D310055
:10126000900D3000600D2E00320D2D00050D2C006C
:10127000D90C2B00AE0C2900850C29005C0C270032
:10128000350C27000E0C2600E80B2400C40B2400AC
:10129000A00B23007D0B23005A0B2100390B2100EA
:1012A000180B2000F80A1F00D90A1E00BB0A1E00F6
:1012B0009D0A1D00800A1D00630A1C00470A1B00CE
:1012C0002C0A1B00110A1A00F7091A00DD0919007F
:1012D000C4091900AB091900920917007B0918000D
:1012E000630917004C09160036091600200916007C
:1012F0000A091500F5081500E0081400CC081400D0
:10130000B8081400A4081400900813007D08120007
:101310006B08130058081200460812003408110028
:10132000230811001208110001081100F007100035
:10133000E0071000D0071000C0071000B0070F0032
:10134000A107100091070E0083070F0074070F001C
:1013500065070E0057070E0049070E003B070D00FA
:101360002E070E0020070D0013070D0006070D00C5
:10137000F9060C00ED060D00E0060C00D4060C008A
:10138000C8060C00BC060C00B0060C00A4060B003E
:1013900099060C008D060B0082060B0077060B00E9
:1013A0006C060B0061060A0057060B004C060A008B
:1013B00042060A0038060A002E060A0024060A0021
:1013C0001A060A001006090007060A00FD050900B2
:1013D000F4050900EB050900E2050900D90509003B
:1013E000D0050900C7050900BE050900B5050800BC
:1013F000AD050800A50509009C0508009405080036
:101400008C050800840508007C05080074050800A8
:101410006C050700650508005D0507005605080016
:101420004E0507004705070040050800380507007E
:10143000310507002A050700230507001C050600E3
:10144000160507000F05070008050600020507003E
:10145000FB040600F5040700EE040600E80406009D
:10146000E2040700DB040600D5040600CF040600F2
:10147000C9040600C3040600BD040600B704060044
:10148000B1040500AC040600A6040600A004050093
:101490009B04060095040500900406008A040500DC
:1014A00085040500800406007A0405007504050023
:1014B000700405006B040500660405006104050066
:1014C0005C04050057040500520405004D040500A6
:1014D00048040500430405003E0404003A040500E6
:1014E00035040500300404002C0405002704040022
:1014F000230405001E0404001A0404001604050059
:10150000110404000D04040009040500040404008F
:1015100000040400FC030400F8030400F4030400C6
:10152000F0030400EC030400E8030400E4030400F7
:10153000E0030400DC030400D8030400D403040027
:10154000D0030400CC030400C8030300C503030058
:1015500024F404D9201BC40C5C0E9804C4095F0257
:1015600065077101F405F900FB04B3004804870026
:10157000C10369005803550003034500BE023A0049
:101580008402310053022A002902250004022000AF
:10159000E4011C00C8011900AF01170098011400F4
:1015A00084011300710110006101100051010E004F
:1015B00043010D0036010B002B010B0020010B0035
:1015C000150109000C01090003010800FB000800D7
:1015D000F3000800EB000700E4000600DE00060050
:1015E000D8000600D2000600CC000500C7000500A8
:1015F000C2000500BD000400B9000400B5000400ED
:10160000B1000400AD000400A9000400A50003001F
:10161000A20003009F0004009B0003009800030049
:101620009500020093000300900003008D0002006B
:101630008B00030088000200860002008400030083
:10164000810002007F0002007D0002007B0002009A
:1016500079000200770001007600020074000200A9
:1016600072000100710002006F0002006D000100B5
:101670006C0002006A0001006900020067000100BE
:1016800066000100650001006400020062000100C4
:1016900061000100600001005F0002005D000100C8
:1016A0005C0001005B0001005A00010059000100CC
:1016B00058000100570001005600010055000100CC
:1016C00054000100530000005300010052000100CB
:1016D00051000100500001004F0001004E000000C9
:1016E0004E0001004D0001004C0001004B000000C5
:1016F0004B0001004A0001004900010048000000C1
:1017000048000100470001004600000046000100BB
:1017100045000000450001004400010043000000B6
:1017200043000100420000004200010041000000AF
:1017300041000100400001003F0000003F000100A7
:101740003E0000003E0001003D0000003D000100A1
:101750003C0000003C0000003C0001003B00000099
:101760003B0001003A0000003A000100390000008F
:101770003900010038000000380000003800010086
:10178000370000003700010036000000360000007E
:101790003600010035000000350000003500010072
:1017A0003400000034000000340001003300000069
:1017B000330000003300010032000000320000005E
:1017C0003200010031000000310000003100010052
:1017D0003000000030000000300001002F00000049
:1017E0002F0000002F0000002F0001002E0000003D
:1017F0002E0000002E0001002D0000002D00000032
:101800002D0000002D0001002C0000002C00000025
:101810002C0000002C0001002B0000002B00000019
:101820002B0000002B0001002A0000002A0000000D
:101830002A0000002A000100290000002900000001
:1018400029000000290000002900010028000000F4
:1018500028000000280000002800000028000100E7
:1018600027000000270000002700000027000000DC
:1018700027000100260000002600000026000000CE
:1018800026000000260001002500000025000000C1
:1018900025000000250000002500000025000100B3
:1018A00024000000240000002400000024000000A8
:1018B000240001002300000023000000230000009A
:1018C000230000002300000023000000230001008B
:1018D0002200000022000000220000002200000080
:1018E0002200000022000100210000002100000071
:1018F0002100000021000000210000002100000064
:101900002100010020000000200000002000000055
:101910002000000020000000200000002000000047
:10192000200001001F0000001F0000001F00000039
:101930001F0000001F0000001F0000001F0001002A
:101940001E0000001E0000001E0000001E0000001F
:10195000393000003325000087190000B00F000067
:10196000DB080000BD040000740200003F0100001D
:1019700057616974696E6720666F7220686561746B
:1019800075702E0A004C656176696E6720473236A5
:10199000003F53706563696669656420582C59205F
:1019A000636F6F7264696E617465206F7574206F08
:1019B0006620626F756E64732E0A003F2852296597
:1019C000706561742076616C7565206E6F7420702F
:1019D0006C61757369626C653B206D757374206210
:1019E00065206174206C6561737420312E0A003F9C
:1019F0002852296570656174206D75737420626565
:101A000020737065636966696564207768656E2018
:101A10006E6F74207573696E6720616E204C43444D
:101A20002E0A003F537065636966696564206E6FB6
:101A30007A7A6C652074656D706572617475726513
:101A4000206E6F7420706C61757369626C652E0A0C
:101A5000003F5370656369666965642066696C61FF
:101A60006D656E742073697A65206E6F7420706C7A
:101A700061757369626C652E0A003F537065636916
:101A800066696564207072696D65206C656E677447
:101A900068206E6F7420706C61757369626C652E5E
:101AA0000A003F5072696D65206C656E677468202E
:101AB0006D7573742062652073706563696669650E
:101AC00064207768656E206E6F74207573696E6729
:101AD00020616E204C43442E0A003F5370656369B9
:101AE00066696564206E6F7A7A6C652073697A65C1
:101AF000206E6F7420706C61757369626C652E0A5C
:101B0000003F52657472616374696F6E204D756C2D
:101B10007469706C696572206D75737420626520DC
:101B20007370656369666965642E0A003F5370656A
:101B30006369666965642052657472616374696F74
:101B40006E204D756C7469706C696572206E6F746F
:101B500020706C61757369626C652E0A003F53706A
:101B600065636966696564206C6179657220686582
:101B700069676874206E6F7420706C617573696238
:101B80006C652E0A0043292E0A003F537065636975
:101B900066696564206265642074656D7065726154
:101BA00074757265206E6F7420706C6175736962F4
:101BB0006C65202834302D004732362073746172F2
:101BC00074696E672E2E2E0A0043616E6E6F74204C
:101BD0006F70656E207375626469722000534420D3
:101BE00063617264206F6B0A006F70656E526F6F75
:101BF00074206661696C65640A00766F6C756D654A
:101C00002E696E6974206661696C65640A005344CC
:101C100020696E6974206661696C0A004D32340077
:101C20004D32332025730057726974696E672074D2
:101C30006F2066696C653A20002E0A006F70656E31
:101C4000206661696C65642C2046696C653A2000E9
:101C50002E0A006F70656E206661696C65642C20C9
:101C600046696C653A200046696C652073656C6551
:101C7000637465640A002053697A653A20004669F6
:101C80006C65206F70656E65643A200066726573DE
:101C90006800646F696E67002066696C653A2000B1
:101CA0004E6F772000454E4420535542524F5554B5
:101CB000494E450A002220706F7300222070617225
:101CC000656E743A2200535542524F5554494E4561
:101CD0002043414C4C207461726765743A22007451
:101CE0007279696E6720746F2063616C6C20737504
:101CF000622D67636F64652066696C657320776920
:101D0000746820746F6F206D616E79206C657665E4
:101D10006C732E204D4158206C6576656C2069737C
:101D20003A310A005344207072696E74696E6720FC
:101D30006279746520004E6F74205344207072697C
:101D40006E74696E670A00FFFDFCFAF8F6F4F2F0B3
:101D5000EEECEAE9E7E5E3E1E0DEDCDAD9D7D5D479
:101D6000D2D0CFCDCBCAC8C7C5C3C2C0BFBDBCBA15
:101D7000B9B7B6B4B3B2B0AFADACAAA9A8A6A5A482
:101D8000A2A1A09E9D9C9A99989795949392908FCA
:101D90008E8D8B8A8988878684838281807F7E7DF1
:101DA0007B7A797877767574737271706F6E6D6CFB
:101DB0006B6A696867666564636261605F5E5D5CEB
:101DC0005B5A5958585756555453525150504F4ECC
:101DD0004D4C4B4A4A494847464645444342424196
:101DE000403F3E3E3D3C3B3B3A393838373635354F
:101DF000343332323130302F2E2E2D2C2B2B2A29FA
:101E00002928272726252524232322212120201F96
:101E10001E1E1D1C1C1B1B1A191918181716161527
:101E20001514131312121111100F0F0E0E0D0D0CAD
:101E30000C0B0A0A09090808070706060505040429
:101E400003030202010000486F6D652025732573AE
:101E5000257320466972737400220A00556E6B6EFA
:101E60006F776E20636F6D6D616E643A2022002083
:101E7000746F6F206C6F6E6720657874727573690C
:101E80006F6E2070726576656E7465640A002063FB
:101E90006F6C6420657874727573696F6E207072F0
:101EA0006576656E7465640A007C3C3E5E2B3D3F42
:101EB0002F5B5D3B2C2A225C0050726F62696E675B
:101EC00020506F696E740025532025692F25690005
:101ED0002E0A002F0050726F62696E67206D657365
:101EE0006820706F696E7420002028445259525542
:101EF0004E2900473239204175746F2042656420B5
:101F00004C6576656C696E67003F20284C2C522C1E
:101F1000462C4229206F7574206F6620626F756EA3
:101F200064732E0A003F2856296572626F7365201C
:101F30006C6576656C20696D706C61757369626C37
:101F4000652028302D34292E0A00426164205A2051
:101F500076616C75650A004E6F2062696C696E650A
:101F6000617220677269640A005374616E64617201
:101F70006420446576696174696F6E3A200020526E
:101F8000616E67653A2000204D61783A2000204D4F
:101F9000696E3A20004D65616E3A200046696E69AF
:101FA00073686564210A002072616E67653A2000DB
:101FB000206D61783A2000206D696E3A2000207310
:101FC00069676D613A2000206D65616E3A20003AC4
:101FD000207A3A2000206F662000205900476F6960
:101FE0006E6720746F3A20580043570A00206469D6
:101FF000723A0020616E676C653A005374617274C6
:10200000207261646975733A00506F736974696F07
:102010006E696E67207468652070726F62652E2E1F
:102020002E0A003F4E756D626572206F66206C65EA
:10203000677320696E206D6F76656D656E74206EB6
:102040006F7420706C61757369626C652028302D27
:102050003135292E0A003F2028582C5929206F7528
:1020600074206F6620626F756E64732E0A003F5392
:10207000616D706C652073697A65206E6F74207075
:102080006C61757369626C652028342D3530292E9A
:102090000A004D3438205A2D50726F626520526507
:1020A000706561746162696C6974792054657374D8
:1020B0000A003F2856296572626F7365206C657649
:1020C000656C20696D706C61757369626C65202840
:1020D000302D34292E0A00290A0020627974657394
:1020E0003B20637263200053657474696E677320CC
:1020F00053746F726564202800454550524F4D203F
:102100006461746173697A65206572726F722E0AF8
:1021100000290A002062797465733B206372632092
:10212000002073746F7265642073657474696E67E0
:1021300073207265747269657665642028002028B2
:1021400063616C63756C6174656429210A002021E8
:102150003D2000454550524F4D20435243206D696C
:10216000736D61746368202D202873746F726564C9
:102170002920002053697A653A2000496E64657809
:102180003A2000204D61726C696E3D563730290A45
:1021900000454550524F4D2076657273696F6E2031
:1021A0006D69736D617463682028454550524F4DC9
:1021B0003D002042002050006F6B00526573656E39
:1021C000643A200043616E6E6F74206F70656E20FC
:1021D00073756264697220002569730025696D203A
:1021E000256973002569682025696D2025697300BC
:1021F000256964202569682025696D20256973009B
:1022000025697920256964202569682025696D2064
:102210002569730023646566696E652044454641FF
:10222000554C545F0000626564004B6420004B69AC
:1022300020004B702000504944204175746F747524
:102240006E652066696E69736865642120507574D7
:1022500020746865206C617374204B702C204B696E
:1022600020616E64204B6420636F6E7374616E74C2
:10227000732066726F6D2062656C6F7720696E7473
:102280006F20436F6E66696775726174696F6E2E39
:10229000680A00504944204175746F74756E65205A
:1022A0006661696C6564212074696D656F75740A77
:1022B00000453120544845524D414C2052554E4125
:1022C0005741590042454420544845524D414C2005
:1022D00052554E4157415900546865726D616C20EA
:1022E00052756E6177617900453120486561746986
:1022F0006E67204661696C656400426564204865CC
:102300006174696E67204661696C65640048656147
:1023100074696E67206661696C6564005049442089
:102320004175746F74756E65206661696C656421B2
:102330002054656D706572617475726520746F6F7D
:1023400020686967680A00204B643A2000204B69C6
:102350003A2000204B703A20000A20436C617373CE
:10236000696320504944200A00204B643A20002031
:102370004B693A2000204B703A20000A204E6F2013
:102380006F76657273686F6F740A002054753A2017
:1023900000204B753A2000206D61783A2000206DB6
:1023A000696E3A200020643A200020626961733A25
:1023B0002000504944204175746F74756E65207318
:1023C000746172740A00504944204175746F7475C9
:1023D0006E65206661696C6564212054656D706569
:1023E00072617475726520746F6F20686967680A1E
:1023F00000504944204175746F74756E65206661A4
:10240000696C65642120426164206578747275642A
:102410006572206E756D6265720A0053544F5020CC
:1024200063616C6C65642062656361757365206FC0
:102430006620424C546F756368206572726F72201B
:102440002D20726573746172742077697468204DF1
:102450003939390A0053544F502063616C6C6564FC
:102460002062656361757365206F6620424C546F0E
:10247000756368206572726F72202D2072657374A7
:102480006172742077697468204D3939390A002FD8
:102490002F616374696F6E3A00627574746F6E00B9
:1024A000656E640070726F6D70745F0073686F7733
:1024B000004D38373620526573706F6E64696E67F1
:1024C0002050524F4D50545F00554E4B4E4F574E7B
:1024D0002053544154450047434F44455F494E46BD
:1024E0004F004C43445F50415553455F524553554F
:1024F0004D450046494C414D454E545F52554E4F57
:1025000055545F434F4E54494E55450046494C4142
:102510004D454E545F52554E4F5554004D32340088
:10252000436F6E74696E75650044697361626C65B2
:1025300052756E6F7574005075726765204D6F72BD
:102540006500506175736564007061757365640042
:10255000486F74656E6420746F6F20636F6C640ADB
:10256000004469736D697373005061757365005041
:102570007265737320627574746F6E20286F722099
:102580004D3130382920746F20726573756D650A7E
:1025900000496E736572742066696C616D656E7456
:1025A00020616E6420707265737320627574746F3D
:1025B0006E20286F72204D313038290A00436F6E2B
:1025C00074696E75650052656865617420446F6E4C
:1025D0006500526568656174696E672E2E2E005223
:1025E0006568656174696E670048656174657254F9
:1025F000696D656F75740052656865617400486542
:102600006174657254696D656F757400507265739D
:102610007320627574746F6E20286F72204D313094
:10262000382920746F2068656174206E6F7A7A6C27
:10263000650A004E6F7A7A6C65205061726B656432
:1026400000436F6E74696E7565004E6F7A7A6C65C3
:10265000205061726B656400486F74656E6420740D
:102660006F6F20636F6C640A00726573756D6564CB
:1026700000626567696E00436F6E74696E75650010
:1026800044697361626C6552756E6F757400507544
:102690007267654D6F726500506175736564004CBB
:1026A0006F61642046696C616D656E7400436F6E86
:1026B00074696E7565004C6F61642046696C616D6C
:1026C000656E74205400496E736572742066696C7F
:1026D000616D656E7420616E642070726573732025
:1026E000627574746F6E20286F72204D31303829F6
:1026F0000A004469736D69737300526573756D697F
:102700006E67000A20696E6974207A70726F626564
:102710005F7A6F6666736574203D200045455052B0
:102720004F4D20496E697469616C697A65640A006D
:1027300048617264636F6465642044656661756CAA
:10274000742053657474696E6773204C6F6164659F
:10275000640A000000FA430000C843000070410012
:102760000096420000A0420000A0420000C84300C2
:10277000000C43E8030000BC020000640000004BB2
:102780000000003A0A0020204D363033200020445B
:102790000020204D34313220530046696C616D6554
:1027A0006E742072756E6F75742073656E736F72C0
:1027B0003A0A002055004C0046696C616D656E74E4
:1027C000206C6F61642F756E6C6F6164206C656E38
:1027D000677468733A0A00205A0020590020204D7F
:1027E0003835312058005A2D50726F6265204F667F
:1027F000667365740020440020490020204D33306A
:102800003420500020440020490020204D33303136
:102810002050005049442073657474696E67733AA0
:102820000A00205A00204A00202047323920572031
:102830004900205A0020204D343230205300417589
:10284000746F20426564204C6576656C696E673AEA
:102850000A00205A0020590020204D3230362058DE
:1028600000486F6D65206F66667365743A0A0020D4
:102870004A0020540020530020204D3230352042A1
:1028800000204A3C6A756E635F6465763E00416471
:1028900076616E6365643A20423C6D696E5F736574
:1028A000676D656E745F74696D655F75733E205307
:1028B0003C6D696E5F66656564726174653E205447
:1028C0003C6D696E5F74726176656C5F66656564A8
:1028D000726174653E0020540020520020204D3269
:1028E0003034205000416363656C65726174696FB8
:1028F0006E2028756E6974732F7332293A20503C0C
:102900007072696E745F616363656C3E20523C72E5
:102910006574726163745F616363656C3E20543CEF
:1029200074726176656C5F616363656C3E0A00205A
:102930004500205A0020590020204D3230312058C7
:10294000004D6178696D756D20416363656C6572DA
:102950006174696F6E2028756E6974732F733229E4
:102960003A0A00204500205A0020590020204D320C
:1029700030332058004D6178696D756D206665654E
:102980006472617465732028756E6974732F73297E
:102990003A0A0053746570732070657220756E6911
:1029A000743A0A0020204D3230302044300A002092
:1029B000204D3230302044002044697361626C65E0
:1029C000640A0046696C616D656E74207365747489
:1029D000696E67733A0020286D6D29002020473208
:1029E00031202020203B20556E69747320696E20B1
:1029F0006D6D00486F6D696E67204661696C656436
:102A0000006F70656E005452494747455245440077
:102A10003A200066696C616D656E74007A5F6D695D
:102A20006E00795F6D696E00785F6D696E0052654A
:102A3000706F7274696E6720656E6473746F702056
:102A40007374617475730A00205A3A0020593A0071
:102A500020436F756E7420583A0020453A00205A82
:102A60003A0020593A00583A00446F6E652E0A0029
:102A700066616C7365004641494C3A204E6F207484
:102A80007269676765722064657465637465640A5A
:102A9000004641494C3A204E6F6973652064657465
:102AA0006563746564202D20706C656173652072A8
:102AB000652D72756E20746573740A0020646574E8
:102AC00065637465642E0A003D20424C546F756343
:102AD00068207072652056332E3120286F72206373
:102AE0006F6D70617469626C6529003D205A2053D6
:102AF0006572766F2050726F6265003D20424C54C3
:102B00006F7563682056332E310020282B2F2D201F
:102B1000346D73293A20003A2033306D73206F7280
:102B2000206D6F72650A002E2050756C73652077DA
:102B300069647468002A2A20506C6561736520748A
:102B40007269676765722070726F62652077697459
:102B500068696E20333020736563202A2A0A004694
:102B600041494C3A20424C544F55434820656E61D0
:102B7000626C6564202D2053657420757020746824
:102B800069732064657669636520617320612053F1
:102B90006572766F2050726F626520776974682065
:102BA000494E56455254494E472073657420746F00
:102BB000202774727565272E0A0020204445504C4A
:102BC0004F5945442073746174653A204C4F572027
:102BD000286C6F6769632030290020204445504CE1
:102BE0004F5945442073746174653A2048494748F9
:102BF00020286C6F676963203129003D204D656393
:102C000068616E6963616C205377697463682064DE
:102C1000657465637465640A005741524E494E47B6
:102C20003A20494E56455254494E472073657474B4
:102C3000696E672070726F6261626C792062616395
:102C40006B77617264732E0A002E204465706C6F7E
:102C50007920262073746F7720342074696D657332
:102C60000A003D20424C546F75636820436C6173C9
:102C700073696320312E322C20312E332C20536D7A
:102C800061727420312E302C20322E302C20322EC6
:102C9000322C20332E302C20332E31206465746585
:102CA000637465642E0A002E20436865636B20669A
:102CB0006F7220424C544F5543480A002E205A5FF1
:102CC0004D494E5F454E4453544F505F494E564513
:102CD0005254494E473A20002E2050726F626520B0
:102CE0005A5F4D494E5F50494E3A20002C20737474
:102CF0006F7720616E676C653A202020002C20647D
:102D000065706C6F7920616E676C653A2000536561
:102D100072766F2070726F626520746573740A2E0C
:102D2000207573696E6720696E6465783A202000AB
:102D30004D343320576169742043616C6C656400C5
:102D4000436F6E74696E7565004D34332057616949
:102D5000742043616C6C6564005761746368696ECC
:102D6000672070696E730A0064697300656E0061A4
:102D7000626C65640A00656E6473746F70206D6FB9
:102D80006E69746F722000204500205A002059009F
:102D9000204D3932205800205A0020590020580078
:102DA00020204D61783A2000200020204D696E3AA5
:102DB0002000536F667420656E6473746F70733A8D
:102DC00020004732380020496E76616C69642065C6
:102DD00078747275646572200070012C019001276F
:102DE00001B0012201C0011D01F001180110021300
:102DF0000130020E016002090190020401C002FFCD
:102E0000000003FA004003F5008003F000D003EB5C
:102E1000002004E6007004E100E004DC004005D777
:102E200000C005D2004006CD00D006C8008007C310
:102E3000003008BE00F008B900C009B400B00AAF05
:102E400000B00BAA00D00CA500000EA000500F9BF4
:102E500000C01096005012910000148C00C015871D
:102E600000B0178200B0197D00D01B7800001E73DF
:102E70000040206E0090226900F024640040275F2B
:102E80000090295A00E02B5500102E500020304BA6
:102E90000010324600E033410090353C00103737D7
:102EA0000070383200A0392D00B03A2800A03B2332
:102EB00000603C1E00103D1900903D1400103E0FB4
:102EC00000703E0A00C03E0500003F0000403FFB8E
:102ED000FF803FF6FFC03FF1FF202D20496E766155
:102EE0006C6964206578747275646572206E756DA6
:102EF00062657220210A001000C90210012C0140F5
:102F000001220170011801B0010E01F0010401500D
:102F100002FA00B002F0003003E600D003DC0090BB
:102F200004D2007005C800A006BE000008B400B0BE
:102F300009AA00D00BA000600E960060118C000062
:102F400015820020197800C01D6E00A0226400B018
:102F5000275A00902C500000314600E0343C00100D
:102F6000383200903A2800603C1E00A03D140080DA
:102F70003E0A00203F0000453120544845524D4153
:102F80004C2052554E415741590042454420544827
:102F900045524D414C2052554E41574159005468BD
:102FA00065726D616C2052756E6177617900453193
:102FB000204572723A204D415854454D500045729B
:102FC000723A204D415854454D5020424544004DE1
:102FD000415854454D502074726967676572656445
:102FE000004531204572723A204D494E54454D50AE
:102FF000004572723A204D494E54454D502042458D
:1030000044004D494E54454D5020747269676765C0
:10301000726564000A0A0020205A5F4D494E3A004A
:103020002020595F4D494E3A002020585F4D494EAF
:103030003A004D383420582059205A204500202F7E
:10304000002042403A0020403A0020573A002057E2
:103050003A00496E76616C696420657874727564B3
:1030600065720A0020746F6F206C6F6E6720657840
:1030700074727573696F6E2070726576656E7465B3
:10308000640A0020636F6C642065787472757369DC
:103090006F6E2070726576656E7465640A0000005C
:1030A0000000000000000000000000004842000096
:1030B0004842000080405761726E696E673A20484E
:1030C0006F6D696E672042756D7020446976697313
:1030D0006F72203C20310A000202040000A0400070
:1030E00000A040000000400080ED430000E14300EC
:1030F00000EB43FFFFFF00000001000000010000A3
:103100008000555555000000400033333300AAAA13
:103110002A004992240000002000C7711C009999E0
:103120001900D1451700555515003BB1130024492E
:10313000120011111100000010000F0F0F00E338F2
:103140000E0043790D00CCCC0C00C3300C00E8A27B
:103150000B0064210B00AAAA0A00703D0A009DD84A
:103160000900427B090092240900DCD3080088880A
:1031700008001042080000000800F0C1070087871F
:10318000070075500700711C07003EEB0600A1BC4C
:1031900006006990060066660600703E060061182B
:1031A000060017F4050074D105005BB00500B2906D
:1031B0000500627205005555050078390500B81EF6
:1031C0000500050505004EEC040087D40400A1BDF0
:1031D000040090A7040049920400C17D0400EE6938
:1031E0000400C7560400444404005C320400082173
:1031F000040041100400000004003FF00300F8E068
:10320000030026D20300C3C30300CCB503003AA8D1
:1032100003000A9B0300388E0300C08103009F75E2
:103220000300D0690300505E03001D5303003448BF
:103230000300913D03003333030016290300381FB8
:10324000030097150300300C0300030303000BFA7F
:10325000020049F10200BAE802005CE002002DD849
:1032600002002DD0020059C80200B0C0020031B9DE
:103270000200DAB10200AAAA0200A0A30200BC9CCC
:103280000200FA9502005C8F0200DF880200828251
:103290000200457C02002776020027700200436A84
:1032A00002007C640200D05E02003F590200C85355
:1032B00002005A5F53544F505F50494E005A5F53BB
:1032C0005445505F50494E005A5F4D494E5F50493A
:1032D0004E005A5F454E41424C455F50494E005AA0
:1032E0005F4449525F50494E005A5F43535F504913
:1032F0004E00595F53544F505F50494E00595F5331
:103300005445505F50494E00595F4D494E5F5049FA
:103310004E00595F454E41424C455F50494E005961
:103320005F4449525F50494E00595F43535F5049D3
:103330004E00585F53544F505F50494E00585F53F2
:103340005445505F50494E00585F4D494E5F5049BB
:103350004E00585F454E41424C455F50494E005823
:103360005F4449525F50494E00585F43535F504994
:103370004E0053535F50494E00534552564F335FF2
:1033800050494E00534552564F325F50494E0053FC
:103390004552564F315F50494E00534552564F30BB
:1033A0005F50494E00534453530053445F444554C7
:1033B0004543545F50494E0053434B5F50494E00C4
:1033C00052414D50535F44395F50494E0052414D78
:1033D00050535F44385F50494E0052414D50535F47
:1033E0004431305F50494E004D4F53495F50494E74
:1033F000004D4F534645545F445F50494E004D4980
:10340000534F5F50494E004D4158363637355F5364
:10341000535F50494E004C45445F50494E0048456B
:10342000415445525F4245445F50494E0048454132
:103430005445525F305F50494E0046494C5F5255EB
:103440004E4F55545F50494E0046414E315F5049F2
:103450004E0046414E5F50494E0045315F53544542
:10346000505F50494E0045315F454E41424C455FEB
:1034700050494E0045315F4449525F50494E004526
:10348000315F43535F50494E0045305F53544550C0
:103490005F50494E0045305F454E41424C455F50BC
:1034A000494E0045305F4449525F50494E00453017
:1034B0005F43535F50494E00455F4D5558325F5052
:1034C000494E00455F4D5558315F50494E00455FAC
:1034D0004D5558305F50494E004245455045525F6A
:1034E00050494E004156525F53535F50494E004180
:1034F00056525F53434B5F50494E004156525F4D09
:103500004F53495F50494E004156525F4D49534F0A
:103510005F50494E0054454D505F4245445F50490D
:103520004E0054454D505F315F50494E0054454D5B
:10353000505F305F50494E0046494C57494454480B
:103540005F50494E005458440052584400205400E3
:10355000205200416363656C65726174696F6E3AF5
:1035600020500050574D3A20202534640050574DCC
:103570003A20202534640050574D3A2020253464E9
:103580000050574D3A20202534640050574D3A20C2
:10359000202534640050574D3A20202534640050D3
:1035A000574D3A20202534640050574D3A202025AD
:1035B00034640050574D3A20202534640050574D54
:1035C0003A20202534640050574D3A202025346499
:1035D0000050574D3A20202534640050574D3A2072
:1035E000202534640050574D3A2020253464005083
:1035F000574D3A20202534640050574D3A2020255D
:103600003464003A200020202020434F4D00202029
:10361000206E6F6E2D7374616E64617264205057FA
:103620004D206D6F646500202020636F6D706172A6
:103630006520696E7465727275707420656E616262
:103640006C6564002020206F766572666C6F772051
:10365000696E7465727275707420656E61626C65F6
:1036600064003A20002020202054494D534B004252
:103670003A2000202020205443435200413A2000A9
:103680002020202054434352002020202043533A3E
:1036900020002020202057474D3A200050574D3A17
:1036A00020202534640050574D3A202025346400F2
:1036B00047004800000088008A008C00B300B40076
:1036C000000098009A009C00A800AA00AC00280105
:1036D0002A012C012020202054494D45520044004D
:1036E00045006E00800081006F00B000B1007000E6
:1036F000900091007100A000A10072002001210142
:10370000730020697320616C736F20746965642095
:10371000746F20746869732070696E0054494D4558
:10372000523143000A202E002020002020506F72CA
:10373000743A200020202000202020416E616C6F10
:103740006720696E203D2025356C64003C756E75E0
:103750007365642F756E6B6E6F776E3E0020284127
:103760002532642920200025336420002573504928
:103770004E3A20004F7574707574203D2000496EDC
:1037800070757420203D2000416E616C6F67206968
:103790006E203D2025356C640070726F7465637413
:1037A000656420002028412532642920200025332B
:1037B000642000257350494E3A20004935000145E8
:1037C00035010138353B002D3543002235450015C4
:1037D00035440008353201FB343301EF343401E461
:1037E000343501D9342501CE342801C3342A01B837
:1037F000342C01AE342A01A3341C019534180189FC
:10380000341A017F342C017434220166341E015AAB
:1038100034240152340901493407013A3402012D9C
:10382000340A011E34080116340D0107344201FE2A
:10383000333201F1330701E8333301DA330A01CDC2
:10384000330801C0330901B8333401AA333101A56B
:103850003335019A330B018F330601843305017927
:1038600033040172333501693335015F3337015257
:10387000332601483303013D333601323303012936
:103880003331011F333D011233380108330E01FD7E
:10389000323C01F2320E01E9322801DF323001D22E
:1038A000323E01C8321301BD322E01B2321301443F
:1038B0006966663A200046726F6D5374703A005321
:1038C0007465707065723A00556E4C6576656C3A39
:1038D000004C6576656C65643A005261773A202049
:1038E0002020000A4C6F676963616C3A0043617085
:1038F0003A004261627973746570205A0050726FA9
:103900006265204F6666736574205A0050726F625C
:1039100065204F66667365745A3A2000290A0020B4
:10392000746F20003F5A206F7574206F662072619B
:103930006E6765202800290A0020746F20003F5917
:10394000206F7574206F662072616E676520282D68
:1039500000290A0020746F20003F58206F757420E2
:103960006F662072616E676520282D00205A002046
:10397000590050726F6265204F66667365742058F7
:1039800000220A00656E7175657565696E67202293
:10399000002E0A006F70656E206661696C65642C8C
:1039A0002046696C653A2000706F7765726F6666B5
:1039B000004B494C4C45442E20005072696E746592
:1039C000722068616C7465642E206B696C6C2829A8
:1039D0002063616C6C6564210A00000021002400F2
:1039E00027002A002D0030003300010100000401EF
:1039F00007010A0100002200250028002B002E00EC
:103A00003100340002010000050108010B01000033
:103A100020002300260029002C002F003200000186
:103A20000000030106010901050505050705080851
:103A30000808020202020A0A080804040404010138
:103A4000010101010101030303030303030304074D
:103A500007070C0C0C0C0C0C0C0C020202020606E4
:103A60000606060606060B0B0B0B0B0B0B0B0102D7
:103A70001020200808102040102040800201020180
:103A80000804020101020408102040808040201038
:103A90000804020180040201804020100804020191
:103AA00008040201010204081020408001020408F9
:103AB0001020408000000A0B02090C0D0E080703BD
:103AC00004010000000000000000000000000000F1
:103AD00000000000000000000000000000000000E6
:103AE00012111000000000000000000000000000A3
:103AF0000000000000000000000050726F62696E5C
:103B000067204661696C65640A0050726F62696E75
:103B100067204661696C656400205A3A200020598C
:103B20003A200042656420583A200053544F5050C8
:103B300045442E20005072696E7465722073746F54
:103B4000707065642064756520746F206572726F93
:103B500072732E2046697820746865206572726FD2
:103B60007220616E6420757365204D393939207477
:103B70006F20726573746172742E202854656D70A5
:103B800065726174757265206973207265736574FE
:103B90002E205365742069742061667465722072EA
:103BA000657374617274696E67290A006563686F72
:103BB0003A004572726F723A0042696C696E6561D3
:103BC00072204C6576656C696E6720477269643A4D
:103BD0000A00544D3344204D617820526561647968
:103BE0002E005072696E74696E672E2E2E00507210
:103BF000696E74205061757365640063616E6365FE
:103C00006C005072696E742041626F72746564005A
:103C10004469736D6973730055492041626F727412
:103C2000656400726573756D65004D323400008007
:103C3000ED430000E1430000EB4300000000000002
:103C4000000000000000626564002C20737973742A
:103C5000656D2073746F70706564212048656174B0
:103C600065725F49443A200042656420486561748A
:103C7000696E67204661696C6564004865617469B6
:103C80006E67206661696C65640042454420544853
:103C900045524D414C2052554E41574159005468B0
:103CA00065726D616C2052756E6177617900453186
:103CB0002048656174696E67204661696C656400BF
:103CC00048656174696E67206661696C656400456A
:103CD0003120544845524D414C2052554E41574198
:103CE0005900546865726D616C2052756E61776120
:103CF00079004F46460A0046616465204865696759
:103D000068742000426564204C6576656C696E6756
:103D100020004661696C656420746F20656E616285
:103D20006C6520426564204C6576656C696E670A37
:103D300000496E76616C6964206D6573682E0A00B7
:103D40008D01D10111241FBECFEFD1E2DEBFCDBF67
:103D500000E00CBF18E0A0E0B2E0E2E8FBE502E022
:103D60000BBF02C007900D92A231B107D9F72DE128
:103D7000A2E1B8E001C01D92AA3FB207E1F71EE13F
:103D8000C1EADEE100E006C021970109802FFE01B3
:103D90000F94EA29C03AD10780E00807A9F70F94E9
:103DA0009B130D94AF2D0C9400002F923F924F92D5
:103DB0005F926F927F928F929F92AF92BF92CF92BB
:103DC000DF92EF92FF920F931F93CF93DF93CDB7C4
:103DD000DEB7A7970FB6F894DEBF0FBECDBF8091B8
:103DE0000901817091E0982720913108921781F1A3
:103DF00090933108811116C00E9487768091181720
:103E000083FF09C08BE993E00E94E55461E080E004
:103E10000F9413071DC060E081E00F94130784EB3B
:103E200093E014C00091181703FB002700F90E94CB
:103E3000167680911817877F80931817002341F01A
:103E400060E081E00F9413078DEC93E00E94E5544D
:103E50008091300881110C94493A80912E089091FC
:103E60002F089C012F5F3F4F30932F0820932E087F
:103E7000883E934010F40C94493A81E080933008D6
:103E800010922F0810922E0880919B0B882309F422
:103E90008CC30E941EAF811188C380912D088F5F53
:103EA00080932D0880912D08853620F010922D08E2
:103EB00010929B0BE0919B0B8E2FEE0F990BAA0B90
:103EC000BB0BFC013197E730F10508F0A0C0882753
:103ED000EE58FF4F8F4F0D94EA290E9416AF8823AA
:103EE00009F495C081E08093260280EE93E00E9461
:103EF000E55480E190E090939D1580939C1585E0BA
:103F00008093901502E80093931584E190E1A0E07E
:103F1000B0E08093941590939515A0939615B09367
:103F200097150E942FF581E09AE590939D15809357
:103F30009C1586E390E090939F1580939E1587E0F3
:103F4000809390150093931584E890E0A0E0B0E092
:103F50008093941590939515A0939615B09397150B
:103F60000E942FF552C00E9416AF882309F44FC05B
:103F700048C08EEE93E00E94E55481E09AE590936C
:103F80009D1580939C1580E490E090939F158093FD
:103F90009E1507E00093901582E88093931584E8BE
:103FA00090E0A0E0B0E08093941590939515A093D5
:103FB0009615B09397150E942FF500939B0B27C081
:103FC00080912C08882319F10E9416AF8823F9F0FC
:103FD0000E941EAF81111BC0EBC20E9416AF882346
:103FE000B1F00E941EAF811112C010C30E941EAF1B
:103FF00081110DC042E060E070E0CB010E9434AF5F
:1040000004C00E941EAF811102C010929B0B8091D0
:104010002602882309F4B1C28091970B9091980BE6
:10402000892B09F08FC18091290890912A08892B4A
:1040300009F01EC184E096E090939D1580939C1535
:1040400080EA90E890939F1580939E1517E0109357
:10405000901502E80093931580EA90E0A0E0B0E0AC
:104060008093941590939515A0939615B0939715FA
:104070000E942FF58091020290910302A091040208
:10408000B09105020097A105B10511F510929D159B
:1040900010929C1515E010939015009393158AE8E3
:1040A00090E1A0E0B0E08093941590939515A093D3
:1040B0009615B09397150E942FF589E090E09093A4
:1040C0009D1580939C15109390150093931540C0F7
:1040D0000196A11DB11D65E0B695A79597958795A9
:1040E0006A95D1F70197A109B109009721E0A207CC
:1040F000B10558F0B0939D15A0939C1590939F1512
:1041000080939E151093901507C090939D158093F2
:104110009C1585E08093901512E8109393158AE81A
:1041200090E1A0E0B0E08093941590939515A09352
:104130009615B09397150E942FF588E090E0909324
:104140009D1580939C1585E0809390151093931591
:104150008CE890E1A0E0B0E08093941590939515E1
:10416000A0939615B09397150E942FF580910202A7
:1041700090910302A0910402B0910502009731E0F2
:10418000A307B10550F0B0939D15A0939C15909393
:104190009F1580939E1587E005C090939D15809391
:1041A0009C1585E08093901582E88093931588E8AC
:1041B00090E1A0E0B0E08093941590939515A093C2
:1041C0009615B09397150E942FF580910202909159
:1041D0000302A0910402B0910502BA2FA92F982FD3
:1041E00088270097E1E0AE07B10550F0B0939D1528
:1041F000A0939C1590939F1580939E1587E005C012
:1042000090939D1580939C1585E08093901512E8FE
:104210001093931581EA90E0A0E0B0E080939415AC
:1042200090939515A0939615B09397150E942FF52E
:1042300080911E18882319F082E090E002C083E08C
:1042400090E090939D1580939C1585E08093901548
:104250001093931585E490E1A0E0B0E0809394156D
:1042600090939515A0939615B09397150E942FF5EE
:104270000091290810912A08053611057CF4109345
:104280009D1500939C1585E08093901582E880939E
:10429000931580E090E1A0E0B0E011C0C801845621
:1042A000910990939D1580939C1585E080939015BE
:1042B00082E88093931581E090E1A0E0B0E08093E4
:1042C000941590939515A0939615B09397150E9409
:1042D0002FF50F5F1F4F10932A0800932908093C00
:1042E000110564F18CEF93E00E94E55481E090E0C9
:1042F0009093980B8093970B8093260281E09AE528
:1043000090939D1580939C158DE290E090939F155E
:1043100080939E1587E08093901582E88093931593
:1043200084E890E0A0E0B0E0809394159093951518
:10433000A0939615B09397150E942FF51092300810
:104340000C94493A8091FE149091FF14891B8F7050
:1043500009F0DAC10E947F518111D6C180911817EE
:1043600082FDD2C17DC184E690E090939D1580933B
:104370009C1510939015009393158EE090E1A0E0AA
:10438000B0E08093941590939515A0939615B093F3
:1043900097150E942FF5C60182539048880F991FE8
:1043A00090939D1580939C151093901500939315F1
:1043B0008FE090E1A0E0B0E0809394159093951584
:1043C000A0939615B09397150E942FF50F94E405CE
:1043D00090E090939D1580939C1585E080939015B7
:1043E00082E88093931586E190E1A0E0B0E08093AD
:1043F000941590939515A0939615B09397150E94D8
:104400002FF520E030E048EC52E460918A1770917B
:104410008B1780918C1790918D170F9463230F94B5
:104420005F2B70939D1560939C1515E0109390156C
:1044300002E80093931586E290E1A0E0B0E080935B
:10444000941590939515A0939615B09397150E9487
:104450002FF520E030E0A9016091E00B7091E10BB5
:104460008091E20B9091E30B0F94F3290F945F2B53
:1044700070939D1560939C15109390150093931560
:1044800086E390E1A0E0B0E08093941590939515B9
:10449000A0939615B09397150E942FF56091E708A9
:1044A0007091E8088091E9089091EA080F945F2BD9
:1044B00070939D1560939C15109390150093931520
:1044C0008CE390E1A0E0B0E0809394159093951573
:1044D000A0939615B09397150E942FF58091E40B49
:1044E0009091E50B90939D1580939C1510939015DA
:1044F0000093931584E390E1A0E0B0E080939415DD
:1045000090939515A0939615B09397150E942FF54B
:104510008091EB089091EC0890939D1580939C15E9
:1045200010939015009393158AE390E1A0E0B0E01A
:104530008093941590939515A0939615B093971525
:104540000E942FF50091250801117FC18091270855
:1045500081117BC180912C0881113CC2809144154E
:1045600090914515A0914615B09147158C34F0E116
:104570009F07A105B10509F052C280EEC82E85E162
:10458000D82E0AE18AE793E10E946974E0901A0844
:10459000F0901B08181619060CF09DC31AE1E116DD
:1045A000F10414F40C94E93596C310922D087ACCDA
:1045B0008EEA95E00E94E55480912B0890E0A0E0FF
:1045C000B0E0895B9F4FAE4FB54A21E03AE53093AA
:1045D0009D1520939C1590939F1580939E1587E0C1
:1045E0008093901582E88093931584E890E0A0E092
:1045F000B0E08093941590939515A0939615B09381
:1046000097150E942FF510922C08FFCC81E0809323
:10461000260210929B0B8CEB95E00E94E55481E002
:104620009AE590939D1580939C158EE490E090936D
:104630009F1580939E1587E08093901582E8809364
:10464000931584E890E0A0E0B0E0809394159093F7
:104650009515A0939615B09397150E942FF5D7CC7A
:104660000091E7081091E8082091E9083091EA08E4
:1046700008A319A32AA33BA36091EB087091EC084F
:10468000072E000C880B990B0F9404236B017C01FF
:1046900020E030E040E850E40F94F22928A139A14D
:1046A0004AA15BA10F94532C18160CF433C220E0DE
:1046B00030E0A9016091E00B7091E10B8091E20B79
:1046C0009091E30B0F94F3296CA37DA38EA39FA37A
:1046D0006091E40B7091E50B072E000C880B990B91
:1046E0000F9404234B015C0120E030E040E251E4F0
:1046F0000F94F2292CA13DA14EA15FA10F94532C40
:1047000018160CF407C226C28CE090E090939D1519
:1047100080939C1505E00093901582E88093931593
:1047200084E190E1A0E0B0E080939415909395151A
:10473000A0939615B09397150E942FF50F9411042E
:1047400020E13EE040E050E00F945329211531056F
:1047500011E04107510560F050939D1540939C1561
:1047600030939F1520939E1587E08093901506C087
:1047700030939D1520939C150093901502E80093AB
:10478000931580E190E1A0E0B0E0809394159093C0
:104790009515A0939615B09397150E942FF50F9439
:1047A000110420E13EE040E050E00F9453292CE357
:1047B00030E040E050E00F94532930939D15209352
:1047C0009C1515E0109390150093931582E190E1EC
:1047D000A0E0B0E08093941590939515A093961562
:1047E000B09397150E942FF50F94E405882391F05C
:1047F0000F94E4058F5F80932808C82ED12C833353
:1048000008F0B1CDC601880F991F90939D15809334
:104810009C1504C010929D1510929C151093901534
:10482000009393158EE090E1A0E0B0E080939415A2
:1048300090939515A0939615B09397150E942FF518
:1048400010929D1510929C15AFCD20E030E0A9018B
:104850006091E00B7091E10B8091E20B9091E30B82
:104860000F94F32920E030E048EC52E40F946323E6
:104870006B017C016091E40B7091E50B072E000C3D
:10488000880B990B0F9404239B01AC01C701B6015F
:104890000F94ED2A0F94662B6436710510F064E6D0
:1048A00070E070939D1560939C1595E0A92EA092E1
:1048B000901522E8B22EB092931584E290E1A0E028
:1048C000B0E08093941590939515A0939615B093AE
:1048D00097150E942FF520E030E0A9016091E00BD0
:1048E0007091E10B8091E20B9091E30B0F94F3290F
:1048F0006B017C0120E030E04AE253E40F94532C3A
:1049000018160CF069C1002309F466C1109225083D
:1049100020E030E040E251E460911D0870911E08F3
:1049200080911F08909120080F9463230F945F2BB0
:1049300070939D1560939C15A0929015B09293155D
:1049400084E590E1A0E0B0E08093941590939515F4
:10495000A0939615B09397150E942FF520E030E0B4
:1049600040E251E46091210870912208809123086F
:10497000909124080F9463230F945F2B70939D15DF
:1049800060939C15A0929015B092931588E590E1E4
:10499000A0E0B0E08093941590939515A0939615A0
:1049A000B09397150E942FF58AEC95E00E94E5548C
:1049B00081E09AE590939D1580939C1581E490E0A9
:1049C00090939F1580939E1587E080939015B092E9
:1049D000931551C180911C0801E0080F00931C0839
:1049E00090E090939D1580939C1585E080939015A1
:1049F00082E88093931582E490E1A0E0B0E0809398
:104A0000941590939515A0939615B09397150E94C1
:104A10002FF50A3008F4A2CD10921C089FCD8A34DD
:104A20009041A105B10509F4A8CD20E030E040E2B5
:104A300051E46091061870910718809108189091C0
:104A400009180F9463230F945F2B70939D15609347
:104A50009C1515E01093901502E80093931588E4D7
:104A600090E1A0E0B0E08093941590939515A09309
:104A70009615B09397150E942FF520E030E040E2A4
:104A800051E460910A1870910B1880910C18909164
:104A90000D180F9463230F945F2B70939D156093F3
:104AA0009C1510939015009393158AE490E1A0E073
:104AB000B0E08093941590939515A0939615B093BC
:104AC00097150E942FF520E030E040E251E460911C
:104AD0000E1870910F1880911018909111180F9462
:104AE00063230F945F2B70939D1560939C15109317
:104AF0009015009393158CE490E1A0E0B0E08093D2
:104B0000941590939515A0939615B09397150E94C0
:104B10002FF533CD8DE090E090939D1580939C15FB
:104B200085E08093901582E88093931584E190E16D
:104B3000A0E0B0E08093941590939515A0939615FE
:104B4000B09397150E942FF580919A0B811141C067
:104B500081E03FC020E030E040E850E4C701B6010A
:104B60000F94F32928A139A14AA15BA10F94FD223A
:104B700087FD10C020E030E040E251E4C501B401FF
:104B80000F94F3292CA13DA14EA15FA10F94FD220A
:104B900087FF37CC84E190E090939D1580939C151E
:104BA00085E08093901582E88093931584E190E1ED
:104BB000A0E0B0E08093941590939515A09396157E
:104BC000B09397150E942FF580919A0B811101C027
:104BD00082E080939A0B15CC6091E40B7091E50B09
:104BE000072E000C880B990B0F9404239B01AC013A
:104BF000C701B6010F94532C6091270887FD4AC066
:104C0000662309F4A7CC062E000C770B8EE297E002
:104C10000F9400031092270810922A081092290876
:104C200084E090E090939D1580939C1585E080939F
:104C3000901502E8009393158EE890E1A0E0B0E0B3
:104C40008093941590939515A0939615B09397150E
:104C50000E942FF581E09AE590939D1580939C1515
:104C600083E590E090939F1580939E1587E0809355
:104C700090150093931584E890E0A0E0B0E0809355
:104C8000941590939515A0939615B09397150E943F
:104C90002FF560CC662309F45DCC809129089091B2
:104CA0002A089C012F5F3F4F30932A082093290840
:104CB00065E070E00F94D62990939D1580939C1524
:104CC00085E08093901582E8809393158EE890E1BB
:104CD000A0E0B0E0D4CF1E141F040CF02FCB9091B5
:104CE00041158091E015981322C090914215809152
:104CF000E11598131CC003E0E016F104C4F0909194
:104D0000E215909340158091E315809343159330FD
:104D1000D1F4982F9D7F9038B1F49091E4159F3491
:104D200009F05FC09091E5159B3409F05AC08AE103
:104D3000E0EEF5E1DF011D928A95E9F710921B087C
:104D400010921A08FBCA833809F04BC08091E41511
:104D50009091E515982789279827A0E0B0E08093E7
:104D6000441590934515A0934615B093471540916F
:104D7000E61550E060E070E0409348155093491507
:104D800060934A1570934B1507EEA02E05E1B02EE7
:104D900080E090E0DC0184179507A607B70708F0CC
:104DA0004EC06C017D01F694E794D794C7949601A8
:104DB0002A5F3F4F220F331FF901E05CFA4E7F015B
:104DC000F501208130E0322F22270181202BF701CD
:104DD000318320830296A11DB11DF2E0AF0EB11CFC
:104DE000DACF813861F58091E41590E0A0E0B0E081
:104DF0008093441590934515A0934615B09347159D
:104E00008091E515482F50E060E070E04093481530
:104E10005093491560934A1570934B15A6EEB5E172
:104E2000ECE4F5E190E020E030E02817390739F0B4
:104E30004D9150E0419351932F5F3F4FF6CF8AE160
:104E4000E0EEF5E1DF011D928A95E9F710921B086B
:104E500010921A088DE094E00E94E55460919B0B3B
:104E6000161664F4062E000C770B83E297E00F947D
:104E700000038AE00E94DA530C94DA3560914C15F5
:104E800070914D1581E197E00F94E2028AE00E9453
:104E9000DA53409144155091451560914615709133
:104EA000471582E097E00F94D1028AE00E94DA531E
:104EB0008091441590914515A0914615B0914715E4
:104EC000E5E7F2E000E010E04191519161917191CC
:104ED0004115510561057105D1F1481759076A0758
:104EE0007B0791F5AC01BD01485050416109710942
:104EF000453051056105710568F1AC01BD01477F81
:104F0000423350416105710541F18433F0E19F075F
:104F1000A105B10511F1AC01BD0146545041610933
:104F200071094730510561057105D0F0AC01BD0133
:104F300044555041610971094530510561057105BC
:104F400088F402E110E00EC00F5F1F4FBDCF0FEFDE
:104F50001FEF08C003E010E005C008E010E002C049
:104F60000FE010E08A509042A109B109833D9105FC
:104F7000A105B10530F00F3F2FEF120721F40C947B
:104F8000DA3509E110E0AEE2CA2EA4E0DA2EF6012D
:104F900081916F01882319F00E94DA53F8CFB8018C
:104FA000012E000C880B990B0E944E540E94DF5476
:104FB00086EF96E00E94E5540A31110510F00C943A
:104FC000D635F8018827E758FF4F8F4F0D94EA290F
:104FD00080914C1590914D1581309105E1F410921E
:104FE00026028FEF80937D1A60E080E00F94130714
:104FF0000CE314E0D8018D918D01882319F00E94F3
:10500000DA53F8CF81E09AE590939D1580939C1533
:105010008EE290E0AFC08230910509F0C5C081E01A
:10502000809326020F94550682EF96E09093200914
:1050300080931F098BE090E090939D1580939C15C1
:1050400005E00093901512E81093931580E092E12B
:10505000A0E0B0E08093941590939515A0939615D9
:10506000B09397150E942FF510929D1510929C15E4
:1050700000939015109393158EE090E1A0E0B0E0BE
:105080008093941590939515A0939615B0939715CA
:105090000E942FF510929D1510929C15009390156B
:1050A000109393158FE090E1A0E0B0E08093941509
:1050B00090939515A0939615B09397150E942FF590
:1050C00010929D1510929C150093901510939315B6
:1050D00086E190E1A0E0B0E080939415909395155F
:1050E000A0939615B09397150E942FF562E070E09B
:1050F00080E090E00E94F8AF10929D1510929C15F0
:10510000009390151093931580E190E1A0E0B0E03A
:105110008093941590939515A0939615B093971539
:105120000E942FF510929D1510929C1500939015DA
:105130001093931582E190E1A0E0B0E08093941584
:1051400090939515A0939615B09397150E942FF5FF
:1051500006E614E0F80181918F01882319F00E947E
:10516000DA53F8CF81E09AE590939D1580939C15D2
:105170008DE290E090939F1580939E1587E0809339
:10518000901582E88093931584E890E0A0E0B0E069
:105190008093941590939515A0939615B0939715B9
:1051A0000E942FF50C94DA358330910549F581E0A2
:1051B0008093260200E914E0D8018D918D018823A7
:1051C000C9F00E94DA53F8CF8091441590914515AB
:1051D000A0914615B0914715823330E19307A105A0
:1051E000B10509F077C480914C1590914D15009749
:1051F00009F035C480910102882309F405C315C361
:10520000049711F00C94DA35109226020C94DA35DA
:1052100080914C1590914D1581309105D1F41092EB
:10522000260280910102882319F082E090E002C0FA
:1052300083E090E090939D1580939C1585E080938A
:10524000901582E8809393158EE190E1A0E0B0E0A4
:105250009FCF8230910519F50AEB14E0F801819196
:105260008F01882319F00E94DA53F8CF81E08093F0
:10527000260280919A0B843049F081E09AE5909360
:105280009D1580939C1585E390E074CF81E09AE5AD
:1052900090939D1580939C1586E390E06BCF8330AF
:1052A000910509F04CC020910102222319F190933D
:1052B0009D1580939C1585E08093901582E88093DE
:1052C00093158EE190E1A0E0B0E080939415909367
:1052D0009515A0939615B09397150E942FF540E071
:1052E00060E070E088EC92E40F94C4061092010232
:1052F0000C94DA3582E090E090939D1580939C1594
:1053000085E08093901582E8809393158EE190E17B
:10531000A0E0B0E08093941590939515A093961516
:10532000B09397150E942FF540E060E070E0CB014C
:105330000F94C40681E0809301020C94DA3504973F
:1053400011F00C94DA358091FA088823F1F082E0AC
:1053500090E090939D1580939C1585E08093901527
:1053600082E8809393158FE190E1A0E0B0E0809314
:10537000941590939515A0939615B09397150E9448
:105380002FF51092FA080C94DA3583E090E09093B0
:105390009D1580939C1585E08093901582E88093FD
:1053A00093158FE190E1A0E0B0E080939415909385
:1053B0009515A0939615B09397150E942FF581E04F
:1053C0008093FA080C94DA3500914C1510914D1524
:1053D000B80180E090E00F9402236B017C0120E093
:1053E00030E040E251E40F94FD2287FD0DC020E043
:1053F00030E04AEF53E4C701B6010F94532C18165E
:1054000034F0902F812F05C09AE080E002C094EF25
:1054100081E090935502809356020C94DA35809186
:10542000441590914515A0914615B09147158830C7
:10543000F0E19F07A105B10509F050C081E09AE5B0
:1054400090939D1580939C158DE290E090939F150D
:1054500080939E1587E08093901512E81093931522
:1054600084E890E0A0E0B0E08093941590939515C7
:10547000A0939615B09397150E942FF510929D1545
:1054800010929C1505E0009390151093931580E100
:1054900090E1A0E0B0E08093941590939515A093CF
:1054A0009615B09397150E942FF510929D151092A6
:1054B0009C15009390151093931582E190E1A0E064
:1054C000B0E08093941590939515A0939615B093A2
:1054D00097150E942FF50F9455068FC08A3000E172
:1054E0009007A105B105E1F580914C1590914D15FE
:1054F000813F910511F00C94DA3581E09AE59093A3
:105500009D1580939C1586E390E090939F15809362
:105510009E1587E08093901582E88093931584E828
:1055200090E0A0E0B0E08093941590939515A0933F
:105530009615B09397150E942FF541E755E068E75F
:1055400075E084E00E940DBC60E08EEE9BE30F945A
:10555000160687E695E09093200980931F094DC0B9
:105560008C309041A105B10509F047C080914C15E0
:1055700090914D15019709F040C00F94B91D1092FC
:105580009A0B81E0809326028CE090E090939D1529
:1055900080939C1585E08093901512E810939315E5
:1055A00084E190E1A0E0B0E080939415909395158C
:1055B000A0939615B09397150E942FF581E09AE578
:1055C00090939D1580939C1585E390E090939F1593
:1055D00080939E1587E0809390151093931584E82F
:1055E00090E0A0E0B0E08093941590939515A0937F
:1055F0009615B09397150E942FF5809144159091C0
:105600004515A0914615B09147158C309041A105E4
:10561000B10511F00C94DA3580914C1590914D152F
:10562000029711F00C94DA350F94B91D81E0809344
:10563000270810929A0B8093260210922A08109243
:10564000290881E09AE590939D1580939C1582E549
:1056500090E090CD20914C1530914D15B90180E02E
:1056600090E037FF09C00F94022320E030E040E8CB
:1056700057E40F94F22902C00F94022320E030E097
:1056800048EC52E40F94ED2A6B017C0120E030E0FD
:1056900040EA51EC0F94532C87FD31C020E030E0FC
:1056A00040EA51E4C701B6010F94FD2218163CF1FF
:1056B000A701960160918A1770918B1780918C17C2
:1056C00090918D170F94F22920E030E048EC53E4DC
:1056D0000F94632390580F945F2BCB010E948DF899
:1056E000C0928A17D0928B17E0928C17F0928D1788
:1056F0008DEE96E09093200980931F0928C020E04A
:1057000030E048EC52E460918A1770918B178091D9
:105710008C1790918D170F9463230F945F2B7093C8
:105720009D1560939C1585E08093901582E8809389
:10573000931586E290E1A0E0B0E0809394159093F9
:105740009515A0939615B09397150E942FF560912B
:105750008A1770918B1780918C1790918D178E01FD
:105760000B5E1F4F23E041E00F94D51D9F938F9355
:105770008FED96E09F938F93045111091F930F9320
:105780000F949522C8010E94D2B00F900F900F90F5
:105790000F900F900F900C94DA3580914C159091EA
:1057A0004D15009729F481E0809326020C94DA3598
:1057B00081309105B1F480910102882349F081E0A4
:1057C0009AE590939D1580939C158CE390E0D2CC44
:1057D00081E09AE590939D1580939C158BE390E072
:1057E000C9CC82309105F9F28330910539F5809169
:1057F000010240E0882389F060E070E088EC92E4E8
:105800000F94C4061092010281E09AE590939D15D1
:1058100080939C1589E390E0ADCC60E070E0CB0113
:105820000F94C40681E08093010281E09AE5909391
:105830009D1580939C158AE390E09CCC8530910562
:1058400099F50F94090784EB90E00E9451D71092CC
:10585000FE121092FF121092001310920113109278
:1058600002130E94A8D686E490E00E94456984EB6A
:1058700090E090939D1580939C1505E00093901502
:1058800012E81093931584E390E1A0E0B0E08093D8
:10589000941590939515A0939615B09397150E9423
:1058A0002FF586E490E035C086309105D9F50F9448
:1058B000090780EF90E00E9451D71092FE121092DB
:1058C000FF121092001310920113109202130E9403
:1058D000A8D68EE690E00E94456980EF90E0909314
:1058E0009D1580939C1505E00093901512E8109388
:1058F000931584E390E1A0E0B0E080939415909339
:105900009515A0939615B09397150E942FF58EE6E6
:1059100090E090939D1580939C15009390151093A3
:105920009315D3C0813F910511F00C94DA3540E016
:1059300060E070E0CB010F94C40641E060E070E0ED
:10594000CB010F94C406109201020F94090780E066
:1059500090E00E9451D71092FE121092FF12109206
:10596000001310920113109202130E94A8D680E037
:1059700090E00E94456910929D1510929C1505E0DB
:105980000093901512E81093931584E390E1A0E042
:10599000B0E08093941590939515A0939615B093CD
:1059A00097150E942FF561E070E080E090E00E9482
:1059B000F8AF10929D1510929C15009390151093BE
:1059C00093158AE390E1A0E0B0E080939415909362
:1059D0009515A0939615B09397150E942FF561E049
:1059E00070E080E090E00E94F8AF84E190E0909356
:1059F0009D1580939C15009390151093931584E149
:105A000090E1A0E0B0E08093941590939515A09359
:105A10009615B09397150E942FF581E09AE5909323
:105A20009D1580939C1589E390E090939F1580933A
:105A30009E1587E0809390151093931584E890E06D
:105A4000A0E0B0E08093941590939515A0939615DF
:105A5000B09397150E942FF582E00C94D3358130D6
:105A60009105A9F40F94090780E090E00E9451D7B6
:105A700010929D1510929C1585E08093901582E8F8
:105A80008093931584E390E1A0E0B0E081CB02978E
:105A900011F00C94DA351092FE121092FF1210924F
:105AA000001310920113109202130E94A8D680E0F6
:105AB00090E00E94456910929D1510929C1585E01A
:105AC0008093901582E8809393158AE390E1A0E09B
:105AD000B0E05ECB8433E0E19E07A105B105D9F4C7
:105AE00000914C1510914D150F940907B80180E0F5
:105AF00090E00F94022320E030E046E953E40F9455
:105B0000532C181614F0C80102C08CE291E00E94D8
:105B100051D70C94DA358A339041A105B10511F0C3
:105B20000C94DA3500914C1510914D151092FE121F
:105B30001092FF1210920013109201131092021390
:105B40000E94A8D6B80180E090E00F94022320E0E4
:105B500030E04CE053E40F94532C181614F0C801B5
:105B600002C08CE890E00E9445690C94DA3580917F
:105B70004C1590914D15009709F415CE8130910583
:105B800009F04CC080911E18882319F083E090E042
:105B900002C082E090E090939D1580939C1585E073
:105BA0008093901582E88093931585E490E1A0E0BE
:105BB000B0E08093941590939515A0939615B093AB
:105BC00097150E942FF58AE090E090939D158093A1
:105BD0009C1585E08093901582E88093931580E072
:105BE00092E1A0E0B0E08093941590939515A09376
:105BF0009615B09397150E942FF50E9416AF81114C
:105C000003C08FEC96E002C083EC96E090932009ED
:105C100080931F0982E080939B0B85C182309105A0
:105C200009F0ADC081E08093260288E0EDE1F8E064
:105C3000DF011D928A95E9F780E090E0A0E2B1E4EF
:105C400080931D0890931E08A0931F08B09320080E
:105C50008093210890932208A0932308B0932408EE
:105C600084E690E090939D1580939C1505E0009349
:105C7000901512E81093931584E590E1A0E0B0E050
:105C80008093941590939515A0939615B0939715BE
:105C90000E942FF520E030E040E251E460912108BD
:105CA0007091220880912308909124080F94632317
:105CB0000F945F2B70939D1560939C150093901526
:105CC0001093931588E590E1A0E0B0E080939415DF
:105CD00090939515A0939615B09397150E942FF564
:105CE00020E030E0A9016091E00B7091E10B809120
:105CF000E20B9091E30B0F94F3290F945F2B7093B9
:105D00009D1560939C15009390151093931586E351
:105D100090E1A0E0B0E08093941590939515A09346
:105D20009615B09397150E942FF58091E40B9091F2
:105D3000E50B90939D1580939C15009390151093FF
:105D4000931584E390E1A0E0B0E0809394159093E4
:105D50009515A0939615B09397150E942FF562E0C4
:105D600070E080E090E00E94F8AF81E09AE59093C7
:105D70009D1580939C1581E490E00C941637833038
:105D8000910509F085C010922B0820E030E040E238
:105D900051E460910618709107188091081890914D
:105DA00009180F9463230F945F2B70939D156093D4
:105DB0009C1505E00093901512E81093931588E464
:105DC00090E1A0E0B0E08093941590939515A09396
:105DD0009615B09397150E942FF520E030E040E231
:105DE00051E460910A1870910B1880910C189091F1
:105DF0000D180F9463230F945F2B70939D15609380
:105E00009C1500939015109393158AE490E1A0E0FF
:105E1000B0E08093941590939515A0939615B09348
:105E200097150E942FF520E030E040E251E46091A8
:105E30000E1870910F1880911018909111180F94EE
:105E400063230F945F2B70939D1560939C150093B3
:105E50009015109393158CE490E1A0E0B0E080934E
:105E6000941590939515A0939615B09397150E944D
:105E70002FF562E070E080E090E00E94F8AF81E0F2
:105E80009AE590939D1580939C1587E490E0CEC78A
:105E90008430910509F48EC68530910549F44EE7AA
:105EA00050E160E070E081EE94E00E94EDF582C682
:105EB000069709F07FC68FEB96E0909320098093B8
:105EC0001F098BE090E02BC280914C1590914D15ED
:105ED000019711F51092260281E09AE590939D15A5
:105EE00080939C158FE390E090939F1580939E156F
:105EF00087E08093901582E88093931584E890E082
:105F0000A0E0B0E08093941590939515A09396151A
:105F1000B09397150E942FF580914C1590914D15D7
:105F2000029709F047C681E09AE590939D1580930A
:105F30009C1580E490E01EC9E0914C15F0914D1540
:105F40003197EB30F10508F0E4C18827ED56FF4F9B
:105F50008F4F0D94EA298091781380FF65C686954E
:105F600080FD65C661C62DEC3CEC4CEC5DE36091B8
:105F70008A1770918B1780918C1790918D170F94C1
:105F8000F3296B017C0120E030E040EA51EC0F94F2
:105F9000532C87FDC2C120E030E040EA51E4C70144
:105FA000B6010F94FD2218160CF048C6B6C12DECB0
:105FB0003CEC4CEC5DE360918A1770918B178091FB
:105FC0008C1790918D170F94F2296B017C0120E0C2
:105FD00030E040EA51EC0F94532C87FD9EC120E045
:105FE00030E040EA51E4C701B6010F94FD221816D3
:105FF0000CF09BC692C180E00E9435C00E9416AF93
:10600000811103C086E696E002C088E596E0909391
:10601000200980931F0982E080939B0B81E09AE521
:1060200090939D1580939C1584E590E090939F1527
:1060300080939E1587E08093901582E88093931556
:1060400084E890E0A0E0B0E08093941590939515DB
:10605000A0939615B09397150E942FF55EC183E02B
:1060600080939B0B83E090E090939D1580939C150B
:1060700085E08093901582E8809393158DE890E1F8
:10608000A0E0B0E08093941590939515A093961599
:10609000B09397150E942FF5E12CF12C00E0DD2440
:1060A000D394AA24A39475E0972EE5E08E2EF2E80F
:1060B0007F2EDD2031F0CC24C39465E0B62E10E0B5
:1060C00005C0CC24CA94BB24BA9414E0DA24B116D7
:1060D000D1F1802F90E04897A4F50F5FF701919ED2
:1060E000E00DF11D1124EE0FFF1FEE0FFF1FE35710
:1060F000FD4E20E030E04AE754E460817181828106
:1061000093810F9463230F945F2B70939D1560937D
:106110009C158092901570929315802F90E0815875
:10612000974F880F991F092E000CAA0BBB0B809369
:10613000941590939515A0939615B09397150E947A
:106140002FF51C0DC4CFBFEFEB1AFB0AE5E0EE16EE
:10615000F10409F0AECF81E09AE590939D1580930C
:106160009C1585E590E090939F1580939E1587E0A0
:106170008093901582E88093931584E890E0A0E0E6
:10618000B0E08093941590939515A0939615B093D5
:1061900097150E942FF58AEF95E090932009809340
:1061A0001F09BBC042E060E070E080E890E40E941C
:1061B00034AF40E060E070E08DE693E40E9434AFDD
:1061C00041E060E070E081E693E413C042E060E00B
:1061D00070E080E890E40E9434AF40E060E070E05E
:1061E00080EB91E40E9434AF41E060E070E080EB2E
:1061F00091E40E9434AF86E080939B0B8EC042E016
:1062000060E070E080E890E40E9434AF40E060E03D
:1062100070E882EE93E4E6CF42E060E070E080E870
:1062200090E40E9434AF40E060E070E882EE93E4D6
:106230000CC042E060E070E080E890E40E9434AF7F
:1062400040E060E070E080EB91E40E9434AF41E018
:1062500060E070E086ED93E4CCCF80911E18811150
:106260001CC083E090E090939D1580939C1585E081
:106270008093901582E88093931585E490E1A0E0E7
:10628000B0E08093941590939515A0939615B093D4
:1062900097150E942FF581E01BC082E090E090935B
:1062A0009D1580939C1585E08093901582E88093DE
:1062B000931585E490E1A0E0B0E08093941590936D
:1062C0009515A0939615B09397150E942FF580E031
:1062D0000E9435C020E030E048EC52E460918A171B
:1062E00070918B1780918C1790918D170F94632369
:1062F0000F945F2B70939D1560939C1585E08093A0
:10630000901582E88093931586E290E1A0E0B0E0DA
:106310009BCE8EED95E00E94E5548AE090E090934C
:106320009D1580939C1585E08093901582E880935D
:1063300093154FC184E080939B0B809144159091FD
:106340004515A0914615B091471560914C15709177
:106350004D158834F0E19F07A105B10509F453C03C
:106360008A3400E19007A105B10509F455C08C34C9
:1063700010E19107A105B10509F457C08634904199
:10638000A105B10509F059C063307105B9F58DEC6F
:1063900095E09093200980931F0981E080932C0859
:1063A0008093260210921C0881E09AE590939D1537
:1063B00080939C158AE490E090939F1580939E159E
:1063C00087E08093901512E81093931584E890E08D
:1063D000A0E0B0E08093941590939515A093961546
:1063E000B09397150E942FF58AE090E090939D1549
:1063F00080939C1585E080939015E9C060932B08ED
:1064000010929B0BD7C3412C30E8532E3DEE632EE8
:1064100033E4732E312C11C0412C512C21EE622E0D
:1064200023E4722E3324339408C0412C512C8BEE7C
:10643000682E83E4782E92E0392E80E090E00F946D
:10644000022320E030E040E251E40F94ED2A6B019A
:106450007C0120E030E0A9010F94FD2287FF09C0F4
:106460001092160810921708109218081092190826
:1064700019C0A3019201C701B6010F94532C18163D
:106480004CF0C0921608D0921708E0921808F092CB
:10649000190808C040921608509217086092180810
:1064A0007092190860911608709117088091180869
:1064B00090911908432D0E9434AF61E070E080E0B4
:1064C00090E00E94F8AF20E030E040E251E46091BB
:1064D00006187091071880910818909109180F9468
:1064E00063230F945F2B70939D1560939C1505E0BB
:1064F0000093901512E81093931588E490E1A0E0C2
:10650000B0E08093941590939515A0939615B09351
:1065100097150E942FF520E030E040E251E46091B1
:106520000A1870910B1880910C1890910D180F9407
:1065300063230F945F2B70939D1560939C150093BC
:106540009015109393158AE490E1A0E0B0E0809359
:10655000941590939515A0939615B09397150E9456
:106560002FF520E030E040E251E460910E18709188
:106570000F1880911018909111180F9463230F94A5
:106580005F2B70939D1560939C150093901510934D
:1065900093158CE490E1A0E0B0E080939415909383
:1065A0009515A0939615B09397150E942FF561E06D
:1065B00070E080E090E00E94F8AF10929B0B8AE0C0
:1065C00090E090939D1580939C15009390151093E7
:1065D000931580E092E1A0E0B0E00C94C82880918F
:1065E000441590914515A0914615B09147158635F3
:1065F00030E19307A105B10509F046C020E030E085
:10660000A9016091E00B7091E10B8091E20B9091F8
:10661000E30B0F94F32920E030E04AE253E40F94B7
:10662000FD2220914C1530914D1587FF0AC425306D
:10663000310508F006C48AEA90E090939D15809396
:106640009C1585E08093901512E81093931580E2D5
:1066500090E1A0E0B0E08093941590939515A093FD
:106660009615B09397150E942FF565E070E080E0D5
:1066700090E00E94F8AF81E09AE590939D15809399
:106680009C1582E490E0D2C38435E0E19E07A10529
:10669000B105B9F460914C1570914D1580E090E012
:1066A0000F94022320E030E040E251E40F94ED2A01
:1066B00060931D0870931E0880931F089093200814
:1066C00079C288359041A105B10509F073C2609186
:1066D0004C1570914D1580E090E00F94022320E05E
:1066E00030E040E251E40F94ED2A6093210870936A
:1066F000220880932308909324085CC260914C1573
:1067000070914D1587EB95E00F94E20280914C1546
:1067100090914D1582309105A1F038F4009771F0F9
:106720000197E1F48AE095E043C28430910579F065
:1067300058F0059799F48CE895E00BC084EF94E04D
:1067400037C289EA95E005C08FE995E002C08AE981
:1067500095E09093200980931F092CC28EE195E06B
:1067600027C28DE295E00E94E55480914C159091EE
:106770004D158130910519F46499E4C41BC2892B2D
:1067800009F018C28BE395E00E94E554809112084D
:10679000813039F581E595E00E94E55481E09AE584
:1067A00090939D1580939C158EE290E090939F1599
:1067B00080939E1587E08093901582E880939315CF
:1067C00084E890E0A0E0B0E0809394159093951554
:1067D000A0939615B09397150E942FF51092990BE0
:1067E00035C0823069F485E695E00E94E55481E089
:1067F0009AE590939D1580939C1586E390E00EC0DA
:10680000833031F589E795E00E94E55481E09AE50F
:1068100090939D1580939C1581E490E090939F1533
:1068200080939E1587E08093901582E8809393155E
:1068300084E890E0A0E0B0E08093941590939515E3
:10684000A0939615B09397150E942FF510920418F7
:10685000109212080F945506ADC180914C1590917D
:106860004D158F3F910531F028F08FEF90E0A0E0BB
:10687000B0E002C0A0E0B0E0809302029093030277
:10688000A0930402B093050280910202909103024A
:10689000A0910402B09105020097A105B10509F588
:1068A00010929D1510929C1505E00093901512E82A
:1068B000109393158AE890E1A0E0B0E080939415DE
:1068C00090939515A0939615B09397150E942FF568
:1068D00089E090E090939D1580939C15009390150E
:1068E0003DC00196A11DB11D05E0B695A7959795F0
:1068F00087950A95D1F70197A109B109009701E0A1
:10690000A007B10550F0B0939D15A0939C159093EE
:106910009F1580939E1587E005C090939D158093E9
:106920009C1585E08093901512E8109393158AE8E2
:1069300090E1A0E0B0E08093941590939515A0931A
:106940009615B09397150E942FF588E090E09093EC
:106950009D1580939C1585E0809390151093931559
:106960008CE890E1A0E0B0E08093941590939515A9
:10697000A0939615B09397150E942FF5809102026F
:1069800090910302A0910402B0910502BA2FA92FA1
:10699000982F8827009711E0A107B10550F0B09318
:1069A0009D15A0939C1590939F1580939E1587E04D
:1069B00005C090939D1580939C1585E0809390155C
:1069C00082E88093931581EA90E0A0E0B0E00C9417
:1069D000C8288DE895E00E94E5540E940AAF4091D6
:1069E00044155091451560914615709147158823BF
:1069F00039F0433D20E252076105710509F4E8C30F
:106A0000423D50426105710509F0D4C080914C159A
:106A100090914D15019709F033C50E940AAF882364
:106A200009F42EC580917D1A87FDC4C0A2E18A02B7
:106A3000C0011124885C934E0E942F76C12C90E2F5
:106A4000D92EE12CF12C05E012E810929D15109240
:106A50009C150093901510939315C0929415D092A5
:106A60009515E0929615F09297150E942FF5BFEFBD
:106A7000CB1ADB0AEB0AFB0AEAE0CE16E0E2DE06FE
:106A8000E104F10411F700917D1AF2E10F02800197
:106A900011240053154EF80101900020E9F7C801B8
:106AA0008E1B9F0B439697FD01967C01F594E7940E
:106AB0001E141F040CF0DEC49E012F5F3F4F6901BE
:106AC00084E1D9011D928A95E9F7A7016EE975E085
:106AD000C9010F94662DB801C6018E0D9F1D0F943C
:106AE000512D40E050E260E070E0C6010E94EDF5FB
:106AF00062E070E080E090E00E94F8AF40E060E08B
:106B000070E08FE793E40F94C40641E060E070E02A
:106B10008FE793E40F94C406109201028DE090E099
:106B200090939D1580939C1585E08093901512E8B5
:106B30001093931584E190E1A0E0B0E08093941568
:106B400090939515A0939615B09397150E942FF5E5
:106B500062E070E080E090E00E94F8AF81E09AE5AA
:106B600090939D1580939C1585E390E090939F15DD
:106B700080939E1587E0809390151093931584E879
:106B800090E0A0E0B0E08093941590939515A093C9
:106B90009615B09397150E942FF581E080932602F9
:106BA0008093990B83E080939A0B04C081E895E071
:106BB0000E94E55480E5E0E4F5E1DF011D928A954D
:106BC000E9F78AE58093411585EA809342150C9494
:106BD0009E218AE793E10E944774F701E052FA4E42
:106BE00080838091E0158A3581F01E141F0414F013
:106BF0000C94C222D601E02F1D92EA95E9F710927B
:106C00001B0810921A080C94C22262E070E080E027
:106C100090E00E94F8AFFFEFEF1AFF0AF0921B0816
:106C2000E0921A080C94C2228FEA96E002C08EE924
:106C300096E09093200980931F094CCB88E290E066
:106C40000E948DF82DEC3CEC4CEC5DE360918A17D2
:106C500070918B1780918C1790918D170F94F32959
:106C60006B017C0120E030E040EA51EC0F94532CA2
:106C700087FD12C020E030E040EA51E4C701B601D0
:106C80000F94FD22181644F0C0928A17D0928B17E9
:106C9000E0928C17F0928D1720E030E048EC52E43F
:106CA00060918A1770918B1780918C1790918D1736
:106CB0000F9463230F945F2B70939D1560939C1525
:106CC00085E08093901582E88093931586E290E1A9
:106CD000A0E0B0E08093941590939515A09396153D
:106CE000B09397150E942FF560918A1770918B17BA
:106CF00080918C1790918D178E010B5E1F4F23E0B2
:106D000041E00F94D51D9F938F9380E996E09F9368
:106D10008F93045111091F930F930F949522C8016B
:106D20000E94D2B08BE896E076C088ED9FEF0E947B
:106D30008DF82DEC3CEC4CEC5DE360918A17709182
:106D40008B1780918C1790918D170F94F2296B01FE
:106D50007C0120E030E040EA51EC0F94532C87FD99
:106D600012C020E030E040EA51E4C701B6010F94C0
:106D7000FD22181644F0C0928A17D0928B17E09229
:106D80008C17F0928D1720E030E048EC52E46091CF
:106D90008A1770918B1780918C1790918D170F9493
:106DA00063230F945F2B70939D1560939C1585E072
:106DB0008093901582E88093931586E290E1A0E09D
:106DC000B0E08093941590939515A0939615B09389
:106DD00097150E942FF560918A1770918B178091FB
:106DE0008C1790918D178E010B5E1F4F23E041E0B1
:106DF0000F94D51D9F938F938DE796E09F938F936C
:106E0000045111091F930F930F949522C8010E94FA
:106E1000D2B088E796E09093200980931F090F90E5
:106E20000F900F900F900F900F9077CA90939F152F
:106E300080939E1587E080939015109393150C9482
:106E4000C4282430310539F52091121830911318D7
:106E500040911418509115186091210870912208E2
:106E600080912308909124080F94F32960931218BD
:106E700070931318809314189093151880E090E085
:106E8000A0E8BFE389839A83AB83BC83CE010196DC
:106E90000E94D5E1BBC02530310508F4FDC0263085
:106EA000310509F43CC108F02EC181E0809325082A
:106EB0000F9409078EEB90E00E9451D720E030E05C
:106EC000A9016091E00B7091E10B8091E20B909130
:106ED000E30B0F94F32920E030E048EC52E40F94E8
:106EE00063236B017C016091E40B7091E50B072E2D
:106EF000000C880B990B0F9404239B01AC01C70174
:106F0000B6010F94ED2A0F94662B6436710510F0CC
:106F100064E670E070939D1560939C1505E0009306
:106F2000901512E81093931584E290E1A0E0B0E090
:106F30008093941590939515A0939615B0939715FB
:106F40000E942FF520E030E0A9016091E00B7091E4
:106F5000E10B8091E20B9091E30B0F94F3290F94D6
:106F60005F2B70939D1560939C1500939015109363
:106F7000931586E390E1A0E0B0E0809394159093A0
:106F80009515A0939615B09397150E942FF58091B3
:106F9000E40B9091E50B90939D1580939C150093C5
:106FA00090151093931584E390E1A0E0B0E08093F6
:106FB000941590939515A0939615B09397150E94EC
:106FC0002FF565E070E080E090E00E94F8AF81E08E
:106FD0009AE590939D1580939C1584E490E090939E
:106FE0009F1580939E1587E08093901510939315BD
:106FF00084E890E0A0E0B0E080939415909395151C
:10700000A0939615B09397150E942FF520E030E0DD
:1070100040E251E460911D0870911E0880911F08A4
:10702000909120080F9463230F945F2B70939D150C
:1070300060939C1505E00093901512E8109393154A
:1070400084E590E1A0E0B0E08093941590939515CD
:10705000A0939615B09397150E942FF520E030E08D
:1070600040E251E460912108709122088091230848
:10707000909124080F9463230F945F2B70939D15B8
:1070800060939C15009390151093931588E590E1FB
:10709000A0E0B0E00C94C8282230310589F420919A
:1070A00012183091131840911418509115186091CE
:1070B0001D0870911E0880911F0890912008D4CE61
:1070C0002330310598F02091210830912208409119
:1070D0002308509124086091121870911318809120
:1070E0001418909115180F94F229C0CE2130310553
:1070F00009F08CCF20911D0830911E0840911F0887
:1071000050912008E8CF213F310509F07FCF109240
:10711000250861E070E080E090E00E94F8AF81E037
:107120009AE590939D1580939C1581E490E090934F
:107130009F1580939E1587E08093901582E8809339
:10714000931556CF8BEE95E00E94E55481E00E94A6
:10715000F6BA8DE090E090939D1580939C1585E0A4
:107160008093901512E81093931584E190E1A0E0CC
:10717000B0E08093941590939515A0939615B093D5
:1071800097150E942FF583E080939A0B81E09AE592
:1071900090939D1580939C1585E390E090939F15A7
:1071A00080939E1587E0809390151093931584E843
:1071B00090E0A0E0B0E08093941590939515A09393
:1071C0009615B09397150E942FF510921208F2CCE5
:1071D00083E096E00E94E55480917E1A90917F1A98
:1071E000992720914C1530914D158217930708F47B
:1071F000E1CC86E995E00E94E55480914C158150E0
:1072000080937D1AA4ED8A2EA0E29A2EA12CB12C97
:1072100005E012E810929D1510929C1500939015B0
:10722000109393158092941590929515A0929615AF
:10723000B09297150E942FF53FEF831A930AA30A85
:10724000B30A8EED881680E29806A104B10411F706
:1072500080917D1AA2E18A02C0011124FC01E05351
:10726000F54E7F0101900020E9F7C7018E1B9F0BAF
:10727000439697FD01968C011595079510161106FA
:10728000FCF49E012F5F3F4F690184E1D9011D92FB
:107290008A95E9F7A8016EE975E0C9010F94662D9A
:1072A000B701C601800F911F0F94512D44ED50E29C
:1072B00060E070E0C6010E94EDF505E012E806C04E
:1072C00044ED50E260E070E0C701F5CF10929D15EB
:1072D00010929C150093901510939315809294151D
:1072E00090929515A0929615B09297150E942FF541
:1072F000BFEF8B1A9B0AAB0ABB0AE6EE8E16E0E2E2
:107300009E06A104B10411F78E010F5F1F4F84E1A7
:10731000D8011D928A95E9F780917F1A8F93809109
:107320007E1A8F9380914D158F9380914C158F937A
:1073300088EA95E09F938F931F930F930F94802D6E
:107340004EED50E260E070E0C8010E94EDF562E0B1
:1073500070E080E090E00E94F8AF0FB6F894DEBFD6
:107360000FBECDBF31E2C32E32E1D32EE12CF12C82
:1073700043E1442E40E6542E612C712C88248394E2
:10738000912CAA24AA94BA2C75E0272EE2E83E2E6E
:107390000AE010E080917E1A90917F1A8815990575
:1073A00094F1B0929D15A0929C1520929015309268
:1073B000931540929415509295156092961570927F
:1073C00097150E942FF510939D1500939C15209200
:1073D000901530929315C0929415D0929515E09225
:1073E0009615F09297150E942FF5FFEF8F1A9F0ABE
:1073F00020E1420E511C611C711C3FEFC31AD30ADD
:10740000E30AF30AC7CF80914C1590914D1524E003
:10741000880F991F2A95E1F78D5F9F49A0E0B0E0A2
:1074200020EF37E830939D1520939C1505E00093DD
:10743000901512E8109393158093941590939515D9
:10744000A0939615B09397150E942FF580914C1537
:1074500090914D15805E9D4EA0E0B0E026E030E0BA
:1074600030939D1520939C150093901510939315C0
:107470000C94C82840E050E260E070E0C80136CBD0
:1074800080914C1590914D15892B11F40C94D32BB0
:1074900091CBA7960FB6F894DEBF0FBECDBFDF919C
:1074A000CF911F910F91FF90EF90DF90CF90BF9001
:1074B000AF909F908F907F906F905F904F903F9094
:1074C0002F9008952F923F924F925F926F927F92EA
:1074D0008F929F92AF92BF92CF92DF92EF92FF92E4
:1074E0000F931F93CF93DF93CDB7DEB7C154D1096C
:1074F0000FB6F894DEBF0FBECDBF22968FAF229796
:10750000209142082CAF81E08093420880916B1358
:107510008D3409F4B4C3843511F40C94894B873449
:1075200011F00C94904B8091691390916A138B31F8
:10753000910509F427C1B4F48430910534F4823004
:107540009105E4F597FF2EC096C38531910511F49E
:107550000C94924B8A31910509F410C1049709F0FB
:107560008AC3CDC08A32910509F4ADC24CF48D3185
:107570009105B1F00CF420C14E9709F45CC17BC3B6
:107580008B35910509F41CC28C35910509F41DC297
:107590008A35910509F06FC3109241080C94924B03
:1075A00014E036C180916F02882311F40C94924B41
:1075B0000E94DFC70E9461DE0C94924B20916F0203
:1075C000222311F40C94924B11E0029709F010E081
:1075D0000E94DFC719821A821B821C821D821E82B2
:1075E0001F82188682E50E948DBA882309F457C04D
:1075F0000E940DBA6B017C0120E030E0A9010F94DC
:10760000FD22882309F461C0809106189091071823
:10761000A0910818B091091888A799A7AAA7BBA795
:1076200080910A1890910B18A0910C18B0910D1828
:107630008CA79DA7AEA7BFA78091651790916617ED
:10764000A0916717B091681788AB99ABAAABBBAB99
:107650008091691790916A17A0916B17B0916C1780
:107660008CAB9DABAEABBFAB28A939A94AA95BA92E
:1076700068A579A58AA59BA50F94FD2281110C947C
:107680009D4B2CA93DA94EA95FA96CA57DA58EA5F2
:107690009FA50F94FD228823C1F00C949D4B89E493
:1076A0000E948DBA882331F00E940DBA69837A83D3
:1076B0008B839C838AE40E948DBA882331F00E94D8
:1076C0000DBA6D837E838F83988720E030E0A90117
:1076D00069817A818B819C810F94FD2281110C94A8
:1076E000A24C20E030E0A9016D817E818F819885D8
:1076F0000F94FD2281110C94A24C0C94B54C80E5A2
:107700000E948DBA882329F00E94AFEB6B017C01A7
:1077100003C0C12CD12C760183E50E948DBA882349
:1077200061F00E940DBA20E030E04AE754E40F9483
:1077300063230F94662B6B017C010E94058280916C
:107740008E17811105C060E085E897E00F9416065A
:107750000E94A4FDC60ED71EE81EF91E0E94A4FDBD
:10776000DC01CB018C199D09AE09BF09B7FD02C030
:107770000C94924B80E00E940655F0CF0E947869ED
:107780000C94924B0E94BD9281110C94924B8CE010
:10779000EDEDF2E0DE01119601900D928A95E1F790
:1077A00060E070E080E50E948ECABE016F5F7F4F8F
:1077B0000F9499040C94924B8091AD0B8770873095
:1077C00011F00C94BC4C60E08FE40E94636981115D
:1077D0000C94924B0C94BC4C80911E1881111DC0CE
:1077E0000E94B29F8823F9F0115011F40C94994E25
:1077F00043EF57E06BEF77E085E00E9454BB61E018
:1078000086EE97E00E949ABA8EEC97E00E949CF474
:107810000E94BD92882301F306C060E08FE40E94BD
:1078200063698823E9F20E94BEBA89E998E00E9460
:107830009CF40C94924B20918217309183174091C5
:1078400084175091851760910618709107188091E0
:107850000818909109180F94F329AB01BC0188E531
:107860000E9441B169837A838B839C832091861720
:1078700030918717409188175091891760910A18A5
:1078800070910B1880910C1890910D180F94F3299A
:10789000AB01BC0189E50E9441B16D837E838F837A
:1078A0009887BE016B5F7F4FCE0101960F94411008
:1078B000882311F40C94924B80E00E9435C00E9402
:1078C0004FE161E085E40E946369182F21E0482FB1
:1078D000BE016B5F7F4FCE0101960E94AAF96B013A
:1078E0007C019B01AC010F94E52C81115FC0898064
:1078F0009A80AB80BC8020E030E0A901C501B401D2
:107900000F94FD2287FF05C027E137EB41E558EBD7
:1079100004C027E137EB41E558E3C501B4010F94FA
:10792000F329AB01BC018BEB98E00F94EF028D8043
:107930009E80AF80B88420E030E0A901C501B40189
:107940000F94FD2287FF05C027E137EB41E558EB97
:1079500004C027E137EB41E558E3C501B4010F94BA
:10796000F329AB01BC0186EB98E00F94EF0220E015
:1079700030E0A901C701B6010F94FD2287FF05C0C1
:1079800067E177EB81E598EB04C067E177EB81E590
:1079900098E3A70196010F94F329AB01BC0181EB99
:1079A00098E00F94EF028AE00E94DA530E9436E1D9
:1079B000113011F40E94027E0E9427C30C94924B56
:1079C0008FE0809341080C94924B17E9212E13E02D
:1079D000312E06E2E02E03E1F02E26E038E13DA351
:1079E0002CA386E7C82E87E1D82E00E010E0D10155
:1079F0008D911D010E948DBA882309F44BC00E940D
:107A00000DBA2B013C01133049F0F6012081318180
:107A1000428153810F94F2292B013C01ACA1BDA1FD
:107A20002D913D914D915C91C301B2010F94F229CA
:107A30004B015C012DEB37E346E855EB0F94532CDB
:107A400087FD0AC02DEB37E346E855E3C501B401D5
:107A50000F94FD221816F4F4133051F440921218CA
:107A600050921318609214187092151801E012C009
:107A7000A5019401F70160817181828193810F9446
:107A8000F329D7016D937D938D939C931397812F49
:107A90000E94A4DD1F5FB4E0EB0EF11CECA1FDA180
:107AA0003496FDA3ECA3F4E0CF0ED11C143009F002
:107AB0009ECF002321F082E198E10E9416820E946D
:107AC00027C30C94924B80916F02882311F40C947D
:107AD000924B89E40E948DBA082F882321F00E94DE
:107AE00009BAE82E01C0E12C8AE40E948DBA182F51
:107AF000882321F00E9409BAF82E01C0F12C00233E
:107B000019F024E02E1528F0112349F034E03F1538
:107B100030F483EC98E00F943B020C94924B80E19C
:107B2000E6E0F8E1A5E6B7E101900D928A95E1F76C
:107B30000023F1F020918112309182124E2D4203E8
:107B4000B001439F700D11248091D0119091D111FB
:107B5000680F791F072E000C880B990B0F940423D4
:107B600060936517709366178093671790936817F3
:107B70001123F1F020918312309184124F2D420392
:107B8000B001439F700D11248091D2119091D311B7
:107B9000680F791F072E000C880B990B0F94042394
:107BA0006093691770936A1780936B1790936C17A3
:107BB00060E080E50E9463698823C1F10023D1F071
:107BC0002091821730918317409184175091851727
:107BD000609165177091661780916717909168178B
:107BE0000F94F22960936517709366178093671757
:107BF000909368171123D1F0209186173091871741
:107C000040918817509189176091691770916A1790
:107C100080916B1790916C170F94F22960936917FC
:107C200070936A1780936B1790936C1740E050E045
:107C3000BA0186E40E9441B16B017C0120E030E092
:107C4000A9010F94532C18164CF420E030E040E7C3
:107C500052E4C701B6010F94ED2A03C060E070E062
:107C6000CB0169837A838B839C83CE0101960E942A
:107C70006EE10C94924B0E9485920C94924B8091F1
:107C8000691390916A138537910511F40C94354668
:107C90000CF053C18934910509F4FCC40CF069C09F
:107CA0008A31910509F484C39CF58431910509F466
:107CB000FEC27CF48131910509F4D8C22CF40297FC
:107CC00008F451C20C94864B429709F425C70C94D2
:107CD000864B8731910509F40FC38CF485319105EA
:107CE00009F406C3469711F00C94864B0E94167651
:107CF00080911817877F809318170C94924B8831C6
:107D0000910509F411C3499709F447C30C94864BB4
:107D10008F31910509F477C47CF48C31910509F415
:107D2000BCC30CF453C38D31910509F4C0C34E9705
:107D300009F4C4C30C94864B8A32910509F483C4B8
:107D400064F48032910509F418C4819711F00C9401
:107D5000864B0E94CEB70C94924B8B32910509F45E
:107D600095C4C09711F00C94864B0E946F9B0C94A5
:107D7000924B8836910509F435C5ECF581359105AE
:107D800009F4AEC6C4F48C34910509F492C44CF4E1
:107D90008B34910511F00C94864B0E94067F0C9455
:107DA000924B8D34910509F488C48E34910509F401
:107DB00088C40C94864B8435910509F4ADC68CF4C7
:107DC0008235910509F4A1C68335910511F00C9413
:107DD000864B809141088F7E8062809341080C948D
:107DE000924B8535910509F49AC68C35910509F4B5
:107DF000AFC60C94864B8E36910509F4ACC5D4F40D
:107E00008B36910509F49AC554F48936910509F425
:107E10005FC58A36910509F46FC50C94864B8C3684
:107E2000910511F40C94924B8D36910509F4F9C427
:107E30000C94864B8137910509F4E3C55CF48F36C9
:107E4000910509F499C58037910511F40C94924B72
:107E50000C94864B8237910509F404C7833791054A
:107E600011F00C94864B8DE79BE00F943B0260E091
:107E70008DE69BE00E9421F360E088E59BE00E9494
:107E800021F361E081E59BE00E9421F361E086E45B
:107E90009BE00E9421F361E086E39BE00E9421F3D6
:107EA00060E08DE29BE00E9421F361E083E29BE0D1
:107EB0000E9421F361E089E19BE00E9421F361E0EF
:107EC00081E19BE00E9421F361E083E09BE00E945E
:107ED00021F361E085EF9AE00E9421F360E086EEF5
:107EE0009AE00E9421F360E088ED9AE00E9421F37D
:107EF00060E082EC9AE00E9421F361E081EB9AE07D
:107F00000E9421F361E082EA9AE00E9421F361E09D
:107F10008DE89AE00E9421F361E08AE79AE00E94EE
:107F200021F360E08DE69AE00E9421F360E089E5AC
:107F30009AE00E9421F30C94924B8E32A1E09A07B2
:107F400011F40C94A6490CF077C08B3C910509F410
:107F500052C7ACF58D37910509F4BFC5BCF487371E
:107F6000910509F4CDC60CF491C68837910509F442
:107F7000CAC68937910511F00C94864B10920F09EF
:107F800010920E090E94A0C10C94924B8E3B910559
:107F900009F46BC554F48C38910509F454C58B3938
:107FA000910509F474C50C94864B883C910509F43D
:107FB000B2C6893C910509F4FBC60C94864B8D3DF5
:107FC000910509F47FC7CCF48E3C910509F448C7AC
:107FD00054F48C3C910509F42DC78D3C910509F4AE
:107FE0002CC70C94864B833D910509F45BC78C3DEF
:107FF000910509F45AC70C94864B8232E1E09E0742
:1080000011F40C949B485CF4823E910509F4B0C7CE
:108010008831914011F40C9404480C94864B8C32B6
:1080200031E0930711F40C949E488D32914011F485
:108030000C94B3480C94864B843FA1E09A0711F44A
:108040000C94D44A0CF043C08239E1E09E0711F44D
:108050000C94F049DCF4803321E0920711F40C9485
:10806000334914F40C94EA49803941E0940711F43F
:108070000C94ED498139914011F00C94864B81E0CC
:108080000E944A7E0E9427C30C94924B843AB1E02E
:108090009B0711F40C94034A6CF48A39F1E09F07B2
:1080A00011F40C94924B8C39914011F40C94F849D2
:1080B0000C94864B853A31E0930711F40C94064AF0
:1080C0008C3A914011F40C94764A0C94864B883586
:1080D000A2E09A0711F40C94FC4A1CF5873FE1E0FA
:1080E0009E0711F40C94DA4A7CF4853F21E0920754
:1080F00011F40C94D74A863F914011F00C94864BB2
:108100000E94BAC10C94924B883F41E0940711F44D
:108110000C94E34A8C30924011F40C94F44A0C9481
:10812000864B8C36B3E09B0711F40C94924B7CF495
:108130008B35F2E09F0711F40C94FF4A833593408E
:1081400011F00C94864B0E9409EC0C94924B803AEF
:1081500033E0930709F447C2873E934011F40C942F
:10816000784B0C94864B0091691210916A1280E54D
:108170000E948DBA882361F00E94AFEB6B017C01F5
:10818000BB24B394672B682B692B31F4B12C04C04A
:10819000B12CC12CD12C760183E50E948DBA8823A5
:1081A00011F40C94AB4E0E940DBA20E030E04AE787
:1081B00054E40F9463230F94662B6B017C01B11080
:1081C0000BC0672B682B692B39F40115110521F0C1
:1081D000D8018C91811102C0B12C02C0BB24B39490
:1081E0000E940582B11003C082E196E001C0C8017F
:1081F0000E9417B11091420883E08093420881E009
:108200008093041844EF58E06DEF78E082E00E941C
:1082100054BB82EE98E00E9417B1C114D104E1046E
:10822000F104B1F00E94A4FDC60ED71EE81EF91E8F
:108230000E94A4FDDC01CB018C199D09AE09BF0988
:10824000B7FF0EC08091041881110C94B04E08C085
:1082500080910418882321F080E00E940655F8CF11
:1082600010920418109342080C94924B80916C1356
:1082700084FF02C00C94B54E80916E1387FF02C03C
:108280000C94B54E80916F13837011F00C94B54E21
:1082900060E08FE099E00F9416065F988A988091CD
:1082A000080181708093060112980C94924B87E22A
:1082B00099E00F943B0280E794E10E944E958BE198
:1082C000E0E7F4E1DE01119601900D928A95E1F765
:1082D00060E070E0CE0101960E941678CE01019612
:1082E0000E94849688E199E00F943B020C94924B93
:1082F0000E9487760C94924BE0916912F0916A1279
:108300008081882329F0803209F410823196F8CFD9
:1083100040E061E08091691290916A120E94737945
:10832000109205180C94924B8091200B8823E9F051
:1083300080E090E0A0EAB1E488A399A3AAA3BBA33C
:108340001C8E1D8E1E8E1F8E19821A821B821C820D
:1083500020E0AE01405E5F4FBE01645E7F4FCE0104
:1083600001960E9414BC0C94924B0E947F5188236A
:1083700021F00E9427760E94067F61E083E29CE361
:108380000E949ABA48E359E060E479E085E00E94EF
:108390000DBC0F949A060C94924B8091181782FF93
:1083A00003C08B7F809318170E94CBC90C94924B0B
:1083B0008091181783FD02C00C94924B83E50E94B4
:1083C0008DBA81110C94D14E0C94924B83E40E948F
:1083D00044BA8823C1F186E599E00F943B0280916D
:1083E0001A14882339F1BE016F5F7F4F87E194E152
:1083F0000E9415948E010F5F1F4FF80181918F012C
:10840000882319F00E94DA53F8CFCE0101960E941A
:10841000457980912E1A882389F080E20E94DA53F0
:108420000EE21AE1D8018D918D01882339F00E9466
:10843000DA53F8CF8CE499E00F943B028AE00E9473
:10844000DA530C94924B83E50E948DBA882309F18C
:108450000E94F5B9182F90E0CD970CF01CE3109313
:1084600036080E94A4FD6B017C01212F30E0A8EEAC
:10847000B3E00F94A729C60ED71EE81EF91EC092BE
:108480003208D0923308E0923408F09235080C9408
:10849000924B0E94EF750C94924B40E060E080910B
:1084A000691290916A120E9473790C94924B809198
:1084B00018178E7F809318170C94924B8091181781
:1084C00083FD02C00C94924B0E947CFB8091181794
:1084D00083FD02C00C94924B6091691270916A12F4
:1084E000CE014C960E94A5F78C01009711F40C94D4
:1084F000924B6C8D7D8D19821C8222E0AC01CE01E5
:1085000001960E947E9A811102C0F12C14C0CE0106
:1085100001960E9413F78823C1F361E0CE01019612
:108520000E94F993009789F325EEFC0120831C82B9
:108530000E940896F82ECE0101960E948496B801FA
:10854000FF2089F080E899E00F940D038AE00E94F3
:10855000DA531092141710921517109216171092E2
:1085600017170C94924B88E699E00F940D0385E65B
:1085700099E00F943B020C94924B8091181782FD66
:108580000E9405828091181783FD02C00C94924BC3
:1085900060E080E50E946369182F482F61E08091B8
:1085A000691290916A120E94737983E50E948DBAD4
:1085B000882381F00E94E5B9AB01BC0140931417F8
:1085C00050931517609316177093171787E194E16E
:1085D0000E940F930E94277611110C94924B0E94D7
:1085E000067F0C94924B2091691230916A129091FF
:1085F000181792609093181740E060E0C9010E943C
:1086000073790C94924B0F9411046C8F7D8F8E8F25
:108610009F8FBE016F5F7F4FCE014C960E94EFB6D9
:1086200060E0CE0101960F9471060F942403BE0101
:108630006F5F7F4F8EE899E00F940D038AE00E94F0
:10864000DA530C94924B83E50E948DBA882311F47F
:108650000C94924B0E94F5B9F82E6DE070E080E525
:108660000F9475118C0197FF02C00C94924BE82E69
:1086700060E089E40E94636981110C94E24E802FCE
:108680000E943D51811191C40C94E24E0E9421CC74
:108690000C94924B80E50E9444BA882311F40C9408
:1086A000924B8091181782FF02C00C94924B0C944D
:1086B000FB4E0F9460040C94924B0E94B67F0C9476
:1086C000924B60E070E083E50F9475118E34910554
:1086D00031F40E9468800F949A060C94924B89EFB3
:1086E00099E00F943B026091FE087091FF0880EFC3
:1086F00099E00F94E202609100097091010983EE04
:1087000099E00F94E2026091FE087091FF08809159
:10871000000990910109681B790B8091A00B815091
:1087200021E030E0823010F020E030E0621B730B7B
:1087300088ED99E00F94E2028AE00E94DA5380ED1E
:1087400099E00F943B028091020990910309A09156
:108750000409B09105098C8F9D8FAE8FBF8FBE012C
:108760006F5F7F4FCE014C960E94EFB6BE016F5FE8
:108770007F4F83EC99E00F940D038091060990914F
:108780000709A0910809B09109098C8F9D8FAE8FC0
:10879000BF8FBE016F5F7F4FCE014C960E94EFB638
:1087A000BE016F5F7F4F83EB99E00F940D0320E0D4
:1087B00030E04AE754E460910A0970910B09809116
:1087C0000C0990910D090F94ED2AAB01BC018BE9C6
:1087D00099E00F94EF028DE60E94DA538AE00E943E
:1087E000DA53A0C78091751183FD9CC70E94A6C86B
:1087F00087FD98C783E50E948DBA882379F00E948F
:108800000DBA0F945F2B8B01CB010E9451D7063517
:10881000110524F40E94B67F0F949A060F94871CCA
:1088200081C78091751183FD7DC70E94A6C8F82E6F
:1088300087FD78C783E50E948DBA082F811106C095
:1088400082E50E948DBA182F8823C1F10E940DBACB
:108850000F945F2BCB010E9451D70E940DBA20E0EC
:1088600030E04AEA52E40F94FD22181614F40C94F6
:10887000064F0E94B67F0F949A066091E40B7091A8
:10888000E50B072E000C880B990B0F9404234B016A
:108890005C014090E00B5090E10B6090E20B709017
:1088A000E30BA30192010F94532C181614F40C94AB
:1088B000244F002311F40C940A4F11E00F94871CED
:1088C000112309F42FC7602F8F2D0E944DD12AC785
:1088D0000E94A6C8182F87FD0AC08CE19AE00F9469
:1088E0003B02812F0E9458CF8AE00E94DA53FCADF0
:1088F000F09342080C945A5060E080E50F94841184
:10890000182F823008F00EC781E40E9444BA8823F1
:1089100021F06091C90B70E002C06FEF70E083E559
:108920000E948ECAE12FF0E0E753F44F8F3F91058C
:1089300019F010F08FEF90E08083F4C660E080E5DE
:108940000F948411823008F0EDC6E82FF0E0E75371
:10895000F44F1082E7C68EE40E948DBA882309F492
:10896000E1C60E94E5B96093651270936612809328
:10897000671290936812D6C683E50E9444BA882392
:1089800031F060E083E50F948411809375110F94AA
:1089900024038DE29AE00F943B02809175118823A5
:1089A00069F1B3E2EB2EBAE0FB2E00E010E020E02C
:1089B0008091751190E0A0E0B0E0002E04C0B69563
:1089C000A795979587950A94D2F780FF0EC0DD246E
:1089D000D394D20E222319F08CE20E94DA53F701CD
:1089E000859194910F943B022D2D0F5F1F4F32E024
:1089F000E30EF11C05301105D9F620CD8FE19AE088
:108A00001BCD83E50E948DBA882371F00E94F5B9D1
:108A1000282F30E02D3331051CF48093000282C6EC
:108A20008CE3809300027EC60F94240340910002E1
:108A300050E060E070E084E39AE00F94D1028AE0B5
:108A40000E94DA536FC68091751183FD6BC683E572
:108A50000E948DBA882309F465C60E940DBA0F944E
:108A60005F2BCB010E9445695DC68091751183FD26
:108A700059C683E50E948DBA182F81110C94274F97
:108A800082E50E948DBA81110C94274F4BC683E575
:108A90000E948DBA882309F445C60E94F5B9182FA3
:108AA00090E0CD970CF01CE310933B080E94A4FDCE
:108AB0006B017C01212F30E0A8EEB3E00F94A729D1
:108AC000C60ED71EE81EF91EC0923708D09238088D
:108AD000E0923908F0923A0825C60E94CBC922C616
:108AE0000E9462D70E94B67F0E946A830E948D51C5
:108AF0001092AC0B1092AB0B1092AA0B68EE73E0C5
:108B000080E090E00F940C020DC6809141088F7DAB
:108B100080618093410806C60E9490CB03C683E51E
:108B20000E9444BA882309F4FDC50E940DBA20E0D2
:108B300030E04AE754E40F9463230F94662B60936C
:108B40003C0870933D0880933E0890933F08EAC527
:108B50000E94A6C887FDE6C590916C1394FD04C0E1
:108B600090916E1397FF0AC0F7E9CF2EF3E0DF2E46
:108B7000A6E7EA2EA1E1FA2E10E009C090916F134A
:108B8000937091F7682F81E00E94E6CBCBC5D601A8
:108B90008D916D010E948DBA882309F459C013305C
:108BA00009F04FC00E940DBA4B015C0120E030E09B
:108BB00040EA51E40F94FD2287FF3AC0A5019401D9
:108BC00060919611709197118091981190919911DF
:108BD0000F94ED2A2B013C019B01AC016091A61181
:108BE0007091A7118091A8119091A9110F946323FE
:108BF0006093A6117093A7118093A8119093A91167
:108C00006091C10B7091C20B8091C30B9091C40B0A
:108C10000F940223A30192010F9463230F94662BF8
:108C20006093C10B7093C20B8093C30B9093C40BE2
:108C30008092961190929711A0929811B0929911EA
:108C400007C00E940DBAF701648B758B868B978BDA
:108C50001F5FF4E0EF0EF11C143009F098CF0E9472
:108C6000E18160C50E943BF35DC5809169129091DE
:108C70006A12009741F0DC012C91222321F060E080
:108C80000F9471064FC50F949A064CC50091691256
:108C900010916A1294E0F12C40E0915021F1F8011A
:108CA0008081282F2B7F213421F421812133D9F495
:108CB00007C08035C1F4818180538A3048F013C0E9
:108CC000813421F0853421F441E002C0FF24F39483
:108CD00098012E5F3F4F89012F5F3F4FF801808140
:108CE0008032C9F3DACF41110F942403FF2021F021
:108CF00084E69CE00F943B02C8010E94E55412C533
:108D00000E9449C10FC581E080930F0980930E092D
:108D10000E94A0C107C50E94A6C8182F87FD02C5E2
:108D200084E40E9444BA882309F43FC00E940DBA2B
:108D30006B017C0101E020E030E0A9010F94FD22ED
:108D4000811101C000E00093321320E030E0A9015E
:108D5000C701B6010F94FD22882339F10E940DBA94
:108D600024E01202F0011124E95CFC4E608371835F
:108D70008283938320E030E0A901609137137091E2
:108D800038138091391390913A130F94FD22811179
:108D90000CC080E090E0A0EEBFE380933713909387
:108DA0003813A0933913B0933A130E949FDABAC4D0
:108DB0000E94A6C887FDB6C4E7E9EE2EE3E0FE2ECA
:108DC00006E711E1D7018D917D010E9444BA882305
:108DD00059F00E940DBA0F94662BF80160837183DD
:108DE000828393830E949A810C5F1F4FF1E10638C2
:108DF0001F0741F797C40E94A6C887FD93C477E96F
:108E0000E72E73E0F72E06E711E1D7018D917D0182
:108E10000E9444BA882339F00E940DBAF80164A375
:108E200075A386A397A30C5F1F4FF1E106381F07B8
:108E300061F778C40E9439EB75C480916C1381FF8F
:108E400002C00C945C4F80916D1381FF02C00C94A2
:108E50005C4F80916E138C7011F00C945C4F62C467
:108E600057E9C52E53E0D52E62E1E62E69E0F62ED5
:108E700010E0D6018D916D010E9444BA882351F013
:108E80000E940DBAF7016083718382839383812FDF
:108E90000E94A4DD1F5FF4E0EF0EF11C133049F7D0
:108EA0000C945F3D0E94A1CA3DC483E50E948DBA27
:108EB000882309F437C40E9409BA9093560280931C
:108EC000550230C40E94A6C8F82E87FD2BC483E546
:108ED0000E948DBA0F2D0F2C000C110B882369F105
:108EE0000E9409BAF801EE0FFF1FE55AFD4F91836A
:108EF0008083000F111F000F111F9801295D3D4F46
:108F00007901BC01990F880B990B0F9404232AE077
:108F100037ED43E25CE30F946323F801ED5CFC4E14
:108F200020813181428153810F946323D7016D9356
:108F30007D938D939C931397F5C30F94240385E43D
:108F40000E94DA5380E38F0D0E94DA53F801EE0F8E
:108F5000FF1FE55AFD4F6081718187E89CE00F9407
:108F6000000385E20E94DA538AE00E94DA53DAC3F2
:108F700080E50E9444BA882309F4D4C360E070E01D
:108F800080E50F947511F82E6FEF7FEF83E50F9456
:108F900075118C010196039708F0C4C3F7FCC2C396
:108FA0008F2D0E943D51882339F00F9420038FE8C4
:108FB0009CE00F943B02B6C30E94058260E08F2DB7
:108FC0000E9446FC0F3FBFEF1B0731F00130110537
:108FD00071F000E010E00DC08F2D0E94EEFB31E03B
:108FE00020E0892B09F030E0032F122F02C001E0AE
:108FF00010E08F2D0E94EEFB8017910709F492C3B9
:1090000080E00E940655F5CF80E50E9444BA88238F
:1090100009F488C30E9409BA8C01892B09F07FC02A
:1090200083E50E9444BA882389F00E9409BA8F3FE1
:10903000EFEF9E0729F488EF94E10E94925172C3EA
:10904000BC0188EF94E10E9462526CC30F94240328
:1090500060E070E087EB9CE00F9400038091FA14CD
:1090600028E532E06901C81AD10887FDD394CC0CF9
:10907000DD1CCC0CDD1C0D2C000CEE08FF088091D3
:10908000F91428E830E04901881A910887FD939483
:10909000880C991C880C991C092C000CAA08BB0888
:1090A0008091F8148F3FC1F090E0FC01EE0FFF1F9C
:1090B0008E0F9F1FFC01E557FB4E2181328113E08B
:1090C000220F331F1A95E1F704E0369527950A958C
:1090D000E1F72E5F3F4F02C020E030E02F5F3F4FAF
:1090E000C901330FAA0BBB0B9C01AD01281939092B
:1090F0004A095B09A4EBB0E00F949429A7019601FB
:10910000281939094A095B090F947529B90184EBBB
:109110009CE00F9400038AE00E94DA5303C30F948B
:109120002003B8018DEA9CE00F9400038EE99CE0D7
:109130000F943B02F7C20E94B5EEF4C264E071E006
:1091400083E50E948ECA8C0168EE73E080E50E9480
:109150008ECA8938F3E19F0710F088E893E1B801DF
:109160000F94B705DFC260E085E40F94841181118C
:1091700073C080E50E9444BA882351F00E940DBA62
:109180006093E70B7093E80B8093E90B9093EA0BE5
:1091900089E40E9444BA882381F00E940DBA2CEA27
:1091A00035EC47E25EE30F9463236093EB0B70931F
:1091B000EC0B8093ED0B9093EE0B84E40E9444BA89
:1091C000882381F00E940DBA2CEA35EC47E25EE379
:1091D0000F94ED2A6093EF0B7093F00B8093F10BDB
:1091E0009093F20B0F9424034091E70B5091E80BFE
:1091F0006091E90B7091EA0B89ED9CE00F94EF020E
:109200002CEA35EC47E25EE36091EB0B7091EC0BDE
:109210008091ED0B9091EE0B0F94ED2AAB01BC0108
:1092200085ED9CE00F94EF022CEA35EC47E25EE31B
:109230006091EF0B7091F00B8091F10B9091F20B1C
:109240000F946323AB01BC0181ED9CE00F94EF020E
:109250008AE00E94DA5366C20F9420038FEB9CE0F1
:109260000F943B025FC280E50E9444BA882351F00C
:109270000E940DBA6093EE087093EF088093F00897
:109280009093F10889E40E9444BA882381F00E94F7
:109290000DBA2CEA35EC47E25EE30F94632360934A
:1092A000F2087093F3088093F4089093F50884E42F
:1092B0000E9444BA882381F00E940DBA2CEA35EC52
:1092C00047E25EE30F94ED2A6093F6087093F70887
:1092D0008093F8089093F9080F9424034091EE08C6
:1092E0005091EF086091F0087091F10885EE9CE0D4
:1092F0000F94EF022CEA35EC47E25EE36091F2084E
:109300007091F3088091F4089091F5080F94ED2A7C
:10931000AB01BC0181EE9CE00F94EF022CEA35EC2E
:1093200047E25EE36091F6087091F7088091F808D3
:109330009091F9080F946323AB01BC018DED9CE083
:109340000F94EF028AE00E94DA53ECC183E50E9499
:1093500044BA182F882371F00E940DBA0F945F2B26
:1093600070932C0260932B0221E0672B09F020E020
:109370002093DB0B80E50E9444BA882359F02091AA
:109380002B0230912C02232B11F00E945369809301
:10939000DB0BC8C11111C6C10F94240385E09DE009
:1093A0000F943B028091DB0B882319F08DEE9CE03B
:1093B00002C089EE9CE00F943B0260912B027091F9
:1093C0002C0284EF9CE00F94000380EF9CE00F944C
:1093D0003B02A8C10E9458B1A5C10E940582A2C14A
:1093E00080E00E944A7E0E94027E0E9427C39AC1AA
:1093F00080916C13887809F0DCC580916E138670BB
:1094000009F0D7C5B2C50F9490118CC16FEF7FEFF3
:1094100089E40F947511F82E6FEF7FEF8AE40F94B3
:109420007511E82E8AE50E9444BA182F811105C0F3
:1094300081E50E9444BAB82E01C0B12CF7FC06C0E9
:10944000E7FC04C0111109C0B11007C00F9420033C
:109450008FE69DE00F943B0265C124E02F1510F0CC
:109460002E1538F40F94200380E59DE00F943B0205
:1094700059C1CF2C0F2C000CDD080E2D0E2C000C2A
:10948000110B0E940DBABB2099F025E02C9DF00134
:109490002D9DF00D1124E00FF11FEE0FFF1FEE0FB9
:1094A000FF1FE357FD4E208131814281538103C06C
:1094B00020E030E0A9010F94F3299B01AC0185E085
:1094C0008C9DF0018D9DF00D1124E00FF11FEE0F2A
:1094D000FF1FEE0FFF1FE357FD4E208331834283B2
:1094E00053836E2D8F2D0E9413B01CC10E94BD921C
:1094F000811118C10EE910E386E098E19DA38CA3C9
:10950000DE0111961D0143EFC42E40E3D42E7D01F0
:10951000F8016591759185919491ECA1FDA18190DF
:109520009190A190B190FDA3ECA3A50194010F949B
:10953000F2292B013C01D7016D937D938D939C9370
:10954000139720E030E040EA51EC0F94532C87FD54
:109550000AC020E030E040EA51E4C301B2010F94B8
:10956000FD2218162CF4F601849118160CF451C53E
:10957000D7018D909D90AD90BD907D0120E030E0B1
:1095800040EA51ECC501B4010F94532C87FD4BC543
:1095900020E030E040EA51E4C501B4010F94FD221F
:1095A00018160CF052C53FC50E9418ABBBC00E94F4
:1095B000D2C6B8C061E083E50E94636991E0892763
:1095C0000E94DCC3AFC081E080937C120E941EA584
:1095D00010927C12882309F4A5C00F9424038BEC0D
:1095E0009DE00F943B029EC08091181782FF9AC0A5
:1095F00080648093181796C00E94CFC893C00E94C1
:10960000A6C8082F87FD8EC085E50E9444BA88232E
:10961000B1F1E02E002E000CFF080E940DBA4B01A4
:109620005C0120E030E0A9010F94532C87FF04C0B7
:10963000B7FAB094B7F8B094C70123E0880F991F28
:109640002A95E1F79C012B573D4E7901D9018D9266
:109650009D92AD92BC92139720E030E04AEF53E424
:10966000C501B4010F94532C18164CF480E090E01F
:10967000AAEFB3E4F70180839183A283B3838CE4E0
:109680000E9444BA882309F44DC0002E000C110B2F
:109690000E940DBA6B017C0120E030E0A9010F941B
:1096A000532C87FF04C0F7FAF094F7F8F09420E009
:1096B00030E04AEF53E4C701B6010F94532C9801F0
:1096C00093E0220F331F9A95E1F7F901EB57FD4E16
:1096D00018162CF0C482D582E682F78223C080E07F
:1096E00090E0AAEFB3E484839583A683B7831AC07E
:1096F00081E080936F021092CE1760E083E50E94B4
:10970000636981110FC00E94F3B80CC00E9485925A
:1097100009C080916913882329F00E9443CF02C0B9
:109720000E9485922296FFAD2297F11102C00E94FD
:109730009EB82CAD20934208BDC420E030E0A901C2
:10974000C701B6010F94FD22881F8827881F1817AC
:1097500009F4F3C080E090E0A0E8BFEB88AF99AFD8
:10976000AAAFBBAF28A539A54AA55BA568A979A969
:109770008AA99BA90F94F2292B013C012CA53DA598
:109780004EA55FA56CA97DA98EA99FA90F94F2296A
:109790006CA37DA38EA39FA3A3019201C301B20179
:1097A0000F9463234B015C012CA13DA14EA15FA14D
:1097B000CA01B9010F9463239B01AC01C501B40137
:1097C0000F94F3290F94A12C4B015C0120E030E0B1
:1097D00040E05FE30F94632321966CAF7DAF8EAFC3
:1097E0009FAF2197A7019601C701B6010F9463238C
:1097F0006B017C0121962CAD3DAD4EAD5FAD219747
:10980000CA01B9010F9463239B01AC01C701B601E2
:109810000F94F2290F94A12C6B017C018CA19DA1C6
:10982000AEA1BFA1B0588CA39DA3AEA3BFA32DEB47
:1098300037E346E855EBC501B4010F94532C87FD7F
:109840000AC02DEB37E346E855E3C501B4010F9498
:10985000FD2218165CF4A501940160E070E080E838
:109860009FE30F94ED2A4B015C0103C0812C912CE6
:109870005401A5019401C301B2010F94632328ADE3
:1098800039AD4AAD5BAD0F946323A70196010F94E8
:1098900063232B013C0128A939A94AA95BA968A522
:1098A00079A58AA59BA50F94F32920E030E040E03C
:1098B0005FE30F9463239B01AC01C301B2010F94DA
:1098C000F32928A539A54AA55BA50F94F229698338
:1098D0007A838B839C83A50194016CA17DA18EA1C9
:1098E0009FA10F94632328AD39AD4AAD5BAD0F94B2
:1098F0006323A70196010F9463236B017C012CA9BC
:109900003DA94EA95FA96CA57DA58EA59FA50F9425
:10991000F32920E030E040E05FE30F9463239B01F4
:10992000AC01C701B6010F94F3292CA53DA54EA5A6
:109930005FA50F94F2290C94613B80E090E0A0E8D1
:10994000BFE30CCF412FBE016F5F7F4F85E697E1EC
:109950000E945BEF0E94A4FD6093701370937113DB
:109960008093721390937313DDCE0F9420038FE6D0
:1099700097E00F943B02D6CE0E94058290911E186C
:109980009CAB80E00E9435C00E944FE181E0809353
:109990000F090E94A0C188E50E9444BA182F89E5EA
:1099A0000E9444BA082F8AE50E9444BA1013BFC12E
:1099B000181711F0012FBBC101E011E091E09CA745
:1099C00080E1E6E0F8E1A5E6B7E101900D928A9525
:1099D000E1F782E50E948DBA882361F00E940DBAFA
:1099E0006B017C0120E030E0A9010F94FD22882367
:1099F00069F106C0C12CD12C90E8E92E90E4F92E33
:109A0000111103C0002309F4FCC0C0926D17D0925D
:109A10006E17E0926F17F0927017A7019601609190
:109A20000E1870910F1880911018909111180F94C2
:109A3000FD2287FF0BC019821A821B821C82BE0185
:109A40006F5F7F4F8DE697E10E94D3E2112309F407
:109A5000D3C0002309F4CDC0109206181092071845
:109A6000109208181092091810920A1810920B18E8
:109A700010920C1810920D180E9486E3E3EFF0E3A9
:109A8000A491A8AFE7EEF0E3C590D590E590F490EF
:109A9000EBEEF0E385909590A590B490A50194012C
:109AA000C701B6010F94532C18162CF4A701960188
:109AB000C501B40104C0A5019401C701B6010F940A
:109AC000ED2A2B013C01EEEAF0E385919591A591F9
:109AD000B4918CA39DA3AEA3BFA3EAEAF0E3859162
:109AE0009591A591B49188A799A7AAA7BBA79C0116
:109AF000AD016CA17DA18EA19FA10F94532C1816CE
:109B000034F428A439A49AA598AB1BA505C02CA0B1
:109B10003DA0AEA1A8AB1FA1A3019201C301B20158
:109B20000F94632320E030E040E85FE30F94F329D3
:109B30000F94A12C910148A9512F0F94632368A37E
:109B400079A38AA39BA3E4EFF0E3149120E030E033
:109B500040EC5FE3C501B4010F9463234B015C014A
:109B6000612F110F770B880B990B0F9404239B0126
:109B7000AC01C501B4010F94632369837A838B839D
:109B80009C8320E030E040EC5FE3C701B6010F9416
:109B900063236B017C01B8AD6B2FBB0F770B880B78
:109BA000990B0F9404239B01AC01C701B6010F94DC
:109BB00063236C8F7D8F8E8F9F8FAE01405E5F4FD2
:109BC000BE016F5F7F4FCE014C960E94B1E20E94B2
:109BD000AFC1109206181092071810920818109230
:109BE000091810920A1810920B1810920C18109263
:109BF0000D1880E00E9488E3002319F081E00E94A4
:109C000088E3ECA5EE2309F484C080E00E94B9BF8C
:109C1000809178138370833051F060E080EC97E09E
:109C20000F9416060F94240381EB97E06EC00E94F8
:109C300086E380900E1890900F18A0901018B090A6
:109C400011182091821730918317409184175091F9
:109C5000851760E070E080EA92E40F94F229609347
:109C60006517709366178093671790936817209114
:109C7000861730918717409188175091891760E0B7
:109C800070E080EA92E40F94F2296B017C0160930A
:109C9000691770936A1780936B1790936C172091D4
:109CA0008A1730918B1740918C1750918D17C501F1
:109CB000B4010F94F22960936D1770936E1780931F
:109CC0006F1790937017B701A60185E697E10F947F
:109CD0005C13882389F019821A821B821C82AE01D0
:109CE0004F5F5F4F69E677E185E697E10E94B1E259
:109CF00082E00E9488E30BC060E080EA97E00F9466
:109D000016060F9424038EE897E00F943B020E94FE
:109D1000027E0E9486E380910E0980930F098CA930
:109D20000E9435C00E9436E10E9427C3FBCC8CA75D
:109D300047CE61E08CE898E00E949ABA87E198E00B
:109D40000E949CF461E08BEF9BE30E949ABA88E04A
:109D500098E00E943EF6B1100C94EC400C94E54063
:109D600080E00E9406550C94184188E50E9444BA90
:109D700081115F9889E50E9444BA81118A988AE529
:109D80000E9444BA882329F0809108018170809351
:109D9000060185E40E9444BA882309F4C3CC1298D2
:109DA000C1CC0E94E5B9AB01BC014093141750939C
:109DB0001517609316177093171787E194E10E94A7
:109DC0000F93B0CC61E0802F0E9446FC6F2D802F56
:109DD0000E9417FC6F2D70E0802F0E9482FCA7E08C
:109DE000EA1203C0F092CA0B9DCCB9E0EB129ACCF8
:109DF000F092C90B97CC0E94F5B990E08536910599
:109E000014F084E690E0809305188CCC0E94067FC5
:109E10000C943D44A3019201C501B4010F94532C4D
:109E2000181694F081E09AE09F938F9387E19AE06F
:109E30009F938F931F920E9490F90F900F900F9015
:109E40000F900F900C945D448CE09AE0EDCF0E944F
:109E50000DBA0F945F2BCB010E9445690E940DBA89
:109E600020E030E040EA50E40F94532C181614F42C
:109E70000E94067F6091EB087091EC08072E000CA1
:109E8000880B990B0F9404232091E7083091E80880
:109E90004091E9085091EA080F94532C18161CF4CD
:109EA0008AE49AE002C08BE39AE060E00F94160621
:109EB000812F0E94CFCF36CC82E40E9444BA8823FF
:109EC00051F00E94AFEB60938611709387118093DD
:109ED00088119093891183E50E9444BA882351F038
:109EE0000E940DBA6093B6117093B7118093B811A8
:109EF0009093B91184E50E9444BA882351F00E94DE
:109F00000DBA6093BA117093BB118093BC119093FA
:109F1000BD118AE40E9444BA882309F403CC0E944C
:109F20000DBA6B017C012AE037ED43E25CE30F944C
:109F3000532C87FD13C02AE939E949E95EE3C701DB
:109F4000B6010F94FD2218164CF0C092B10BD092BE
:109F5000B20BE092B30BF092B40BE4CB0F9420035E
:109F600088E69CE00F943B02DDCB0F9424038FE343
:109F70009DE00F943B0280911102811117C088E18E
:109F80009DE00F943B028AE00E94DA5340912D023B
:109F900050912E0260912F02709130028FE19DE06E
:109FA0000F94EF028AE00E94DA53BCCB8CE19DE073
:109FB000E8CF88E40E9444BA882321F00E945369C4
:109FC0008093400882E50E9444BA082F83E50E94EE
:109FD00044BA182F011102C0882351F01092E108F1
:109FE0000E946251112321F00E9453698093110253
:109FF00084E40E9444BA882309F494CB0E940DBAE9
:10A0000060932D0270932E0280932F029093300262
:10A0100089CBB7FAB094B7F8B094F70180829182F7
:10A02000A282B382A5CA0F9420038DEA9DE00F940B
:10A030003B0261E08FE99DE00F94160668E270E054
:10A0400088EC90E00F94B7056DCB0C5F1F4FFFEFCE
:10A05000CF1ADF0A20E30A3A120709F059CA32E19F
:10A06000E32E39E0F32E10E0F10181919191A1915D
:10A07000B1911F01F70181939193A193B1937F0156
:10A08000812F0E94A4DD1F5F133071F70E9427C348
:10A0900060E08FE89DE00F94160663E972E084E6C5
:10A0A00090E00F94B7056AEB72E084E690E00F94BD
:10A0B000B70538CBCF5BDF4F0FB6F894DEBF0FBECE
:10A0C000CDBFDF91CF911F910F91FF90EF90DF9067
:10A0D000CF90BF90AF909F908F907F906F905F9048
:10A0E0004F903F902F900895CF92DF92EF92FF9282
:10A0F0000F931F93CF93DF936C018B017A01EC01D7
:10A10000CB5AD74F888187FF04C0FB011182108290
:10A1100024C02CE02C9DC0012D9D900D1124288180
:10A12000AC01420F511D27FD5A952091F71430E0E4
:10A130004217530794F42881AC01420F511D27FDAB
:10A140005A959A01FA01EE0FFF1F2E0F3F1FF901DA
:10A15000E557FB4E208127FD19C088818F5F8883DA
:10A160002CE02C9DC0012D9D900D11242881AC0167
:10A17000420F511D27FD5A952091F71430E04217E8
:10A180005307BCF428812C3044F113C02881820F7E
:10A19000911D27FD9A95FC01EE0FFF1F8E0F9F1F4B
:10A1A000FC01E557FB4E808160E08F770E9417FC31
:10A1B000D4CFF80180819181049680349C4918F4B1
:10A1C00080E49CE904C0F801808191810496F70144
:10A1D000918380838FEF888345C0F801408151814E
:10A1E0002881BC01620F711D27FD7A959B01FB013F
:10A1F000EE0FFF1F2E0F3F1FF901E557FB4E218188
:10A200003281240F351FF701318320832881AC016F
:10A21000420F511D27FD5A959A01FA01EE0FFF1FBB
:10A220002E0F3F1FF901E557FB4E208127FF1AC073
:10A230002881820F911D27FD9A95FC01EE0FFF1FCB
:10A240008E0F9F1FFC01E557FB4E808161E08F77E9
:10A25000DF91CF911F910F91FF90EF90DF90CF9002
:10A260000C9417FCDF91CF911F910F91FF90EF900D
:10A27000DF90CF900895129A0895FF920F931F9345
:10A28000CF93DF931F92CDB7DEB7F82E00EF1DE01E
:10A2900041E050E0B801CE0101960F943722898148
:10A2A0008F1102C081E007C00F5F1F4F8EE00930A1
:10A2B000180771F780E00F90DF91CF911F910F91F8
:10A2C000FF90089580912D0290912E02A0912F026F
:10A2D000B09130028093A90A9093AA0AA093AB0A86
:10A2E000B093AC0A089580915808811107C00E946C
:10A2F000D2C6882319F081E0809358080895909180
:10A30000181793FB882780F993FF06C081E090918E
:10A310001A14911101C080E00895E9ECFBE010826D
:10A3200011820895DC01EC91F0E0CF01880F991FB4
:10A33000E80FF91FE557FB4E80818F7780830895E2
:10A340008F929F92AF92BF92CF92DF92EF92FF9245
:10A350000F93CF93DF931F92CDB7DEB75C016B01F4
:10A360007A014901F501808191810F942D2989831A
:10A37000002311F0F6018083BE016F5F7F4FC4019F
:10A380000E94D5F5F50180819181019691838083AA
:10A39000FFEFCF1ADF0A81E0E81AF10819F780E031
:10A3A0000F90DF91CF910F91FF90EF90DF90CF90C2
:10A3B000BF90AF909F908F9008957F928F929F92C1
:10A3C000AF92BF92CF92DF92EF92FF920F931F93C3
:10A3D000CF93DF931F92CDB7DEB77C0159018B017C
:10A3E0006B01C40ED51E0C151D0559F1F7018080B7
:10A3F0009180F80171908F017982C4010F942D2909
:10A40000781691F0672DC4010F943529C4010F947B
:10A410002D299981891741F00F94240386ED9DE041
:10A420000F943B0281E00EC0BE016F5F7F4FC501FC
:10A430000E94D5F5F70180819181019691838083F7
:10A44000D2CF80E00F90DF91CF911F910F91FF90BD
:10A45000EF90DF90CF90BF90AF909F908F907F90C4
:10A460000895009781F41092900082E0809391000B
:10A470001092950010929400C19A809171008260B0
:10A480008093710008958130910569F41092A000C5
:10A4900082E08093A1001092A5001092A40089BBD5
:10A4A000809372000895029761F41092200182E077
:10A4B0008093210110922501109224018ABB809380
:10A4C000730008957F928F929F92AF92BF92CF9226
:10A4D000DF92EF92FF920F931F93CF93DF93FC01D4
:10A4E0009081943208F0CEC06B017F01892F90E0FB
:10A4F000FC01EE0FFF1F8E0F9F1FFC01E557FB4E67
:10A50000808161E08F770E9446FCF7011182128200
:10A5100080816CE00F94B629FCE08F9FB00111247C
:10A5200040E050E09B01240F351FF901EE0FFF1FA3
:10A530002E0F3F1FF901E557FB4E908197FD08C094
:10A540004F5F5F4F4C30510569F790E00E943152E8
:10A55000F7017080C72DD0E08E01000F111FF801A8
:10A56000EC0FFD1FE557FB4E80818068808377FCF0
:10A5700089C0F0E2CF16F2E0DF060CF041C0F7012F
:10A58000828128E532E0281B310987FD3395220FAF
:10A59000331F220F331F032E000C440B550B8181F8
:10A5A00068E870E04B01881A910887FD9394880C45
:10A5B000991C880C991C092C000CAA08BB08D7FC14
:10A5C0000BC0B601653B710514F064EB70E0072E1B
:10A5D000000C880B990B03C060E070E0CB012819D8
:10A5E00039094A095B090F94432924EB30E040E024
:10A5F00050E00F947529820E931EA41EB51E01C053
:10A600004601F3E2F71558F1F701218188E890E05F
:10A61000821B910927FD9395880F991F880F991F19
:10A620008816990684F0F701228188E592E0821B62
:10A63000910927FD9395880F991F880F991F8816F8
:10A6400099060CF4C40102972FB7F894C00FD11FDC
:10A65000C557DB4E880F991F9A8389832FBF62E30A
:10A6600070E080E090E0DF91CF911F910F91FF901B
:10A67000EF90DF90CF90BF90AF909F908F907F90A2
:10A680000D940C02DF91CF911F910F91FF90EF90ED
:10A69000DF90CF90BF90AF909F908F907F90089564
:10A6A0001F920F920FB60F9211240BB60F922F9399
:10A6B0003F934F935F936F937F938F939F93AF934A
:10A6C000BF93EF93FF9348E251E064E271E082E0D0
:10A6D00090E00E947450FF91EF91BF91AF919F91D4
:10A6E0008F917F916F915F914F913F912F910F903B
:10A6F0000BBE0F900FBE0F901F9018951F920F92D8
:10A700000FB60F9211240BB60F922F933F934F93D6
:10A710005F936F937F938F939F93AF93BF93EF93C9
:10A72000FF9348EA50E064EA70E081E090E00E9424
:10A730007450FF91EF91BF91AF919F918F917F9155
:10A740006F915F914F913F912F910F900BBE0F90A2
:10A750000FBE0F901F9018951F920F920FB60F9279
:10A7600011240BB60F922F933F934F935F936F93E8
:10A770007F938F939F93AF93BF93EF93FF9348E99A
:10A7800050E064E970E080E090E00E947450FF9136
:10A79000EF91BF91AF919F918F917F916F915F9159
:10A7A0004F913F912F910F900BBE0F900FBE0F90C6
:10A7B0001F9018959091C00095FFFCCF8093C60024
:10A7C00008958F929F92AF92BF92EF92FF920F9354
:10A7D0001F93CF93DF93CDB7DEB7A0970FB6F89452
:10A7E000DEBF0FBECDBF611571058105910591F1E9
:10A7F00000E0842E912CA12CB12C102FEE24E39498
:10A80000F12CEC0EFD1EE00EF11C07FDFA94A501E3
:10A8100094010F945329F7016083B901CA010F5FB6
:10A82000611571058105910541F71F3F31F1E1E0A7
:10A83000F0E0EC0FFD1FE10FF11D17FDFA9580818F
:10A840008A3010F097E301C090E3890F0E94DA5339
:10A850001150EBCF80E3A0960FB6F894DEBF0FBE89
:10A86000CDBFDF91CF911F910F91FF90EF90BF90DF
:10A87000AF909F908F900C94DA53A0960FB6F894F7
:10A88000DEBF0FBECDBFDF91CF911F910F91FF9023
:10A89000EF90BF90AF909F908F900895CF92DF92EE
:10A8A000EF92FF926B017C0197FF0BC08DE20E943B
:10A8B000DA53F094E094D094C094C11CD11CE11CF4
:10A8C000F11C4AE0C701B601FF90EF90DF90CF90F6
:10A8D0000C94E1538F929F92AF92BF92CF92DF92EE
:10A8E000EF92FF92CF936B017C01B42E20E030E019
:10A8F000A9010F94FD2287FF07C08DE20E94DA5361
:10A90000F7FAF094F7F8F094C0E060E070E080E0CF
:10A910009FE3CB1541F02DEC3CEC4CEC5DE30F9448
:10A920006323CF5FF6CF9B01AC01C701B6010F9443
:10A93000F3296B017C010F94662B4B015C014AE00B
:10A940000E94E153CC2389F1C501B4010F94022385
:10A950009B01AC01C701B6010F94F2296B017C0188
:10A960008EE20E94DA5320E030E040E251E4C70179
:10A97000B6010F9463234B015C010F945F2B6B01B5
:10A98000770FEE08FF08C701B6010E944E54C701B9
:10A99000B6010F9404239B01AC01C501B4010F94CF
:10A9A000F2296B017C01C150F1F6CF91FF90EF903D
:10A9B000DF90CF90BF90AF909F908F9008958DE0E3
:10A9C0000E94DA538AE00C94DA53CF93DF93EC01C0
:10A9D0008991882319F00E94DA53FACFDF91CF9141
:10A9E0000C94DF548091E1119091E211981759F085
:10A9F000E92FF0E0EF51FE4E82819F5F9F779093A9
:10AA0000E21190E008958FEF9FEF08952F923F920B
:10AA10004F925F926F927F928F929F92AF92BF926E
:10AA2000CF92DF92EF92FF920F931F93CF93DF931A
:10AA3000CDB7DEB728970FB6F894DEBF0FBECDBFF7
:10AA4000E82E0E94D51E0E94A4FD4B015C0180915E
:10AA50000002882359F180914208882339F14091FE
:10AA6000590850915A0860915B0870915C089501F3
:10AA70008401041B150B260B370B37FD2AC08330CE
:10AA800079F03CF4813094F00F94240388E39EE045
:10AA90000BC0843059F40F94240389E09EE004C075
:10AAA0000F94240381E29EE00F943B022091000268
:10AAB00030E0A8EEB3E00F94A729860E971EA81EDB
:10AAC000B91E8092590890925A08A0925B08B092E1
:10AAD0005C0880911102882309F48EC08091E108FE
:10AAE00081118AC08091A00B813021F080911817CC
:10AAF00082FF0CC6F89464990EC66091A90A709101
:10AB0000AA0A8091AB0A9091AC0A789420E030E0D8
:10AB1000A9010F94FD2287FF6FC011E01093E10897
:10AB20008091200B811166C085E296E00E94E55479
:10AB300084E080939A0B82E08093120881E09AE58A
:10AB400090939D1580939C158EE490E090939F15B3
:10AB500080939E1587E08093901582E880939315EB
:10AB600084E890E0A0E0B0E0809394159093951570
:10AB7000A0939615B09397150E942FF510936B1222
:10AB80000E94BEBA40E069E77EE081E796E20E945B
:10AB9000CABA80E30E94DA538AE00E94DA530E9424
:10ABA000B2BA8091400860E0182719F089E495E274
:10ABB0000DC087E69EE00E949ABA80E30E94DA53B5
:10ABC0008AE00E94DA5360E08AE49EE00E949ABA2A
:10ABD00085E59EE00F943B0280E30E94DA538AE011
:10ABE0000E94DA53112331F080E59EE09093200912
:10ABF00080931F090E9405828091A20A843008F088
:10AC00007FC20E94A4FD4B015C018091A20A8111C8
:10AC10001DC08091E1119091E211891B8F77B1F4F1
:10AC20008091C2089091C308A091C408B091C50852
:10AC3000A5019401281B390B4A0B5B0BDA01C901F2
:10AC4000885E9340A109B109B7FF76C560E6F62E8C
:10AC50008091A20A843008F036C18091E111909170
:10AC6000E211891B8F7709F42EC10E94F254AC01C6
:10AC700097FDEECF20916312309164128A3019F063
:10AC80008D3009F0E8C01092C1082115310519F482
:10AC90000F94CE0BDDCFF901EF59F74F10821092D0
:10ACA00064121092631201E618E0F801819180327B
:10ACB00011F48F01FACF8E3409F07AC00115110515
:10ACC00009F476C061EB7FE0C8010F947B226C0130
:10ACD000892B41F06EE470E0C80104960F94462D74
:10ACE000009709F4C8014AE050E060E070E0019686
:10ACF0000F94F31F60935D0870935E0880935F0864
:10AD000090936008409065125090661260906712B0
:10AD1000709068123FEF431A530A630A730A64156E
:10AD200075058605970531F0CD2821F460E08EE7A2
:10AD30009FE0C7C06AE270E0C8010F94752D9C01C6
:10AD4000009709F1982F901BD12C992339F091503D
:10AD5000F801E90FF11D8081D826F7CF4AE050E0D5
:10AD600060E070E0C90101960F94F31F4D2C512C47
:10AD7000612C712C641575058605970541F060E01E
:10AD80008FE59FE09EC060E085E39FE09AC08091E0
:10AD90005D0890915E08A0915F08B0916008809373
:10ADA000651290936612A0936712B093681212C056
:10ADB0008091181780FF0EC06BE271E1C8010F94FB
:10ADC0007B22009709F47AC0FC01838180538A308A
:10ADD00008F474C080916F0281111CC067E470E0B8
:10ADE000C8010F94462D0097A9F04AE050E060E0BA
:10ADF00070E001960F94F31F643071058105910591
:10AE000048F484E99EE00F943B0260E08AE89EE00B
:10AE10000F9416068092C2089092C308A092C408AC
:10AE2000B092C508809161088B3309F411CF8091ED
:10AE3000A20A843008F00CCF80911E09F89EC00150
:10AE4000112461E678E08F5D964F0F94512D81E0DB
:10AE50000E94C2EBFDCE2F3531050CF0F9CE8C35BA
:10AE6000C1F40E94F25497FDF3CE2091C108211144
:10AE7000EFCE2091631230916412A9014F5F5F4FB2
:10AE80005093641240936312F901EF59F74F808396
:10AE9000DFCE8B3321F481E08093C108D9CE80913D
:10AEA000C1088111D5CEC901019690936412809397
:10AEB0006312F901EF59F74F4083CACE60E08BE08F
:10AEC0009FE00E940FB98091181782FF19C18091ED
:10AED000A20A811102C01092C708DD24D3944091C8
:10AEE00014175091151760911617709117178091CC
:10AEF000101790911117A0911217B09113174817BE
:10AF000059076A077B0708F4D12C00E010E0CC2435
:10AF1000C39430E6B32E44E6A42E59E6952E8091D4
:10AF2000A20A843008F0ECC0D110EAC08091C708B2
:10AF30008111E6C080911F1490912014A0912114DA
:10AF4000B09122148093141790931517A09316179D
:10AF5000B093171741E050E0BE016F5F7F4F87E16C
:10AF600094E10E94F496019719F4898190E002C05F
:10AF70008FEF9FEFF82E40901417509015176090A8
:10AF80001617709017174091101750911117609174
:10AF9000121770911317DD24D394441655066606D4
:10AFA000770608F4D12C4416550666067706B0F4E9
:10AFB000019609F461C02AE0F21609F46EC03DE082
:10AFC000F31609F46AC043E2F41619F05AE3F512D5
:10AFD0007CC08091C608811178C054C00E9405824F
:10AFE00087E194E10E947B9680910F17882339F1C5
:10AFF000815080930F17989EC001112441E061E0B9
:10B000008B5D944F0E947379E0910F1764E0E69F87
:10B01000F0011124EF5DF44F408151816281738111
:10B0200040931417509315176093161770931717C2
:10B0300087E194E10E940F930E94277616C00E9438
:10B0400016760E946A830E94B67F0F9411046D33B6
:10B0500071058105910518F48CEB9FE002C081EC2D
:10B060009FE00E9438B9A09205188091181782FDC0
:10B070000DC084ED9FE004C00F94200385EC9FE099
:10B080000F943B0273E2F71208C005C053E2F512B9
:10B0900060C300E010E0C092C7081092C608011516
:10B0A000110519F40F94CE0B0DC080911E09B89EA6
:10B0B000000D111D1124F801EF5DF64F108280E0A4
:10B0C0000E94C2EB00E010E02ACF0F35110508F016
:10B0D00026CF8BE3F81203C0C092C60820CF809120
:10B0E000C60881111CCF80911E09F801B89EE00DA1
:10B0F000F11D1124EF5DF64FF0820F5F1F4F0FCF50
:10B100000E94A4FD4B015C0140913C0850913D0818
:10B1100060913E0870913F08411551056105710528
:10B1200029F18091701390917113A0917213B091D5
:10B130007313840F951FA61FB71F95018401081B69
:10B14000190B2A0B3B0B37FD11C00F9420036091A4
:10B15000AF0B7091B00B88EE9FE00F940D038AE067
:10B160000E94DA5380E090E00E943EF64091310266
:10B1700050913202609133027091340241155105B1
:10B180006105710509F44EC09091FE148091FF1481
:10B19000981759F00E94A4FD609370137093711377
:10B1A00080937213909373133DC08091200B811193
:10B1B00037C0E11035C08091701390917113A09148
:10B1C0007213B0917313840F951FA61FB71FA501AB
:10B1D0009401281B390B4A0B5B0B57FD21C0809152
:10B1E000D80881111FC081E08093D8085F9A8091B0
:10B1F00078138E7F809378138A9A809178138D7F4D
:10B200008093781380910801809581708093060166
:10B21000809178138B7F809378130E943B5102C0FA
:10B220001092D8088091D4089091D508A091D608A2
:10B23000B091D708B501A401481B590B6A0B7B0BD1
:10B2400077FDAAC19091FE148091FF1420913502E0
:10B250001091360298130EC06091C90B269FB00161
:10B260001124660F672F661F770B7195062F80914B
:10B27000CA0B17C08091FF1458E5859FC0011124A7
:10B280008D50944FFC01EA5AFF4F0081029FB0019C
:10B290001124660F672F661F770B7195062F319665
:10B2A0008081819FB0011124660F672F661F770B85
:10B2B0007195162F002331F10E94A4FDC090CC0897
:10B2C000D090CD08E090CE08F090CF08DC01CB0103
:10B2D000C114D104E104F10469F48C599F4FAF4FBC
:10B2E000BF4F8093CC089093CD08A093CE08B09325
:10B2F000CF0806C08C199D09AE09BF09B7FF0AC067
:10B300000FEF08C01092CC081092CD081092CE0812
:10B310001092CF08602F70E089E00E9482FC112318
:10B3200031F10E94A4FDC090D008D090D108E090E7
:10B33000D208F090D308DC01CB01C114D104E104A0
:10B34000F10469F48C599F4FAF4FBF4F8093D008E1
:10B350009093D108A093D208B093D30806C08C195B
:10B360009D09AE09BF09B7FF0AC01FEF08C01092C0
:10B37000D0081092D1081092D2081092D308612FF1
:10B3800070E087E00E9482FC80910813882309F412
:10B39000F6C0E0901E02F0901F0200912002109172
:10B3A00021026091E40B7091E50B6E5F7F4F072ED9
:10B3B000000C880B990B0F9404239701A8010F949C
:10B3C000FD2287FDDCC03090FF14212C1A821B82E5
:10B3D0001C828091FE14831509F467C0832D90E0D0
:10B3E00068E5689FF001699FF00D1124ED50F44F5E
:10B3F000458956896789708D452B462B472B89F4E3
:10B40000418D528D638D748D452B462B472B49F40E
:10B41000458D568D678D70A1452B462B472B09F422
:10B420003FC078E5789F9001799F300D1124C901C4
:10B430008D50944F6C01FC016181728183819481F4
:10B440000F94A12C2B013C01F60161A172A183A1F3
:10B4500094A10F9402236D837E838F839887F601D6
:10B4600065A176A187A190A50F9402239B01AC0151
:10B470006D817E818F8198850F94ED2AA3019201C1
:10B480000F9463233B016C01222D3A814B815C8137
:10B490000F94532C181624F4262C7A82CB82DC824B
:10B4A00081E0830D8F70382E94CF2091220230914D
:10B4B00023024091240250912502622D7A818B81D2
:10B4C0009C810F9463239701A8010F94F3293B01FA
:10B4D0006C0120901A0230901B0240901C02509088
:10B4E0001D029B01AC01B701C8010F94532C181623
:10B4F0006CF09101A201B301C6010F94532C1816F0
:10B500001CF47101820102C0730186014090C808D9
:10B510005090C9086090CA087090CB089701A801A4
:10B52000C301B2010F94532C1816C4F420E037ED78
:10B5300043EA5CE3B701C8010F9463236B017C010C
:10B5400028E431EE4AE75FE3C301B2010F946323BD
:10B55000A70196010F94F3297B018C01C701D80143
:10B560008093C8089093C908A093CA08B093CB08E9
:10B57000B701C8010F945F2BCB010E9451D7F4E6AD
:10B580008F0E911CA11CB11C8092D4089092D508FA
:10B59000A092D608B092D7080F94CE0B8091A00B42
:10B5A000813009F06EC00E94A4FD6B017C01809186
:10B5B000DD089091DE08A091DF08B091E0089701C6
:10B5C0008601081B190B2A0B3B0B37FD3AC08090F4
:10B5D000A10B9090A20BA090A30BB090A40B0F9482
:10B5E00011046093A10B7093A20B8093A30B909313
:10B5F000A40B0091020910910309209104093091D4
:10B600000509081919092A093B09DC01CB01800F3A
:10B61000911FA21FB31F8093020990930309A09367
:10B620000409B0930509D701C601805F984DAF4F5B
:10B63000BF4F8093DD089093DE08A093DF08B0939E
:10B64000E0088091D9089091DA08A091DB08B091C8
:10B65000DC08A7019601281B390B4A0B5B0B57FD31
:10B6600010C030E8C30E3EEED31EE11CF11CC092A8
:10B67000D908D092DA08E092DB08F092DC080E9448
:10B68000907F0F942F0580913B08882391F00E94B2
:10B69000A4FD0091370810913808209139083091A5
:10B6A0003A08DC01CB01801B910BA20BB30BB7FF57
:10B6B00053C00E94A4FD6B017C0120913608222317
:10B6C00009F468C08091320890913308A091340841
:10B6D000B0913508B701A601481B590B6A0B7B0BCB
:10B6E00077FD58C030E0A8EEB3E00F94A729C60E4E
:10B6F000D71EE81EF91EC0923208D0923308E0929D
:10B700003408F09235080E94EF7544C08091200BF8
:10B710008111F0C971CA80912D0290912E02A091E1
:10B720002F02B09130028093A90A9093AA0AA093A5
:10B73000AB0AB093AC0AE1C986EB9FE00F943B02E1
:10B740008092C2089092C308A092C408B092C50823
:10B750007DCA1092C608A6CC0E94A4FD6B017C0194
:10B7600020913B0830E0A8EEB3E00F94A729C60E65
:10B77000D71EE81EF91EC0923708D0923808E09212
:10B780003908F0923A0880E00E9458CF8AE00E947F
:10B79000DA538FCF28960FB6F894DEBF0FBECDBF19
:10B7A000DF91CF911F910F91FF90EF90DF90CF909D
:10B7B000BF90AF909F908F907F906F905F904F90D1
:10B7C0003F902F9008951F920F920FB60F92112461
:10B7D0000F900FBE0F901F9018951F920F920FB6EB
:10B7E0000F9211240BB60F920F931F932F933F9339
:10B7F0004F935F936F937F938F939F93AF93BF9379
:10B80000CF93DF93EF93FF930091E211D091E11179
:10B8100011E01D0F1F77C091C60090915408492F69
:10B82000092E000C550B660B770B4131510508F0C2
:10B8300064C0FA018827E256FF4F8F4F0D94EA2922
:10B84000CD3449F0CE34B9F481E006C0CA3338F0C3
:10B85000CD3409F043C082E08093540876C0C033F1
:10B8600008F073C0C03209F470C0CD32B9F56DC0B4
:10B87000C13351F018F4C03289F567C0C43331F0D8
:10B88000C83361F58BE0E8CF83E0E6CF88E0E4CF12
:10B89000C03321F0C13311F586E0DECF84E0DCCF88
:10B8A000C833E1F485E0D8CFC233C1F487E0D4CF08
:10B8B000C133A1F489E0D0CFC03381F48AE0CCCF8A
:10B8C000C73361F48CE0C8CFC63341F48DE0C4CFF8
:10B8D000C032D9F1C33511F48EE0BECF80E1BCCFC8
:10B8E00080ED8C0F8A3088F59FE090935408809308
:10B8F00053082BC0CA3049F526C0CA3031F58091B3
:10B90000FE15882301F1973089F03CF49530D9F485
:10B91000109210021092041816C09A3059F09F30FD
:10B9200091F4809153080E94F6BA0DC081E0809393
:10B93000BF1D09C00E94C0830E9405828EEF0E9435
:10B9400018E30E9486E310925408011731F0ED2F9E
:10B95000F0E0EF51FE4EC283D12FD093E111FF9161
:10B96000EF91DF91CF91BF91AF919F918F917F9197
:10B970006F915F914F913F912F911F910F910F9078
:10B980000BBE0F900FBE0F901F9018958EBD0DB47B
:10B9900007FEFDCF08958FEF8EBD0DB407FEFDCFDE
:10B9A0008EB50895909164009B7F90936400982FCA
:10B9B000906A96959CBD80FD03C091E0863009F4A5
:10B9C00090E09DBD08952F923F924F925F926F92AB
:10B9D0007F928F929F92AF92BF92CF92DF92EF921F
:10B9E000FF920F931F93CF93DF93CDB7DEB72F97BF
:10B9F0000FB6F894DEBF0FBECDBF8FEF9FEF9093D1
:10BA00008900809388001AE0D12E1F861E867894C4
:10BA10008091F00A9091F10AA091F20AB091F30A94
:10BA2000892B8A2B8B2B09F0D5C18091A21D8823ED
:10BA3000D1F01092A21D8091A01D9091A11D892B83
:10BA400091F01092B10A1092A11D1092A01D909138
:10BA5000FE148091FF14981731F08091FF148F5FCE
:10BA60008F708093FF148091A01D9091A11D892B50
:10BA700009F4B0C10091EC0A1091ED0A2091EE0A90
:10BA80003091EF0A8091E80A9091E90AA091EA0AC0
:10BA9000B091EB0A4091DF0A50E060E070E0801B5B
:10BAA000910BA20BB30B481759076A077B0710F4D9
:10BAB000DB01CA01482F800F911FA21FB31F809383
:10BAC000EC0A9093ED0AA093EE0AB093EF0A8091EE
:10BAD0008400909185004E968090B60A9090B70AA7
:10BAE000A090B80AB090B90A0091C60A1091C70A8E
:10BAF0002091C80A3091C90A080D191D2A1D3B1D45
:10BB00000093C60A1093C70A2093C80A3093C90A43
:10BB100037FD1CC0889A0091A50A002E000C110B5D
:10BB2000220B330B8090AF1D9090B01DA090B11DE3
:10BB3000B090B21D080D191D2A1D3B1D0093AF1DAD
:10BB40001093B01D2093B11D3093B21D8090BA0A9E
:10BB50009090BB0AA090BC0AB090BD0A0091CA0A9E
:10BB60001091CB0A2091CC0A3091CD0A080D191DF5
:10BB70002A1D3B1D0093CA0A1093CB0A2093CC0ABE
:10BB80003093CD0A37FD1CC08E9A0091A60A002E74
:10BB9000000C110B220B330B8090B31D9090B41D41
:10BBA000A090B51DB090B61D080D191D2A1D3B1D96
:10BBB0000093B31D1093B41D2093B51D3093B61D93
:10BBC0008090BE0A9090BF0AA090C00AB090C10AAF
:10BBD0000091CE0A1091CF0A2091D00A3091D10A5B
:10BBE000080D191D2A1D3B1D0093CE0A1093CF0A84
:10BBF0002093D00A3093D10A37FD21C020910B0148
:10BC000020952870209309010091A70A002E000CAE
:10BC1000110B220B330B8090B71D9090B81DA09094
:10BC2000B91DB090BA1D080D191D2A1D3B1D0093AA
:10BC3000B71D1093B81D2093B91D3093BA1D809085
:10BC4000C20A9090C30AA090C40AB090C50A00919D
:10BC5000D20A1091D30A2091D40A3091D50A080D46
:10BC6000191D2A1D3B1D0093D20A1093D30A20935D
:10BC7000D40A3093D50A37FD1CC0149A0091A80A43
:10BC8000002E000C110B220B330B8090BB1D9090EB
:10BC9000BC1DA090BD1DB090BE1D080D191D2A1D14
:10BCA0003B1D0093BB1D1093BC1D2093BD1D309305
:10BCB000BE1D209184003091850028173907C8F3F4
:10BCC0000091C60A1091C70A2091C80A3091C90A8A
:10BCD00037FD15C08090B20A9090B30AA090B40AC4
:10BCE000B090B50A081919092A093B090093C60A38
:10BCF0001093C70A2093C80A3093C90A8898009104
:10BD0000CA0A1091CB0A2091CC0A3091CD0A37FD96
:10BD100015C08090B20A9090B30AA090B40AB09077
:10BD2000B50A081919092A093B090093CA0A109390
:10BD3000CB0A2093CC0A3093CD0A8E980091CE0A7C
:10BD40001091CF0A2091D00A3091D10A37FD19C045
:10BD50008090B20A9090B30AA090B40AB090B50A4D
:10BD6000081919092A093B090093CE0A1093CF0A32
:10BD70002093D00A3093D10A20910B012870209390
:10BD800009010091D20A1091D30A2091D40A30916E
:10BD9000D50A37FD15C08090B20A9090B30AA090E2
:10BDA000B40AB090B50A081919092A093B09009389
:10BDB000D20A1093D30A2093D40A3093D50A149848
:10BDC000415041F0209184003091850028173907B7
:10BDD000C8F381CE8091F00A9091F10AA091F20A05
:10BDE000B091F30A892B8A2B8B2B11F00C941165DF
:10BDF000E091A01DF091A11D309711F40C9498666C
:10BE00008091EC0A9091ED0AA091EE0AB091EF0AB0
:10BE10004091E80A5091E90A6091EA0A7091EB0AB0
:10BE200084179507A607B70708F46EC08091110222
:10BE3000882309F44EC085899689A789B08D892BFE
:10BE40008A2B8B2BA1F4818D928DA38DB48D892BA0
:10BE50008A2B8B2B61F4858D968DA78DB0A1892BB4
:10BE60008A2B8B2B21F48091200B882391F161A1E7
:10BE700072A183A194A18090A90A9090AA0AA0908F
:10BE8000AB0AB090AC0AEB5BFF4F208123FF07C0E9
:10BE900090958095709561957F4F8F4F9F4F0F9430
:10BEA00004232091D70B3091D80B4091D90B50919E
:10BEB000DA0B0F9463239B01AC01C501B4010F940D
:10BEC000F2296093A90A7093AA0A8093AB0A90930F
:10BED000AC0A1092B10A1092A11D1092A01D90916F
:10BEE000FE148091FF14981711F40C9498668091B9
:10BEF000FF148F5F8F708093FF14B0ED4B2EB7E06F
:10BF00005B2E612C712CE7C34091E40A5091E50A45
:10BF10006091E60A7091E70A481759076A077B079C
:10BF200008F4A5C18090E00A9090E10AA090E20A8E
:10BF3000B090E30A85A996A9A7A9B0AD881699067D
:10BF4000AA06BB0608F077C181149104A104B104CC
:10BF500049F48091AD0A9091AE0AA091AF0AB091D8
:10BF6000B00A65C1B0E0AC2D882D392D2A2DF9819C
:10BF7000EA817B816C815D814E819F815091A50B0F
:10BF8000589F712D66274091A60B489F700D611D2B
:10BF90001090A70B189E600D539F700D611D439F5D
:10BFA000600D529F600DF72FE62FF79F512D44270C
:10BFB0009927F69F500D411D9B1FE79F500D411D76
:10BFC0009B1FE69F400D911DF42FE92FF79FA12D98
:10BFD00044279927F69FA00D411D9B1FE79FA00DA9
:10BFE000411D9B1FE69F400D911DF42FE92F552702
:10BFF0008091AD0A3091AE0A2091AF0A00904F08AF
:10C000000B2A09F484C040914B084F9F51198B0BA8
:10C010003B0B2B0B90914C089F9F501981093B0BB8
:10C020002B0BA0914D08AF9F801931092B0B4E9F10
:10C03000501981093B0B2B0B9E9F801931092B0B4B
:10C04000AE9F30192109F79FA12D44279927F69F0C
:10C05000A00D411D9B1FE79FA00D411D9B1FE69F4B
:10C06000400D911DF42FE92F409147084F9F510D2E
:10C070008B1F3B1F2B1F909148089F9F500D811DC8
:10C080003B1F2B1FA0914908AF9F800D311D2B1F17
:10C090004E9F500D811D3B1F2B1F9E9F800D311DFC
:10C0A0002B1FAE9F300D211DF79FA12D44279927EF
:10C0B000F69FA00D411D9B1FE79FA00D411D9B1FDB
:10C0C000E69F400D911DF42FE92F409143084F9FAB
:10C0D00051198B0B3B0B2B0B909144089F9F5019D0
:10C0E00081093B0B2B0BA0914508AF9F80193109AB
:10C0F0002B0B4E9F501981093B0B2B0B9E9F8019D8
:10C1000031092B0BAE9F301921090C940961409124
:10C110004B084F9F510D8B1F3B1F2B1F90914C08BD
:10C120009F9F500D811D3B1F2B1FA0914D08AF9F5E
:10C13000800D311D2B1F4E9F500D811D3B1F2B1F4E
:10C140009E9F800D311D2B1FAE9F300D211DF79F2F
:10C15000A12D44279927F69FA00D411D9B1FE79F06
:10C16000A00D411D9B1FE69F400D911DF42FE92F4F
:10C17000409147084F9F51198B0B3B0B2B0B909114
:10C1800048089F9F501981093B0B2B0BA091490830
:10C19000AF9F801931092B0B4E9F501981093B0B22
:10C1A0002B0B9E9F801931092B0BAE9F3019210953
:10C1B000F79FA12D44279927F69FA00D411D9B1F96
:10C1C000E79FA00D411D9B1FE69F400D911DF42F81
:10C1D000E92F409143084F9F510D8B1F3B1F2B1F91
:10C1E000909144089F9F500D811D3B1F2B1FA091D4
:10C1F0004508AF9F800D311D2B1F4E9F500D811D97
:10C200003B1F2B1F9E9F800D311D2B1FAE9F300D9E
:10C21000211D1124CA2EF983EA837B836C835D83FD
:10C220004E839F8390E0932BA0E0B0E0A22B20E50B
:10C2300039E111E011C081A992A9A3A9B4A9F7CF4E
:10C24000B695A79597958795110F2C5F3F4F49E1BC
:10C250002C36340709F43BC4F90145915591659199
:10C260007491481759076A077B0750F330C440910F
:10C27000DB0A5091DC0A6091DD0A7091DE0A4817F2
:10C2800059076A077B0708F0B9C18091DA0A811162
:10C290001FC0DF01AF5BBF4FED90FD900D911C9172
:10C2A00013971D962D913D914D915C9161A972A9B5
:10C2B00083A994A90E94FB7C51E05093DA0AE09193
:10C2C000A01DF091A11D81A892A8A3A8B4A887C120
:10C2D0008091D60A9091D70AA091D80AB091D90A34
:10C2E00041AD52AD63AD74AD84179507A607B7078E
:10C2F00008F06FC10097A105B10549F48090AD0A1F
:10C300009090AE0AA090AF0AB090B00A68C130E039
:10C310004885882E292F8A2FE9857A856B855C854B
:10C320009D859091A50B989D612D55272090A60B7A
:10C33000289C600D511D1090A70B189C500D929FCA
:10C34000600D511D229E500D989F500DE62F752FA8
:10C35000E69F912D22243324E59F900D211C331E4E
:10C36000769F900D211C331E759F200C311CE22DF1
:10C37000732DE69F412D22243324E59F400D211C7F
:10C38000331E769F400D211C331E759F200C311CDF
:10C39000E22D732D99278090AD0A2091AE0A8091ED
:10C3A000AF0A00904F08032A09F484C020904B087C
:10C3B0002E9E9119830A230B830B30904C083E9ECE
:10C3C00090198108230B830B40914D084E9F8018D4
:10C3D0002109830B279E90198108230B830B379E1D
:10C3E00080182109830B479F20198109E69F412D61
:10C3F00022243324E59F400D211C331E769F400DDF
:10C40000211C331E759F200C311CE22D732D2090B2
:10C4100047082E9E910D831E231F831F30904808CE
:10C420003E9E900D811C231F831F409149084E9F03
:10C43000800C211D831F279E900D811C231F831FAD
:10C44000379E800C211D831F479F200D811DE69F75
:10C45000412D22243324E59F400D211C331E769F5D
:10C46000400D211C331E759F200C311CE22D732DB5
:10C47000209043082E9E9119830A230B830B309042
:10C4800044083E9E90198108230B830B4091450878
:10C490004E9F80182109830B279E90198108230B3A
:10C4A000830B379E80182109830B479F2019810930
:10C4B0000C94DC6220904B082E9E910D831E231F4E
:10C4C000831F30904C083E9E900D811C231F831FBC
:10C4D00040914D084E9F800C211D831F279E900D7B
:10C4E000811C231F831F379E800C211D831F479FA4
:10C4F000200D811DE69F412D22243324E59F400D10
:10C50000211C331E769F400D211C331E759F200C6D
:10C51000311CE22D732D209047082E9E9119830A1D
:10C52000230B830B309048083E9E90198108230B03
:10C53000830B409149084E9F80182109830B279E49
:10C5400090198108230B830B379E80182109830BD8
:10C55000479F20198109E69F412D22243324E59F1E
:10C56000400D211C331E769F400D211C331E759FEC
:10C57000200C311CE22D732D209043082E9E910D2E
:10C58000831E231F831F309044083E9E900D811C04
:10C59000231F831F409145084E9F800C211D831F40
:10C5A000279E900D811C231F831F379E800C211D09
:10C5B000831F479F200D811D11244887E9877A87B3
:10C5C0006B875C879D87912C922AA12CB12CA82A7D
:10C5D00006C0E25BFF4F80809180A280B38080E53F
:10C5E00099E121E0FC0145915591659174914815BF
:10C5F00059056A057B0508F4CDC2D7C280911202A5
:10C6000090911302A0911402B0911502B7FF5BC084
:10C61000EA5BFF4F80809180A280B38080E599E142
:10C6200021E0FC014591559165917491481559059A
:10C630006A057B0550F4B694A79497948794220FCB
:10C640000496A9E18C369A0761F72093DF0AB0E2DD
:10C650008B169104A104B10408F43BC320E2821AB2
:10C660009108A108B108811438E09306A104B1042F
:10C6700008F40BC344E0949EC0011124805B9A4EE1
:10C68000FC01329625913491782D6627739FA00185
:10C69000729F410D561F0694461F561F112460E0DD
:10C6A00070E0FC0125913491C901A0E0B0E0841B49
:10C6B000950BA60BB70B8093120290931302A093D5
:10C6C0001402B09315024090120250901302609031
:10C6D0001402709015028091A01D9091A11D892BCC
:10C6E00009F097C10E948F7D9093A11D8093A01D9A
:10C6F000892B09F48EC1E091A01DF091A11D8081CC
:10C7000083FF3EC0858D968DA78DB0A1418D528D42
:10C71000638D748D058916892789308D0093AF1D2F
:10C720001093B01D2093B11D3093B21D4093B31DE3
:10C730005093B41D6093B51D7093B61D8093B71DC3
:10C740009093B81DA093B91DB093BA1D81A192A179
:10C75000A3A1B4A18093BB1D9093BC1DA093BD1D4C
:10C76000B093BE1D9091FE148091FF14981709F4A8
:10C77000B9CF8091FF148F5F8F708093FF14B2CF79
:10C78000058916892789308D81E00115110521055C
:10C79000310509F480E0818C928CA38CB48C8114D7
:10C7A0009104A104B10409F08260458D568D678D16
:10C7B00070A1411551056105710509F084608093F0
:10C7C000B10A1092D60A1092D70A1092D80A109283
:10C7D000D90A1092E00A1092E10A1092E20A10922D
:10C7E000E30A85A196A1A7A1B0A58093E80A90933A
:10C7F000E90AA093EA0AB093EB0A442455243201D3
:10C80000481A590A6A0A7B0A4092C60A5092C70A15
:10C810006092C80A7092C90A4092CA0A5092CB0A22
:10C820006092CC0A7092CD0A4092CE0A5092CF0A02
:10C830006092D00A7092D10A4092D20A5092D30AE2
:10C840006092D40A7092D50A41A052A063A074A04D
:10C85000440C551C661C771C000F111F221F331F30
:10C860000093B60A1093B70A2093B80A3093B90A16
:10C87000880C991CAA1CBB1C8092BA0A9092BB0A15
:10C88000A092BC0AB092BD0A440F551F661F771FC5
:10C890004093BE0A5093BF0A6093C00A7093C10AC6
:10C8A0004092C20A5092C30A6092C40A7092C50AAA
:10C8B000880F991FAA1FBB1F8093B20A9093B30AD7
:10C8C000A093B40AB093B50A1092EC0A1092ED0A44
:10C8D0001092EE0A1092EF0A81A592A5A3A5B4A525
:10C8E0008093E40A9093E50AA093E60AB093E70ADE
:10C8F00085A596A5A7A5B0A98093DB0A9093DC0A2D
:10C90000A093DD0AB093DE0AEB5BFF4F808190912C
:10C910001009891721F0809310090E944D7D0E9413
:10C92000DCC08FEF9FEFDC01809312029093130223
:10C93000A0931402B0931502E091A01DF091A11DE7
:10C94000DF01DD96ED90FD900D911C9121A932A99A
:10C9500043A954A9E65BFF4F608171818281938175
:10C960000E94FB7C1092DA0AE091A01DF091A11DBB
:10C97000E65BFF4F80809180A280B38080E599E1E3
:10C9800021E0FC0145915591659174914815590537
:10C990006A057B0558F4B694A79497948794220F60
:10C9A00004964CE659E14817590759F72093DF0AD6
:10C9B00050E285169104A104B10408F4B3C190E2D9
:10C9C000891A9108A108B1088114A8E09A06A10467
:10C9D000B10408F484C1B4E09B9EC0011124805BC3
:10C9E0009A4EFC01329625913491782D6627739FDB
:10C9F000A001729F410D561F0694461F561F112419
:10CA0000FC0145905490612C712C441A550A610820
:10CA100071084092F00A5092F10A6092F20A709204
:10CA2000F30A8091F00A9091F10AA091F20AB09174
:10CA3000F30AAC01BD01009721E0A207B10520F087
:10CA40004FEF5FEF60E070E0841B950BA60BB70B18
:10CA50008093F00A9093F10AA093F20AB093F30A3C
:10CA6000F89480918400909185004096DA94DD20BE
:10CA700061F0AE85BF85A40FB51FBF87AE87A8172D
:10CA8000B90710F40C94075D02C09F878E872E852E
:10CA90003F85309389002093880078942F960FB6B5
:10CAA000F894DEBF0FBECDBFDF91CF911F910F91E4
:10CAB000FF90EF90DF90CF90BF90AF909F908F90BE
:10CAC0007F906F905F904F903F902F9008951093BC
:10CAD000DF0A80329105A105B10508F456C08097A0
:10CAE000A109B109811528E09207A105B105F0F06F
:10CAF00044E0949F90011124205B3A4EF901329654
:10CB000045915491EE27859FB001849F610D7E1F52
:10CB100006946E1F7E1F1124F90145905490612CDC
:10CB2000712C461A570A6108710822C0AC01BD0178
:10CB30007695679557954795FA01EC7FAF01405B75
:10CB40005E4EFA0125913491FA0132966591749105
:10CB50008770869FA001879F500D1124A3E05695F2
:10CB60004795AA95E1F72901441A550A612C712CC1
:10CB7000840C951CA61CB71C8092E00A9092E10AD6
:10CB8000A092E20AB092E30AA6CD80E290E0A0E093
:10CB9000B0E0A5CFB694A79497948794220F0496FB
:10CBA00059E18C36950709F01DCD2093DF0A70E21C
:10CBB00087169104A104B10408F461C070E2871AD9
:10CBC0009108A108B108811488E09806A104B10475
:10CBD000F8F0A4E09A9EC0011124805B9A4EFC01FB
:10CBE000329625913491B82D6627B39FA001B29F4C
:10CBF000410D561F0694461F561F1124FC014590F7
:10CC00005490612C712C441A550A6108710822C095
:10CC1000D501C401B695A79597958795FC01EC7F42
:10CC2000CF01805B9E4EFC0145905490FC013296F2
:10CC300025913491482D4770429FC001439F900D2C
:10CC40001124E3E096958795EA95E1F7481A590A89
:10CC5000612C712C8091D60A9091D70AA091D80AA4
:10CC6000B091D90A840D951DA61DB71D8093D60AD3
:10CC70009093D70AA093D80AB093D90A2CCD60E23A
:10CC8000862E912CA12CB12C99CFD501C401B6953B
:10CC9000A79597958795FC01EC7FCF01805B9E4E11
:10CCA000FC0125913491FC01329645915491682DF7
:10CCB0006770649FC001659F900D112463E0969595
:10CCC00087956A95E1F7281B390BC901A0E0B0E010
:10CCD000F2CC40E2842E912CA12CB12CBFCCD501FA
:10CCE000C401B695A79597958795FC01EC7FCF0178
:10CCF000805B9E4EFC0145905490FC01329625913C
:10CD00003491482D4770429FC001439F900D1124DC
:10CD1000A3E096958795AA95E1F7481A590A612CE0
:10CD2000712C77CE90E2892E912CA12CB12C47CE7C
:10CD300080ED482E87E0582E612C712CD3CC2F9299
:10CD40003F924F925F926F927F928F929F92AF929B
:10CD5000BF92CF92DF92EF92FF921F93CF93DF9318
:10CD600000D01F92CDB7DEB74A011901FC01408007
:10CD7000518062807380FB01C080D180E280F380AB
:10CD80002091061830910718409108185091091801
:10CD9000C301B2010F94FD2281110EC011E0A70161
:10CDA000960160910A1870910B1880910C1890915F
:10CDB0000D180F94FD22811110E080E1E6E0F8E10A
:10CDC000A5E6B7E101900D928A95E1F7F401808024
:10CDD0009180A280B3802091160230911702409179
:10CDE000180250911902C501B4010F94FD22882345
:10CDF00079F180926D1790926E17A0926F17B09292
:10CE000070178092160290921702A0921802B092A8
:10CE1000190220E030E040E05FE36091A2117091E0
:10CE2000A3118091A4119091A5110F94632369839C
:10CE30007A838B839C83CE0101960E946EE180E110
:10CE4000E6E0F8E1A5E6B7E101900D928A95E1F7F9
:10CE50004092651750926617609267177092681734
:10CE6000C0926917D0926A17E0926B17F0926C1714
:10CE7000F10120813181428153816091711770915C
:10CE8000721780917317909174170F94F329609320
:10CE900071177093721780937317909374171123FF
:10CEA00079F02AEF3EE74AE25FE36091A6117091C4
:10CEB000A7118091A8119091A9110F94632304C028
:10CEC00060E070E080EA91E469837A838B839C83DD
:10CED000CE0101960E946EE180E1E6E0F8E1A5E670
:10CEE000B7E101900D928A95E1F70F900F900F90A6
:10CEF0000F90DF91CF911F91FF90EF90DF90CF9037
:10CF0000BF90AF909F908F907F906F905F904F9069
:10CF10003F902F9008950F931F93CF93DF93CDB73A
:10CF2000DEB728970FB6F894DEBF0FBECDBF8C01D9
:10CF30000E9496FB1D821E821F82188620E030E030
:10CF400040E05FE360910E1870910F188091101807
:10CF5000909111180F94F32969837A838B839C83B2
:10CF60009E012B5F3F4FAE014F5F5F4F6AE078E15C
:10CF700086E098E10E949F661D821E821F821886AD
:10CF800020E030E040E05FE3F80160857185828554
:10CF900093850F94F32969837A838B839C83B801EB
:10CFA0006C5F7F4F9E012B5F3F4FAE014F5F5F4F26
:10CFB000C8010E949F6628960FB6F894DEBF0FBE88
:10CFC000CDBFDF91CF911F910F9108952F923F9286
:10CFD0004F925F926F927F928F929F92AF92BF9289
:10CFE000CF92DF92EF92FF920F931F93CF93DF9335
:10CFF000CDB7DEB7A0970FB6F894DEBF0FBECDBF9A
:10D000008C011B014090061850900718609008187A
:10D010007090091880900A1890900B18A0900C1826
:10D02000B0900D18DC018D919D910D90BC91A02DBB
:10D030008D879E87AF87B88B9C01AD01C301B2017C
:10D040000F94F2296B017C01D80114968D919D916A
:10D050000D90BC91A02D898B9A8BAB8BBC8B9C01C6
:10D06000AD01C501B4010F94F2296D8B7E8B8F8BBE
:10D07000988FD1018D919D910D90BC91A02D8D83A4
:10D080009E83AF83B8879C01AD01C301B2010F94A9
:10D09000F229698F7A8F8B8F9C8FD10114968D9195
:10D0A0009D910D90BC91A02D89879A87AB87BC87F5
:10D0B0009C01AD01C501B4010F94F2296D8F7E8FE3
:10D0C0008F8F98A3A7019601C701B6010F94632320
:10D0D0006B017C012D893E894F89588DCA01B901A8
:10D0E0000F9463239B01AC01C701B6010F94F32990
:10D0F0004B015C012D853E854F8558896D817E8170
:10D100008F8198850F94F2292B013C0129893A8956
:10D110004B895C8969857A858B859C850F94F2297A
:10D120006B017C01A3019201C301B2010F9463233F
:10D130002B013C01A7019601C701B6010F9463239F
:10D140009B01AC01C301B2010F94F3290F94A12CF0
:10D150006B017C01298D3A8D4B8D5C8DCA01B90123
:10D160000F9463232B013C012D8D3E8D4F8D58A1D3
:10D17000CA01B9010F9463239B01AC01C301B20141
:10D180000F94F3299B01AC01C501B4010F94532CFA
:10D190001816E4F420E030E0A901C701B6010F94AD
:10D1A000532C87FF04C0C701B601905802C0C701C5
:10D1B000B60120E030E040EA50E40F94532C1816FA
:10D1C0002CF4B801C1010E94E66746C020E030E0BF
:10D1D00040E050E4C501B4010F94532C18161CF420
:10D1E000C8010E948B6719821A821B821C82A801C7
:10D1F000485F5F4FB8016C5F7F4F9E012F5F3F4FCD
:10D20000C8010E949F662DEC3CEC4CEC5CE3C7012E
:10D21000B6010F9463239B01AC0160911C0B7091CC
:10D220001D0B80911E0B90911F0B0F94632369833C
:10D230007A838B839C838091751781110E94C2FB36
:10D24000A101485F5F4FB1016C5F7F4F9E012F5F6F
:10D250003F4FC1010E949F66A0960FB6F894DEBFB3
:10D260000FBECDBFDF91CF911F910F91FF90EF9037
:10D27000DF90CF90BF90AF909F908F907F906F90F6
:10D280005F904F903F902F9008958C3891051CF03F
:10D290002CE880E002C0282F892F2093EB08809390
:10D2A000EC080C94A8D680914D1390914E13892BC5
:10D2B00039F00E94F5B991E0811103C090E001C0FE
:10D2C00091E0892F0895CF93DF93C82FD62F0E9426
:10D2D0008DBA882321F0DF91CF910C9453698C2F64
:10D2E0000E9444BA811101C08D2FDF91CF91089522
:10D2F0002F923F924F925F926F927F928F929F9266
:10D30000AF92BF92CF92DF92EF92FF920F931F9353
:10D31000CF93DF93CDB7DEB7CB56D1090FB6F894D4
:10D32000DEBF0FBECDBF88EB9BE10F943B020E9496
:10D33000BD9281110C94F07384E50E948DBA88230C
:10D3400029F00E9409BA81110E9443CF80E090E049
:10D35000A0E8BFE380931C0B90931D0BA0931E0BC2
:10D36000B0931F0B8093611790936217A09363177C
:10D37000B09364178DEC9CECACE4BEE38093180B87
:10D380009093190BA0931A0BB0931B0B80E090E0C5
:10D39000A0E2B1E48093140B9093150BA093160BAD
:10D3A000B093170B8CE390E09093130B8093120BC8
:10D3B0008DEC90E09093110B8093100B10920F0B5B
:10D3C0004AE959E969E97EE38FE40E9441B129966F
:10D3D0006CAF7DAF8EAF9FAF299760E083E40E9472
:10D3E0006369A5968FAFA59760E08BE40E9463699F
:10D3F000A6968FAFA69782E40E948DBA8823C9F0C3
:10D400000E940DBA0F945F2B7093130B6093120B55
:10D410006115710571F0685271096536710548F042
:10D420006CE870E08AE89BE10F94000385E89BE1DB
:10D43000B0C18CE40E948DBA882301F10E940DBA1C
:10D440006B017C016093180B7093190B80931A0B7E
:10D4500090931B0B20E030E0A9010F94532C87FD23
:10D460000AC020E030E040E050E4C701B6010F946C
:10D47000FD2218161CF48DE59BE18BC181E50E940D
:10D4800044BA882351F180914D1390914E13892B0A
:10D4900009F10E940DBA6B017C01609361177093D2
:10D4A000621780936317909364172DEC3CEC4CE467
:10D4B0005DE30F94532C87FD0AC020E030E040E785
:10D4C00051E4C701B6010F94FD22181634F48CE222
:10D4D0009BE15FC181E09BE15CC183E50E948DBA65
:10D4E0008823C9F00E940DBA4B015C012DEC3CEC85
:10D4F0004CEC5DE30F94532C87FD0AC020E030E034
:10D5000040E050E4C501B4010F94FD22181654F414
:10D510008AED9AE13EC1ADEC8A2EACEC9A2EA92C94
:10D52000AEE3BA2E80E50E9444BA882371F180915F
:10D530004D1390914E13892B19F482EA9AE129C177
:10D5400080910F0B8F5F80930F0B0E940DBA6B01C0
:10D550007C016093140B7093150B8093160B9093C2
:10D56000170B20E030E0A9010F94532C87FD0AC06F
:10D5700020E030E048EC51E4C701B6010F94FD22F1
:10D5800018161CF48AE79AE104C186E40E948DBA59
:10D590008823C9F00E940DBA6B017C0120E030E0C5
:10D5A00040E85FE30F94532C87FD0AC020E030E091
:10D5B00040E850E4C701B6010F94FD2218164CF460
:10D5C00081E59AE1E6C0C12CD12CF0EEEF2EFFE30D
:10D5D000FF2EA7019601C701B6010F9463239B019B
:10D5E000AC0160E070E084E490E40F94ED2A2091B7
:10D5F0001C0B30911D0B40911E0B50911F0B0F9473
:10D6000063232B013C01A5019401C501B4010F94D2
:10D610006323A70196010F9463232CEE31E548EBB9
:10D620005DE30F94ED2A9B01AC01C301B2010F949D
:10D63000632360931C0B70931D0B80931E0B9093C0
:10D640001F0B88E40E948DBA882381F00E940DBAD6
:10D650000F945F2B7093110B6093100B655A710937
:10D660006838710518F083E29AE193C085E50E945D
:10D6700044BA8823F1F00E94A4FD6115710581056B
:10D68000910511F00F948E1E80914D1390914E13C1
:10D69000892B19F00E940DBA04C060E070E088E4A4
:10D6A00092E460930B0B70930C0B80930D0B909393
:10D6B0000E0B82E50E9444BA811103C08FEE99E1FE
:10D6C00068C080914D1390914E13892B61F00E9498
:10D6D00009BA6B969FAF8EAF6B97181619064CF070
:10D6E0008BEB99E156C02AE130E06B963FAF2EAF4D
:10D6F0006B9789E50E948DBA882379F00E940DBA54
:10D7000020917A1730917B1740917C1750917D17AB
:10D710000F94F2296B017C0108C0C0900A18D090C8
:10D720000B18E0900C18F0900D1888E50E948DBA47
:10D73000882369F00E940DBA2091761730917717EF
:10D7400040917817509179170F94F22908C0609191
:10D750000618709107188091081890910918609325
:10D76000030B7093040B8093050B9093060BC092F0
:10D77000070BD092080BE092090BF0920A0BB7014D
:10D78000A60183E09BE00F945C13811106C081E940
:10D7900099E10F943B020C94F07384E40E9444BA24
:10D7A00091E089270E9435C020E030E040EA50E453
:10D7B00060910E1870910F188091101890911118A7
:10D7C0000F94FD2287FF1CC0198A1A8A1B8A1C8AA3
:10D7D00080E090E0A0EAB0E489839A83AB83BC83C5
:10D7E000BE016F5E7F4FCE0101960E94D3E280E1C1
:10D7F000E5E6F7E1A6E0B8E101900D928A95E1F740
:10D8000030913213A7963FAFA797109232130E9420
:10D810009FDA80E799E10F943B028091120B90917F
:10D82000130B8A3191056CF48091100B9091110BC0
:10D830000E9451D761E080E00E944DD1811109C062
:10D840000DC50E94456981E00E94CFCF8111ECCFC8
:10D8500005C51092121810921318109214181092F5
:10D86000151882E198E10E94168280910F0B88239F
:10D8700009F455C020E030E040E751E46091A61182
:10D880007091A7118091A8119091A9110F94ED2A80
:10D8900069837A838B839C8380E1E6E0F8E1A5E6E7
:10D8A000B7E101900D928A95E1F72091140B309128
:10D8B000150B4091160B5091170B609171177091D9
:10D8C000721780917317909174170F94F3296093D6
:10D8D0007117709372178093731790937417CE011A
:10D8E00001960E946EE12091140B3091150B40912E
:10D8F000160B5091170B60917117709172178091F0
:10D900007317909174170F94F229609371177093A5
:10D91000721780937317909374170E9496FB85E09B
:10D92000EEEFFAE0DF01282F1D922A95E9F7E9EFE3
:10D93000FAE0DF01282F1D922A95E9F7E4EFFAE0DB
:10D94000DF011D928A95E9F780E1E6E0F8E1A5E6BE
:10D95000B7E101900D928A95E1F78091180B9091B3
:10D96000190BA0911A0BB0911B0B80936D1790931C
:10D970006E17A0936F17B093701719821A821B82CB
:10D980001C829E012F5F3F4F4DE657E169E677E12C
:10D9900085E697E10E949F669E012B5B3F4F4DE617
:10D9A00057E169E677E185E697E10E949F66A596D3
:10D9B000BFADA597BB23B9F0209106183091071889
:10D9C00040910818509109182E962CAF3DAF4EAFDC
:10D9D0005FAF2E9780910A1890910B18A0910C18A8
:10D9E000B0910D1816C02091030B3091040B40919B
:10D9F000050B5091060B2E962CAF3DAF4EAF5FAF8F
:10DA00002E978091070B9091080BA091090BB09174
:10DA10000A0B69968CAF9DAFAEAFBFAF6997212C53
:10DA2000312C9FEF2A969FAF2A97AFEF6596AFAF45
:10DA30006597BFEF6C96BFAF6C97EFE4A096EFAF22
:10DA4000A097F3ECA296FFAFA29727E4A3962FAF7F
:10DA5000A39781E090E0A0E0B0E0022C04C0880F22
:10DA6000991FAA1FBB1F0A94D2F7AB968CAF9DAF2C
:10DA7000AEAFBFAFAB97AEEFBAE06496BFAFAEAF9D
:10DA8000649700E010E0AC962FAEAC976496EEADD4
:10DA9000FFAD649781916496FFAFEEAF649790E01D
:10DAA000A0E0B0E0AB962CAD3DAD4EAD5FADAB9719
:10DAB00082239323A423B523892B8A2B8B2B09F054
:10DAC00004C18091811290918212289EB001299EFA
:10DAD000700D389E700D11248091D0119091D1114C
:10DAE000680F791F072E000C880B990B0F940423E5
:10DAF00062966CAF7DAF8EAF9FAF629780918312BD
:10DB000090918412089FB001099F700D189F700DAD
:10DB100011248091D2119091D311680F791F072E93
:10DB2000000C880B990B0F9404236B017C01629607
:10DB30002CAD3DAD4EAD5FAD62972E966CAD7DAD1B
:10DB40008EAD9FAD2E970F94F2292B013C01A701BA
:10DB5000960169966CAD7DAD8EAD9FAD69970F94C2
:10DB6000F2294B015C01A3019201C301B2010F94A0
:10DB700063232B013C01A5019401C501B4010F945D
:10DB800063239B01AC01C301B2010F94F3290F94ED
:10DB9000A12C4B015C0162962CAD3DAD4EAD5FAD4D
:10DBA00062976091030B7091040B8091050B90912B
:10DBB000060B0F94F2292B013C01A70196016091FD
:10DBC000070B7091080B8091090B90910A0B0F9431
:10DBD000F2296B017C01A3019201C301B2010F94F0
:10DBE00063232B013C01A7019601C701B6010F94E5
:10DBF00063239B01AC01C301B2010F94F3290F947D
:10DC0000A12C20E030E040E751E40F94ED2AA5017B
:10DC100094010F94F3296B017C0180900B0B909081
:10DC20000C0BA0900D0BB0900E0B20E030E040E804
:10DC30005FE3C501B4010F94532C1816FCF4C50121
:10DC4000B4010F945F2B4B015C01161617061806E2
:10DC500019063CF40F94401EA50194010F947529F8
:10DC600003C060E070E0CB010F9404239B01AC0182
:10DC7000B601C7010F94F3296B017C016C962FAD9F
:10DC80006C97A0963FADA097A2964FADA297A39692
:10DC90005FADA397B601C7010F94FD2287FF15C0A2
:10DCA0002A960FAF2A97AC963FADAC9765963FAFDB
:10DCB00065976C96CFAE6C97A096DFAEA097A296B4
:10DCC000EFAEA297A396FFAEA3970F5F1F4F05304D
:10DCD000110509F0DBCE4FEF241A340A55E0251662
:10DCE000310409F0B6CE65968FAD6597E82FF0E068
:10DCF000E250F54F81E090E02A960FAC2A9702C0DF
:10DD0000880F991F0A94E2F79081892B808365968A
:10DD10009FAD65979F3F09F487C22A96AFAD2A97BA
:10DD2000AF3F09F481C22091811230918212659631
:10DD30004FAD65974203B001439F700D1124809150
:10DD4000D0119091D111680F791F072E000C880B0C
:10DD5000990B0F940423162F072F382E292E862F68
:10DD6000902FA32DB22D21968CAF9DAFAEAFBFAF3C
:10DD7000219720918312309184122A965FAD2A97C1
:10DD80005203B001539F700D11248091D2119091D4
:10DD9000D311680F791F072E000C880B990B0F9475
:10DDA00004236B017C0125966CAF7DAF8EAF9FAFD6
:10DDB0002597AB01BC01CE01CD960F945C1388234F
:10DDC00009F436C220E030E040EA50E4612F702FC1
:10DDD000832D922D0F94F3294B015C01FE01B9961E
:10DDE0008CE0DF011D928A95E9F7C401D50189A76E
:10DDF0009AA7ABA7BCA7CDA6DEA6EFA6F8AA659604
:10DE0000BFAD6597B111B1C22A96EFAD2A97E11166
:10DE10008DC220E030E040EA50E4C701B6010F9423
:10DE2000F3296B017C012A96FFAD2A97FF2309F4A1
:10DE300016C32A963FAD2A9734300CF010C3E2ED9A
:10DE40004E2EE3E55E2EEBE76E2EE1E47E2E89A4F6
:10DE50009AA4ABA4BCA42DA53EA54FA558A92E9667
:10DE60002CAF3DAF4EAF5FAF2E9725966CAD7DAD1D
:10DE70008EAD9FAD25970F94F22962966CAF7DAF62
:10DE80008EAF9FAF6297A501940121966CAD7DADD9
:10DE90008EAD9FAD21970F94F2296DAB7EAB8FAB0A
:10DEA00098AF62968CAD9DADAEADBFAD629789AFB8
:10DEB0009AAFABAFBCAFA501940160910618709109
:10DEC000071880910818909109180F94F2294B01B6
:10DED0005C012E962CAD3DAD4EAD5FAD2E976091A1
:10DEE0000A1870910B1880910C1890910D180F94CE
:10DEF000F2292E966CAF7DAF8EAF9FAF2E97812FFC
:10DF0000902FA32DB22D89839A83AB83BC83CD82BE
:10DF1000DE82EF82F886C090180BD090190BE0904B
:10DF20001A0BF0901B0BC986DA86EB86FC862DEC6B
:10DF30003CEC4CEC5CE3C301B2010F9463232091F1
:10DF40001C0B30911D0B40911E0B50911F0B0F9419
:10DF50006323209112183091131840911418509196
:10DF600015180F94F3296D877E878F87988BA501ED
:10DF70009401C501B4010F9463234B015C012E96FB
:10DF80002CAD3DAD4EAD5FAD2E97CA01B9010F94DA
:10DF900063239B01AC01C501B4010F94F32920E078
:10DFA00030E040E050E40F94532C181684F420E045
:10DFB00030E040E05FE3C701B6010F94F32969AB9D
:10DFC0007AAB8BAB9CABCE0189960E948B6780911C
:10DFD000180B9091190BA0911A0BB0911B0B89ABE8
:10DFE0009AABABABBCAB198A1A8A1B8A1C8A9E01FE
:10DFF0002F5E3F4FAE014F5C5F4FBE01635D7F4FB1
:10E00000CE0189960E949F668091751781110E94AA
:10E01000C2FB409061025090620260906302709077
:10E020006402E0909E11F0909F110091A011109158
:10E03000A111A0909A11B0909B11C0909C11D0900A
:10E040009D119501A601B701C8010F94532C181614
:10E0500014F4750186012DEC3CEC4CEC5DE3B7014A
:10E06000C8010F94632360936102709362028093EE
:10E0700063029093640240E0BE016B5C7F4FCE016F
:10E0800001960E945BEF40926102509262026092A0
:10E0900063027092640280E1E6E0F8E1A5E6B7E190
:10E0A00001900D928A95E1F78091180B9091190BD0
:10E0B000A0911A0BB0911B0B898F9A8FAB8FBC8FDD
:10E0C0008DA39EA3AFA3B8A7CC24C394D12CD60113
:10E0D00011976796BFAFAEAF6797812C912C540113
:10E0E000839466960FAC669704C0880C991CAA1C92
:10E0F000BB1C0A94D2F781E090E0A0E0B0E00C2CC9
:10E1000004C0880F991FAA1FBB1F0A94D2F79C0155
:10E11000AD01282939294A295B296F962CAF3DAFDB
:10E120004EAF5FAF6F9781E066960FAC669701C008
:10E13000880F0A94EAF7A2968FAFA29744EF5AE0AD
:10E1400064965FAF4EAF649789EF9AE02C969FAFCD
:10E150008EAF2C97AEEFBAE06096BFAFAEAF6097D0
:10E16000212C312CA1963FAE2EAEA1976096EEAD3C
:10E17000FFAD6097A496FFAFEEAFA497FFEF2F1A05
:10E180003F0A6096AEADBFAD60978C9190E0A0E085
:10E19000B0E06F962CAD3DAD4EAD5FAD6F97822375
:10E1A0009323A423B523281739074A075B0709F4EB
:10E1B0007AC16096EEADFFAD609731966096FFAF85
:10E1C000EEAF6097A496AEADBFADA4978C9190E0F2
:10E1D000A0E0B0E088219921AA21BB21892B8A2BBC
:10E1E0008B2B09F052C164962EAD3FAD64972F5F23
:10E1F0003F4F64963FAF2EAF64972C964EAD5FAD08
:10E200002C974F5F5F4F2C965FAF4EAF2C9755E02A
:10E210002516310409F0A6CF8FEFC81AD80A96E068
:10E22000C916D10409F053CF8091E1118093E21116
:10E230006B96AEADBFAD6B9711976B96BFAFAEAFA0
:10E240006B97AB2B59F06596BFAD6597BF3F31F02B
:10E250002A96EFAD2A97EF3F09F0A9CB6FEF85E83B
:10E2600099E10F9416060E9496FB80E090E0A0EAE8
:10E27000B0E480936D1790936E17A0936F17B093CF
:10E28000701719821A821B821C829E012F5F3F4FDA
:10E290004DE657E169E677E185E697E10E949F66E2
:10E2A0008091070B9091080BA091090BB0910A0B7C
:10E2B0004091030B5091040B6091050B7091060B7C
:10E2C00040936517509366176093671770936817AC
:10E2D0008093691790936A17A0936B17B0936C178C
:10E2E00019821A821B821C829E012F5F3F4F4DE6CE
:10E2F00057E169E677E185E697E10E949F66A79678
:10E30000FFADA797F09332130E949FDAA6962FAD28
:10E31000A697211165C21092EC081092EB080E949A
:10E32000A8D680E090E00E9451D75AC2812F902F4A
:10E33000A32DB22D89A79AA7ABA7BCA720E030E0F8
:10E3400040EA50E4C701B6010F94F2296DA77EA7F9
:10E350008FA798AB2A962FAD2A9724300CF459CD6D
:10E36000182D092D3A2C2B2C7AC065964FAD659748
:10E3700044300CF44CC02A965FAD2A9754307CF0A0
:10E3800020E030E040EA50E4612F702F832D922D81
:10E390000F94F22969A77AA78BA79CA728C0812F81
:10E3A000902FA32DB22D89A79AA7ABA7BCA720E0D9
:10E3B00030E040EA50E4C701B6010F94F3296DA79D
:10E3C0007EA78FA798AB2A968FAD2A9781110FC091
:10E3D00020E030E040EA50E4612F702F832D922D31
:10E3E0000F94F229162F072F382E292E38C020E03F
:10E3F00030E040EA50E4C701B6010F94F2296B0106
:10E400007C012A969FAD2A9794304CF518CD2A9618
:10E41000AFAD2A97A1110DC020E030E040E251E4F9
:10E42000B401C5010F94F229162F072F382E292E7B
:10E4300006CD2A96BFAD2A97B430D4F020E030E064
:10E4400040E251E4B401C5010F94F22969A77AA70B
:10E450008BA79CA7182D092D3A2C2B2CF0CC72EDF4
:10E46000472E73E5572E7BEF672E70E4772EEFCCA7
:10E47000182D092D3A2C2B2C62ED462E63E5562ED5
:10E480006BEF662E61E4762EE2CC808190E0A0E016
:10E49000B0E088219921AA21BB21892B8A2B8B2BC3
:10E4A00009F0D0C0A0CE2C96AEADBFAD2C978C910C
:10E4B00090E0A0E0B0E088219921AA21BB21892B1E
:10E4C0008A2B8B2B09F075CE0091D0111091D111B0
:10E4D000E0908112F090821267964EAD5FAD679723
:10E4E000E49EB001E59E700DF49E700D1124600F46
:10E4F000711F072E000C880B990B0F94042320E04A
:10E5000030E040E050E40F94F3296D8F7E8F8F8FC1
:10E5100098A3CE9CB001CF9C700DDE9C700D112491
:10E52000600F711F072E000C880B990B0F940423AA
:10E5300020E030E040E050E40F94F229698B7A8BC0
:10E540008B8B9C8B4AED51E061E070E0CE014D96E3
:10E550000F94410B8091831290918412A196AEADDD
:10E56000BFADA197A89FB001A99F700DB89F700D76
:10E5700011248091D2119091D311680F791F072E29
:10E58000000C880B990B0F9404232B013C0120E015
:10E5900030E040E85FE30F94FD2287FD12C020E0E9
:10E5A00030E840EE53E4C301B2010F94532C181627
:10E5B00074F4412C30E8532E30EE632E33E4732E86
:10E5C00006C0412C512C20E8622E2FE3722E4D8A7A
:10E5D0005E8A6F8A788E49A25AA26BA27CA24AED0B
:10E5E00051E061E070E0CE0141960F94410B49A1EA
:10E5F0005AA16BA17CA1CE014D960F945C13882388
:10E6000051F04D895E896F89788DCE0141960F94C6
:10E610005C1381110FC02C96EEADFFAD2C9780815D
:10E62000A296FFADA2978F2B2C96AEADBFAD2C97C7
:10E630008C93BFCDBE016F5E7F4FCE014D960E9481
:10E64000E667E9CF6496EEADFFAD6497808190E018
:10E65000A0E0B0E088219921AA21BB21892B8A2B37
:10E660008B2B09F0C0CD0091D2111091D311E09005
:10E670008312F0908412A196EEADFFADA197EE9DAE
:10E68000B001EF9D700DFE9D700D1124600F711F84
:10E69000072E000C880B990B0F94042320E030E028
:10E6A00040E050E40F94F32969A37AA38BA39CA3C1
:10E6B0002E9CB0012F9C700D3E9C700D1124600F9C
:10E6C000711F072E000C880B990B0F94042320E078
:10E6D00030E040E050E40F94F2296D8B7E8B8F8BFD
:10E6E000988F809181129091821267962EAD3FADE6
:10E6F0006797289FB001299F700D389F700D1124D6
:10E700008091D0119091D111680F791F072E000CC4
:10E71000880B990B0F9404232B013C0120E030E07F
:10E7200040E85FE30F94FD2287FD11C020E030E058
:10E730004DEE53E4C301B2010F94532C18166CF440
:10E74000412C512C9DEE692E93E4792E06C0412C6C
:10E75000512C80E8682E8FE3782E498A5A8A6B8A7A
:10E760007C8A4D8E5E8E6F8E78A241EC51E061E026
:10E7700070E0CE0181960F94410B41EC51E061E0D5
:10E7800070E0CE0145960F94410B49A15AA16BA1AF
:10E790007CA1CE014D960F945C13882351F04D89D6
:10E7A0005E896F89788DCE0141960F945C1381113B
:10E7B0000FC06496AEADBFAD64978C91A296BFAD0D
:10E7C000A2978B2B6496EEADFFAD649780830BCD43
:10E7D000BE016F5E7F4FCE014D960E94E667E9CF86
:10E7E000C559DF4F0FB6F894DEBF0FBECDBFDF9126
:10E7F000CF911F910F91FF90EF90DF90CF90BF903E
:10E80000AF909F908F907F906F905F904F903F90D0
:10E810002F900895CF92DF92EF92FF920F931F9364
:10E82000CF93DF936C017A018B01C0E0D0E0CE156D
:10E83000DF0581F0D8016D918D01D601ED91FC913C
:10E840000190F081E02DC6011995892B11F02196D8
:10E85000EECF7E01C701DF91CF911F910F91FF9005
:10E86000EF90DF90CF900895089580E090E00895B4
:10E87000FC01538D448D252F30E0842F90E0821BC6
:10E88000930B541710F0CF96089501970895FC014B
:10E89000918D828D981761F0828DDF01A80FB11DD7
:10E8A0005D968C91928D9F5F9F73928F90E00895FB
:10E8B0008FEF9FEF0895FC01918D828D981731F0B5
:10E8C000828DE80FF11D858D90E008958FEF9FEF09
:10E8D0000895FC01918D228D892F90E0805C9F4FDF
:10E8E000821B91098F73992708958AE793E10E940B
:10E8F000697421E0892B09F420E0822F0895FC013E
:10E90000848DDF01A80FB11DA35ABF4F2C91848DB8
:10E9100090E001968F739927848FA689B7892C93ED
:10E92000A089B1898C91837080648C93938D848D40
:10E93000981306C00288F389E02D80818F7D808343
:10E940000895EF92FF920F931F93CF93DF93EC0103
:10E9500081E0888F9B8D8C8D981305C0E889F9899B
:10E96000808185FD26C0F62E0B8D10E00F5F1F4FB6
:10E970000F731127E02E8C8DE8120CC00FB607FC28
:10E98000FACFE889F989808185FFF5CFCE010E9411
:10E990007F74F1CF8B8DFE01E80FF11DE35AFF4F1D
:10E9A000F0829FB7F8940B8FEA89FB89808180629F
:10E9B0000AC09FB7F894EE89FF896083E889F989D6
:10E9C00080818370806480839FBF81E090E0DF91CD
:10E9D000CF911F910F91FF90EF900895CF93DF9308
:10E9E000EC01888D8823C9F0EA89FB89808185FD47
:10E9F00005C0A889B9898C9186FD0FC00FB607FCA8
:10EA0000F5CF808185FFF2CFA889B9898C9185FFE8
:10EA1000EDCFCE010E947F74E7CFDF91CF910895B3
:10EA200080E090E0892B41F080E090E0892B21F09C
:10EA30000E940000811121C080E090E0892B41F00C
:10EA400080E090E0892B21F00E940000811118C025
:10EA500080E090E0892B21F00E947574811113C031
:10EA600080E090E0892BA1F080E090E0892B81F09C
:10EA70000E94000081110AC008950E940000DCCFAE
:10EA80000E940000E5CF0E940000EACF0C94000035
:10EA900008950F94052DCF93DF93EC01CB01E8810E
:10EAA000F981608171810E94159488819981DC01CE
:10EAB000ED91FC912081AA81BB81222369F02C91E8
:10EAC000293650F43196DC01ED93FC93EA81FB8109
:10EAD00080818F5F8083E9CF8C91893670F48FE2DB
:10EAE0008083E881F981808191810196918380837F
:10EAF000EA81FB8180818F5F8083DF91CF910895D0
:10EB00001F920F920FB60F9211240BB60F922F93F4
:10EB10003F934F935F936F937F938F939F93AF93A5
:10EB2000BF93EF93FF938AE793E10E947F74FF9175
:10EB3000EF91BF91AF919F918F917F916F915F9175
:10EB40004F913F912F910F900BBE0F900FBE0F90E2
:10EB50001F9018951F920F920FB60F9211240BB6AB
:10EB60000F922F938F939F93EF93FF93E0918A13CC
:10EB7000F0918B138081E0919013F091911382FDBD
:10EB800012C09081809193138F5F8F7320919413A3
:10EB9000821751F0E0919313F0E0E658FC4E958F08
:10EBA0008093931301C08081FF91EF919F918F918A
:10EBB0002F910F900BBE0F900FBE0F901F901895C6
:10EBC0008BE1E0E7F4E1A5E5B4E101900D928A95CF
:10EBD000E1F780911817806280931817089580914B
:10EBE000181782FF1FC084E29DE10F943B026091E1
:10EBF00014177091151780911617909117174AE006
:10EC00000E94E1538FE20E94DA53609110177091D5
:10EC1000111780911217909113174AE00E94E15347
:10EC20000C94DF5486E39DE10D943B021092200B7F
:10EC3000809118178F7B8B7F809318170E947F51CC
:10EC4000882321F087E194E10C947B9608958091CC
:10EC5000181783FF03C08460809318170895CF921C
:10EC6000DF92EF92FF920F931F93CF93DF93CDB775
:10EC7000DEB7EDB6FEB6DC010D900020E9F79D0190
:10EC8000281B390B2C5F3F4F4DB75EB7421B530B10
:10EC90000FB6F8945EBF0FBE4DBF0DB71EB70F5F26
:10ECA0001F4F9F938F9380E29CE19F938F931F93BD
:10ECB0000F930F949522680154E0C50ED11C0F905C
:10ECC0000F900F900F900F900F90F6018081882386
:10ECD00049F0082E000C990B0F940A2DF601819330
:10ECE0006F01F3CFC8010E94D7EB8CE19CE10E9439
:10ECF00038B90FB6F894FEBE0FBEEDBEDF91CF91CE
:10ED00001F910F91FF90EF90DF90CF9008958F9219
:10ED10009F92AF92BF92CF92DF92EF92FF92CF93EA
:10ED200080911817877F8093181780917314882318
:10ED300021F080E794E10E947B9610925414109287
:10ED4000511485E3809350140E94A4FD6B017C0153
:10ED500020EDC20E27E0D21EE11CF11CA89561E057
:10ED6000809150140E9417FC61E0809150140E9421
:10ED700046FC209A289A219A2398229A81E00E94A0
:10ED8000D25C85E0809352140E94D25CCAE08FEF7F
:10ED90000E94C65CC150D9F7A89520E030E0A901D7
:10EDA00060E080E594E10E945B958093531481308C
:10EDB00061F00E94A4FDDC01CB018C199D09AE0914
:10EDC000BF09B7FDEACF81E062C0A8952AEA31E029
:10EDD00040E050E068E080E594E10E945B9585307A
:10EDE00011F481E00AC0C4E00E94CB5C809353140C
:10EDF000C150D1F78A3A61F482E080935414A89507
:10EE000080915414823081F0812C912C540111C0D6
:10EE10000E94A4FDDC01CB018C199D09AE09BF093C
:10EE2000B7FDD4CF82E033C0812C912CA12C80E49B
:10EE3000B82E20E030E0A90167E380E594E10E946C
:10EE40005B95A501940169E280E594E10E945B95E0
:10EE500080935314882361F00E94A4FDDC01CB0150
:10EE60008C199D09AE09BF09B7FDE3CF8AE00FC039
:10EE700080915414823021F520E030E0A9016AE34A
:10EE800080E594E10E945B95882361F088E080939F
:10EE9000511480E594E10E9453950F9424038EE071
:10EEA0009CE122C00E94CB5C807C803C19F483E012
:10EEB000809354140E94CB5C0E94CB5C0E94CB5C7C
:10EEC00080E594E10E9453951092521481E00F94D2
:10EED000580981110CC080E00F945809811107C0B6
:10EEE0000F9420038AEF9BE10F943B021AC062E368
:10EEF00074E180E794E10E94A693811105C00F940C
:10EF0000200389EE9BE1F0CF8091181788608093F1
:10EF100018170F9424038DED9BE10F943B020E9480
:10EF20007351CF91FF90EF90DF90CF90BF90AF9053
:10EF30009F908F900C94E075FC0180818823E1F014
:10EF4000853ED1F08E32C1F080912E1A8E32A1F022
:10EF50009385892F8A7081F4987121E0903109F0AE
:10EF600020E08091181720FB84F9809318179031C6
:10EF700041F08085873411F080E0089581858E37D7
:10EF8000D9F381E008950F931F93CF93DF93CDB70B
:10EF9000DEB7EB970FB6F894DEBF0FBECDBF85E5A9
:10EFA00094E10E944E958BE1E5E5F4E1DE01919656
:10EFB00001900D928A95E1F700E010E04EE25AE1EF
:10EFC000BE016F5F7F4FCE0181960E941098181688
:10EFD0003CF4CE0101960E949C77080F111DEECFE4
:10EFE000CE0181960E948496C801EB960FB6F894E4
:10EFF000DEBF0FBECDBFDF91CF911F910F9108955E
:10F00000FC0120E03EE2DB014C91403241F028302F
:10F0100011F430833196DB014C91408331962F5FA0
:10F020006F5F7F4F2B3079F7108208956F927F9238
:10F030008F929F92AF92BF92CF92DF92EF92FF9208
:10F040000F931F93CF93DF93CDB7DEB7C356D1098C
:10F050000FB6F894DEBF0FBECDBF5C018B016DB65D
:10F060007EB67E0187E5E80EF11C4EE25AE1BE0154
:10F070006F5F7F4FC5010E94109818160CF0AFC04B
:10F080008C858871803109F06CC08DB69EB6BE014A
:10F090006F5F7F4FC7010E9400780115110521F0B5
:10F0A000F8018081811191C021E081E090E0F701B9
:10F0B00001900020E9F73197EE19FF09E80FF91FD9
:10F0C00032968DB79EB78E1B9F0B0FB6F8949EBFDE
:10F0D0000FBE8DBFEDB7FEB731966F01211102C093
:10F0E000B80102C06BE776E0C6010F94512DB7015D
:10F0F000C6010F943B2D6BE776E0C6010F943B2DC4
:10F1000019A21CA221E0A701B501CE0181960E949F
:10F110007E9A81110AC00F942403B70189EC9BE108
:10F120000F940D038AE00E94DA538BE1FE01B19641
:10F13000DE01DC9601900D928A95E1F7B601CE01D1
:10F14000CC960E941678CE01CC960E948496CE0171
:10F1500081960E9484960FB6F8949EBE0FBE8DBE17
:10F1600084CFCE0101960E949C77882309F47DCF3D
:10F17000BE016F5F7F4F80E79AE10E940078011522
:10F18000110529F480E7C82E8AE1D82E09C068014C
:10F19000F60181916F018823A9F30E94DA53F8CF19
:10F1A000F60181916F01882319F00E94DA53F8CF9C
:10F1B00080E20E94DA536D8D7E8D8F8D98A14AE09A
:10F1C0000E94E1530E94DF5450CFF80101900020CB
:10F1D000E9F73197CF01801B910B20E068CF0FB684
:10F1E000F8947EBE0FBE6DBECD59DF4F0FB6F894BA
:10F1F000DEBF0FBECDBFDF91CF911F910F91FF906A
:10F20000EF90DF90CF90BF90AF909F908F907F90C6
:10F210006F900895EF92FF920F931F93CF93DF9318
:10F22000CDB7DEB7A0970FB6F894DEBF0FBECDBF47
:10F230007C018B014EE25AE1BE016F5F7F4FC70137
:10F240000E9410981816A4F4CE0101960E949C7793
:10F25000882381F3BE016F5F7F4F80E79AE10E94B0
:10F26000007860E77AE1C8010F94282D892B11F707
:10F27000A0960FB6F894DEBF0FBECDBFDF91CF9141
:10F280001F910F91FF90EF9008950F931F93CF93CD
:10F29000DF93CDB7DEB76B970FB6F894DEBF0FBE26
:10F2A000CDBF8C0185E594E10E944E958BE1E5E5AB
:10F2B000F4E1DE01119601900D928A95E1F7B80113
:10F2C000CE0101960E940A79CE0101960E94849691
:10F2D0006B960FB6F894DEBF0FBECDBFDF91CF9116
:10F2E0001F910F910895DF92EF92FF920F931F935A
:10F2F000CF93DF93CDB7DEB727970FB6F894DEBF75
:10F300000FBECDBF2091181723FF37C1F42EE62E74
:10F310008C010E947F51882309F480C0FF2009F4EA
:10F320008BC080910F17882351F00F9420038FED2D
:10F330009CE10F943B0280E090E00E943EF686E262
:10F340009BE09E838D838FE28093250B81E08F83EA
:10F35000CE0105969A83898302969C838B83F12C38
:10F360009BE1D92E80910E17F81658F4DF9CB0015E
:10F37000112460507A4ECE0101960E944B75F39491
:10F38000F1CF8F818B3558F467E174E1CE0101969E
:10F390000E944B758D819E8101979E838D83ED81A7
:10F3A000FE811082E0910F1784E0E89FF0011124A4
:10F3B000EF5DF44F8091141790911517A0911617D7
:10F3C000B091171780839183A283B3830F94240392
:10F3D000B80186EC9CE10F940D0360910F1789E64C
:10F3E000689FB00111246B5D744F8BEB9CE10F940F
:10F3F0000D034091141750911517609116177091D5
:10F40000171785EB9CE10F94D1028AE00E94DA5332
:10F4100080910F178F5F80930F1726C0FF2039F060
:10F420000F94240385EA9CE10F943B021DC01092C7
:10F430000F1782E0F82E02C0FF24F3940F942403E8
:10F4400080EA9CE10F943B0281E0F81609F492C037
:10F450008CE89CE10F943B02B80188E99CE10F9491
:10F460000D038AE00E94DA530E941676B801CE019D
:10F4700001960E94A5F78C01009709F47EC069816E
:10F480007A81EE2009F44DC021E0AC0187E194E1DE
:10F490000E947E9A8823E9F1809128149091291482
:10F4A000A0912A14B0912B148093101790931117E8
:10F4B000A0931217B09313171092141710921517E8
:10F4C0001092161710921717B8018EE79CE10F944F
:10F4D0000D03409110175091111760911217709100
:10F4E000131786E79CE10F94D1028AE00E94DA5359
:10F4F00087E69CE10F943B02C8010E944579809108
:10F500002E1A811102C0C80102C08EE29AE160E0A9
:10F510002EC0B80183E59CE10F940D0380E59CE1CA
:10F520000FC026E5AC0187E194E10E947E9A81112B
:10F530000AC0B8018CE39CE10F940D0389E39CE1C0
:10F540000F943B021AC0809118178160809318179E
:10F55000C8010E9445791092FE15B80187E29CE12E
:10F560000F940D038AE00E94DA5360E0C8010F9403
:10F57000710603C082E99CE16DCF27960FB6F8941F
:10F58000DEBF0FBECDBFDF91CF911F910F91FF90D6
:10F59000EF90DF900895CF92DF92EF92FF92CF939A
:10F5A0006B017C01C42F8091231A9091241AA091A1
:10F5B000251AB091261A8C159D05AE05BF05D1F010
:10F5C0000E940896811102C080E018C023E238E151
:10F5D000B701A60180912C1A90912D1A0E948A964B
:10F5E000882391F3C092231AD092241AE092251A0C
:10F5F000F092261A81E0C11180932B1ACF91FF90CF
:10F60000EF90DF90CF9008954F925F926F927F922C
:10F610008F929F92AF92BF92CF92DF92EF92FF9222
:10F620000F931F93CF93DF93EC0142305105610597
:10F63000710510F480E069C089859A85AB85BC8529
:10F640000196A11DB11D84179507A607B70790F372
:10F650008F89803149F4852E962EA72EBB248B8965
:10F660009C89AD89BE890FC0803221F78B889C8828
:10F67000AD88BE88DB01CA01E7E0B695A7959795EE
:10F680008795EA95D1F7880E991EAA1EBB1E280100
:10F6900039016A017B0141E0C501B4010E94CB7AC6
:10F6A000882341F29F89903161F4DD24EE24FF2408
:10F6B0009601220F331FF901ED5DF74E5182408212
:10F6C00011C0E894C7F8DD24EE24FF249601220F30
:10F6D000331F220F331FF901ED5DF74E4082518237
:10F6E000628273829A89923080F04D815E816F814F
:10F6F0007885840E951EA61EB71E8092271A9092BA
:10F70000281AA092291AB0922A1ADF91CF911F913C
:10F710000F91FF90EF90DF90CF90BF90AF909F90B0
:10F720008F907F906F905F904F900895CF92DF926F
:10F73000EF92FF920F931F93CF93DF93FC0181858C
:10F740009285A385B4850196A11DB11D84179507E7
:10F75000A607B70710F480E061C08789803149F4BB
:10F76000BB27A72F962F852FC388D488E588F688D6
:10F770000FC0803281F783899489A589B6896A018F
:10F780007B01C7E0F694E794D794C794CA95D1F764
:10F790008C0D9D1DAE1DBF1DE9016A017B018F010E
:10F7A0004091231A5091241A6091251A7091261ABB
:10F7B00084179507A607B70739F040E0BC01CD01D3
:10F7C0000E94CB7A882339F2F8018789803179F455
:10F7D000B701A601552766277727440F551FFA0161
:10F7E000ED5DF74E80819181A0E0B0E012C0B701DD
:10F7F000A6014F77552766277727440F551F440FDB
:10F80000551FFA01ED5DF74E80819181A281B38190
:10F81000BF7088839983AA83BB8381E0DF91CF91F6
:10F820001F910F91FF90EF90DF90CF9008954F922E
:10F830005F926F927F92AF92BF92CF92DF92EF92E0
:10F84000FF920F931F93CF93DF9300D01F92CDB7FA
:10F85000DEB78C0149835A836B837C835901C12CA9
:10F86000D12C7601412C82E0582E612C712C4981DB
:10F870005A816B817C819E012F5F3F4FC8010E949E
:10F88000967B882341F1D301C201F801058404C0AD
:10F89000880F991FAA1FBB1F0A94D2F7C80ED91E42
:10F8A000EA1EFB1E49815A816B817C8187898031E8
:10F8B00039F481E0483F5F4F6105710538F4D7CFD7
:10F8C00081E0483F5F4F6F4F7F4088F2F501C08273
:10F8D000D182E282F3820F900F900F900F90DF9110
:10F8E000CF911F910F91FF90EF90DF90CF90BF903D
:10F8F000AF907F906F905F904F900895CF93DF937C
:10F900008091FE149091FF14891B8F708F3021F429
:10F9100080E00E940655F4CF8091FE148F5F8F70B7
:10F92000A091FE1498E59A9FD0011124FD01ED509D
:10F93000F44FEF0119929A95E9F798E09083A85F48
:10F94000B34F90E1E4E1F5E101900D929A95E1F772
:10F950002091FE149091FF14291303C094E6909314
:10F96000FB148093FE1480916F00826080936F007F
:10F97000DF91CF9108950F930FB70F9300916E0011
:10F980000F930B7F00936E0000916F000D7F00932B
:10F990006F000F930BB70F930CB70F921F922F931B
:10F9A0003F934F935F936F937F938F939F93AF9307
:10F9B000BF93EF93FF9311240E94E35CFF91EF91BB
:10F9C000BF91AF919F918F917F916F915F914F9177
:10F9D0003F912F911F900F900CBF0F910BBF0F9174
:10F9E0000260F89400936F000F9100936E000F91E6
:10F9F0000FBF0F911895EF92FF920F931F93E09214
:10FA0000A50BF092A60B0093A70B1093A80B609385
:10FA1000AD0A7093AE0A8093AF0A9FEFFF27621B77
:10FA2000730B840B30F4809570956195790B890B7D
:10FA3000992790934F08A6E06A9F00924308512DA2
:10FA4000EE277A9F500DE11D8A9FE00D50934408E8
:10FA5000E0934508AFE06A9F00924708512DEE27DA
:10FA60007A9F500DE11D8A9FE00D50934808E09366
:10FA70004908AAE06A9F00924B08512DEE277A9F11
:10FA8000500DE11D8A9FE00D50934C08E0934D0806
:10FA90001F910F91FF90EF9008950000000000006B
:10FAA0008091100980FF03C089988FEF02C0899A66
:10FAB00081E08093A50A80911009869580FF03C09C
:10FAC0008F9A8FEF02C08F9881E08093A60A809171
:10FAD00010098695869580FF08C080910B0180955E
:10FAE0008270809309018FEF06C080910B018270B4
:10FAF0008093090181E08093A70A8091100986957F
:10FB00008695869580FF03C016988FEF02C0169ADF
:10FB100081E08093A80A0000000000000895809111
:10FB2000FE149091FF14891B8F7019F480E090E00F
:10FB300008959091FB14992351F0833030F48FEFA6
:10FB4000890F19F08093FB14F1CF1092FB14E09110
:10FB5000FF1488E5E89FF0011124ED50F44F8081F7
:10FB600080FDE4CF8091FF148F5F8F708093FC1431
:10FB70009091FF148091FD14981304C08091FC149F
:10FB80008093FD14CF0108951F93CF93DF93CDB7DA
:10FB9000DEB728970FB6F894DEBF0FBECDBF6983DE
:10FBA0007A838B839C832D833E834F83588781E0A8
:10FBB0000E949F9269E170E080E090E00F940C0257
:10FBC000BE016B5F7F4FCE0101960E94D3E2109180
:10FBD000A30A80E00E949F921092A30A82E00E94F2
:10FBE00018E30E9486E312FB112710F981E08127B8
:10FBF00028960FB6F894DEBF0FBECDBFDF91CF9130
:10FC00001F910895CF92DF92EF92FF92CF93DF93EF
:10FC1000CDB7DEB728970FB6F894DEBF0FBECDBFC5
:10FC200020E030E040EA50E460910E1870910F1827
:10FC300080911018909111180F94FD228823E9F0FB
:10FC40001D821E821F821886C12CD12C80EAE82ECC
:10FC500080E4F82EC982DA82EB82FC82BE016B5FFF
:10FC60007F4FCE0101960E94D3E2C0920E18D0922F
:10FC70000F18E0921018F092111828960FB6F89409
:10FC8000DEBF0FBECDBFDF91CF91FF90EF90DF9031
:10FC9000CF9008953F924F925F926F927F928F9292
:10FCA0009F92AF92BF92CF92DF92EF92FF920F930B
:10FCB0001F93CF93DF93CDB7DEB728970FB6F89495
:10FCC000DEBF0FBECDBF90911109981709F485C012
:10FCD000382E80E090E0A0E2B1E48D839E83AF8374
:10FCE000B887C0908A17D0908B17E0908C17F0904F
:10FCF0008D1720E030E0A901C701B6010F94FD2265
:10FD000087FF0CC0A701960160E070E080E291E4FB
:10FD10000F94F2296D837E838F83988720E030E0F3
:10FD20004BEE53E46D817E818F8198850F94532C27
:10FD3000181644F480E090E0ABEEB3E48D839E832C
:10FD4000AF83B8872D813E814F81588560910E1811
:10FD500070910F1880911018909111180F94FD2236
:10FD600087FF0BC019821A821B821C82BE016F5F43
:10FD70007F4FCE0105960E94D3E240900618509026
:10FD80000718609008187090091880900A189090D1
:10FD90000B18A0900C18B0900D18332019F00E9489
:10FDA0004EBF02C00E94FFBE19821A821B821C82B3
:10FDB000E0900E18F0900F18009110181091111883
:10FDC000CE0101966C01A5019401C301B2010E940C
:10FDD000F0E1309211090E94A0C180E028960FB690
:10FDE000F894DEBF0FBECDBFDF91CF911F910F9171
:10FDF000FF90EF90DF90CF90BF90AF909F908F904B
:10FE00007F906F905F904F903F900895CF93DF93D6
:10FE1000C091A00B8DE796E00E94E55480919B0B6A
:10FE2000873009F445C083E080939A0B81E080938A
:10FE3000260280E190E090939D1580939C1585E0CB
:10FE400080939015D2E8D093931584E190E1A0E0DF
:10FE5000B0E08093941590939515A0939615B09368
:10FE600097150E942FF561E070E080E090E00E941D
:10FE7000F8AF81E09AE590939D1580939C1585E3FA
:10FE800090E090939F1580939E1587E08093901546
:10FE9000D093931584E890E0A0E0B0E080939415AF
:10FEA00090939515A0939615B09397150E942FF5F2
:10FEB000C13081F1C23059F40F9411046093920B58
:10FEC0007093930B8093940B9093950B02C00F94B7
:10FED000450481E08093A00B0E94A4FD60938E0BEB
:10FEE00070938F0B8093900B9093910BC230A1F085
:10FEF0008091FE089091FF0801969093FF088093EF
:10FF0000FE081092A10B1092A20B1092A30B10925C
:10FF1000A40B02C080E001C081E0DF91CF91089581
:10FF2000CF93DF9300D01F92CDB7DEB78091FD084D
:10FF30008823A9F083E390E09C838B831A82198243
:10FF40009E012F5F3F4F40E150E06EEF78E0CE0121
:10FF500003960E94DD5185E996E00E94E5540F90DA
:10FF60000F900F900F90DF91CF910895CF92DF9275
:10FF7000EF92FF920F931F938091A00B81508230DC
:10FF800010F080E09EC085EB96E00E94E5548091E1
:10FF90009B0B8330C9F140E060E070E0CB010F942F
:10FFA000C40641E060E070E0CB010F94C40681E03C
:10FFB000809301021092990B21E030E03093980B6E
:10FFC0002093970B8093260281E09AE590939D15EC
:10FFD00080939C158DE290E090939F1580939E15E1
:10FFE00087E08093901582E88093931584E890E0F1
:10FFF000A0E0B0E08093941590939515A09396158A
:020000021000EC
:10000000B09397150E942FF51092A00B0E94A4FDAB
:1000100060939C0B70939D0B80939E0B90939F0B12
:1000200080910009909101090196909301098093B4
:100030000009C090A10BD090A20BE090A30BF09010
:10004000A40B0F9411046093A10B7093A20B8093E7
:10005000A30B9093A40B0091020910910309209126
:100060000409309105090C191D092E093F09DC010D
:10007000CB01800F911FA21FB31F809302099093A1
:100080000309A0930409B09305090F94110400918A
:1000900006091091070920910809309109090617EE
:1000A00017072807390750F40F94110460930609C5
:1000B0007093070980930809909309090E94907F23
:1000C00081E01F910F91FF90EF90DF90CF90089506
:1000D000CF93DF9300D01F921F92CDB7DEB781E0A0
:1000E0008093FD08EEEFF8E080E1DF011D928A9534
:1000F000E9F70E94907F86E18D8382E390E09C8304
:100100008B831A8219829E012F5F3F4F41E050E09E
:10011000BE016B5F7F4FCE0103960E94DD510F90B1
:100120000F900F900F900F90DF91CF9108959F92B5
:10013000AF92BF92CF92DF92EF92FF920F931F93F5
:10014000CF93DF9300D01F921F92CDB7DEB7E7E4C5
:10015000FDE10027BB27462F572FA82FAA2341F4E4
:10016000A52F542FB85FAA2319F4A52F5527B85FE0
:10017000A03138F45295A295452F4F70507FA42B93
:10018000BC5FA03428F4550FAA1F550FAA1FBE5FED
:10019000A03818F4550FAA1FB395550FAA1FEA0FE0
:1001A000F01F449151E0AA27B85081F1C8F0B0FF88
:1001B00002C0440F551FB1FF04C0440F551F440F28
:1001C000551FB2FF06C052954295142F1F70407FF5
:1001D000512BB3FF1BC0A52F542F44270C9406812D
:1001E000B195B0FF02C055954795B1FF04C0559534
:1001F000479555954795B2FF05C05295407F42956A
:10020000452B5F70B3FF02C0452F5527DD24CC245A
:10021000BB24B2E0649FD018C108B00AB00B749F31
:10022000C018B108B00B849FB018B109659FC01801
:10023000B108B00B759FB018B109859FB0196A9FBE
:10024000B018B1097A9FB0194D9DA12C9924992716
:10025000332722275D9DA00C911C901F301F201F6B
:10026000AD9D900C911D301F201F4C9DA00C911C2A
:10027000901F301F201F5C9D900C911D301F201F70
:10028000AC9D900D311D201F4B9D900C911D301F7A
:10029000201F5B9D900D311D201FAB9D300D211D3A
:1002A0004B9F900D311D201F5B9F300D211DAB9F7B
:1002B000200DB1E0BB24CC24DD24699FD018C108F7
:1002C000B00AB00B799FC018B108B00B899FB01865
:1002D000B109639FC018B108B00B739FB018B10982
:1002E000839FB019629FB018B109729FB019D61AD6
:1002F000C70AB80A20F0B1E09B0F301F201F11245D
:10030000692F70E0732BCB01A0E0B0E0BC01CD0100
:10031000822B0F900F900F900F900F90DF91CF9145
:100320001F910F91FF90EF90DF90CF90BF90AF9013
:100330009F900895CF92DF92EF92FF920F931F93B9
:10034000CF93DF93C6E7D1E105EB1BE0C12CD12CA5
:100350007601C39469917991899199910F940223BF
:10036000288939894A895B890F9463230F94662B06
:10037000F80161937193819391938F01C616D7060B
:10038000E806F90610F46B017C01F1E1C638DF07DD
:1003900009F76FEF7FEFCB01A70196010F94532967
:1003A0002093C50B3093C60B4093C70B5093C80BDB
:1003B000DF91CF911F910F91FF90EF90DF90CF9041
:1003C00008950F931F93CF93DF930AE811E1CBECCD
:1003D000DBE0F80121913191419151918F0160E071
:1003E00070E080E89FE30F94ED2A699379938993F5
:1003F0009993FBE0CB3DDF0761F70E943F92DF91CD
:10040000CF911F910F910C949A819091FE1480913D
:10041000FF14981306C08091731190917411892B69
:1004200021F080E00E940655F0CF089520919611AA
:10043000309197114091981150919911FC01608170
:100440007181828193810F9463230F94602C609358
:100450002015709321158093221590932315909168
:10046000FE148091FF1498130C947E7C0E940582E8
:1004700080916F00982F927081FF05C080916F006E
:100480008D7F80936F0040912015509121156091D0
:100490002215709123154093BB1D5093BC1D609392
:1004A000BD1D7093BE1D992329F080916F0082605D
:1004B00080936F0008954F925F926F927F928F9218
:1004C0009F92AF92BF92CF92DF92EF92FF920F93E3
:1004D0001F93CF93DF93EC018B015A01F901209117
:1004E0009611309197114091981150919911608116
:1004F0007181828193810F9463230F94602C6B012F
:100500007C0120919211309193114091941150915E
:100510009511F50160817181828193810F9463232C
:100520000F94602C4B015C0120918E1130918F1142
:100530004091901150919111F801608171818281F7
:1005400093810F9463230F94602C2B013C01209125
:100550008A1130918B1140918C1150918D116881CD
:1005600079818A819B810F9463230F94602C60931F
:1005700014157093151580931615909317154092C6
:1005800018155092191560921A1570921B158092C9
:100590001C1590921D15A0921E15B0921F15C092A9
:1005A0002015D0922115E0922215F09223159091FA
:1005B000FE148091FF14981791F0DF91CF911F9155
:1005C0000F91FF90EF90DF90CF90BF90AF909F90F2
:1005D0008F907F906F905F904F900C947E7C0E94E4
:1005E000058280916F00982F927081FF05C08091E5
:1005F0006F008D7F80936F0040911C1550911D15E9
:1006000060911E1570911F15009118151091191504
:1006100020911A1530911B15C0901415D090151506
:10062000E0901615F0901715C092AF1DD092B01D36
:10063000E092B11DF092B21D0093B31D1093B41D52
:100640002093B51D3093B61D4093B71D5093B81D30
:100650006093B91D7093BA1D4091201550912115DA
:1006600060912215709123154093BB1D5093BC1DC2
:100670006093BD1D7093BE1D992329F080916F007A
:10068000826080936F00DF91CF911F910F91FF9057
:10069000EF90DF90CF90BF90AF909F908F907F9022
:1006A0006F905F904F900895CF93DF93C82F0F9472
:1006B000101024E0C29FE0011124C553D44F0F94C1
:1006C0000423288139814A815B810F946323DF9160
:1006D000CF9108959091FE148091FF14981306C055
:1006E0008091731190917411892B21F080E00E9408
:1006F0000655F0CF5F9A809178138E7F80937813A0
:100700008A9A809178138D7F809378138091080165
:100710008095817080930601809178138B7F809300
:1007200078130C943B51CF93DF9390916F00292F56
:10073000227091FF05C090916F009D7F90936F0094
:1007400094E0899FA0011124FA01ED55F24E6081D9
:10075000718182819381222329F020916F00226090
:1007600020936F00EA01C553D44F0F9404232881CE
:1007700039814A815B810F946323DF91CF91089582
:1007800080916F00982F927081FF05C080916F005B
:100790008D7F80936F008091FF148093FE1480936F
:1007A000FD148093FC1484E68093FB1428EE33E060
:1007B0003093741120937311992329F080916F0065
:1007C000826080936F0081E08093A21D08952F9234
:1007D0003F924F925F926F927F928F929F92AF92D1
:1007E000BF92CF92DF92EF92FF920F931F93CF931E
:1007F000DF93CDB7DEB7CB56D1090FB6F894DEBF85
:100800000FBECDBF4B015A0169012D96FFAEEEAE72
:100810002D9720918A1130918B1140918C1150911C
:100820008D11DC016D917D918D919C910F946323CD
:100830000F94602CA3966CAF7DAF8EAF9FAFA39744
:1008400020918E1130918F11409190115091911102
:10085000F40160817181828193810F9463230F94ED
:10086000602CA7966CAF7DAF8EAF9FAFA7972091FE
:100870009211309193114091941150919511D5019D
:100880006D917D918D919C910F9463230F94602CB9
:10089000AB966CAF7DAF8EAF9FAFAB9720919611AB
:1008A000309197114091981150919911F601608102
:1008B0007181828193810F9463230F94602C2B9616
:1008C0006CAF7DAF8EAF9FAF2B978091751183FF7B
:1008D0000EC02B962CAD3DAD4EAD5FAD2B9720934A
:1008E00020153093211540932215509323158091A4
:1008F000731190917411892B11F00C949690D8017A
:100900003C901196BC91BDABF801F281F9AFD801D2
:1009100013962C908091FE149091FF14891B8F7078
:100920008F3021F480E00E940655F4CFB091FE1480
:10093000AC96BFAFAC978091FE14E82FF0E0F8A71B
:10094000EFA3F8E58F9FC00111249C012D50344F77
:1009500023963FAF2EAF23978091141590911515D4
:10096000A0911615B0911715A3968CAC9DACAEACAA
:10097000BFACA397881A990AAA0ABB0A80911815D6
:1009800090911915A0911A15B0911B15A7962CAD31
:100990003DAD4EAD5FADA797281B390B4A0B5B0BE6
:1009A0002BA33CA34DA35EA380911C1590911D1514
:1009B000A0911E15B0911F15AB962CAD3DAD4EAD5F
:1009C0005FADAB97281B390B4A0B5B0B29A73AA7E6
:1009D0004BA75CA78091201590912115A09122151D
:1009E000B09123152B96CCACDDACEEACFFAC2B97C5
:1009F000C81AD90AEA0AFB0A09F477C08091DB0B0E
:100A000081112DC020E030E0A9016091E00B7091D0
:100A1000E10B8091E20B9091E30B0F94F3290F947B
:100A20005F2B20912B0230912C0262177307BCF4CC
:100A30002B968CAD9DADAEADBFAD2B9780932015A1
:100A400090932115A0932215B09323150F9424039E
:100A50008EE89EE10F943B02C12CD12C7601C70198
:100A6000B6010F940423209127023091280240916F
:100A7000290250912A020F9463232B013C0120E0AC
:100A800030E0A9010F94532C87FF04C077FA7094CB
:100A900077F8709420E030E04AEF53E460919611CB
:100AA0007091971180919811909199110F946323EF
:100AB000A30192010F94FD2287FF17C02B962CAD46
:100AC0003DAD4EAD5FAD2B97209320153093211592
:100AD00040932215509323150F9424038FE69EE133
:100AE0000F943B02C12CD12C7601D501C40188277B
:100AF000B7FD83959927AA27BB27182F2BA13CA1C7
:100B00004DA15EA157FD126089A59AA5ABA5BCA514
:100B1000B7FD1460F7FC1860C701B6010F940423F9
:100B200020912702309128024091290250912A02F7
:100B30000F9463236B017C0120E030E0A9010F9446
:100B4000532C87FF04C0C701B601905802C0C701EB
:100B5000B60120E030E040E05FE30F94F3290F940A
:100B6000662B69AB7AAB8BAB9CAB88E5AFA1B8A524
:100B70008A9FF0018B9FF00D1124ED50F44F1082ED
:100B8000EB5BFF4F108329A53AA54BA55CA52796E3
:100B90002CAF3DAF4EAF5FAF279757FF0DC05095BD
:100BA0004095309521953F4F4F4F5F4F27962CAF83
:100BB0003DAF4EAF5FAF27978BA19CA1ADA1BEA16A
:100BC0008DA79EA7AFA7B8ABB7FF0BC0B095A095F8
:100BD000909581959F4FAF4FBF4F8DA79EA7AFA711
:100BE000B8AB24013501B7FE07C0442455243201B7
:100BF000481859086A087B082396AEADBFAD239705
:100C000055964D925D926D927C9258972DA53EA57A
:100C10004FA558A959962D933D934D935C935C979E
:100C200027962CAD3DAD4EAD5FAD27975D962D93CC
:100C30003D934D935C939097C501B4010F940423A9
:100C40002091CB0B3091CC0B4091CD0B5091CE0B22
:100C50000F94632321966CAF7DAF8EAF9FAF21972A
:100C6000698B7A8B8B8B9C8B6BA17CA18DA19EA1B8
:100C70000F9404232091CF0B3091D00B4091D10BD6
:100C80005091D20B0F9463236BA37CA38DA39EA3DF
:100C90006D8B7E8B8F8B988F69A57AA58BA59CA574
:100CA0000F9404232091D30B3091D40B4091D50B9A
:100CB0005091D60B0F9463234B015C01698F7A8F9F
:100CC0008B8F9C8F2091D70B3091D80B4091D90BF3
:100CD0005091DA0BC701B6010F9463236B017C01BD
:100CE0006D8F7E8F8F8F98A3B6E04B1651046104F1
:100CF00071049CF52DA53EA54FA558A926303105B8
:100D00004105510554F527968CAD9DADAEADBFADF7
:100D100027970697A105B10504F520E030E0A90169
:100D2000C701B6010F94532C87FF04C0F7FAF09463
:100D3000F7F8F09488E5AFA1B8A58A9F80018B9F52
:100D4000100D11240D50144F20E030E0A901C7010F
:100D5000B6010F94F329F80154C02D96AEADBFAD86
:100D60002D97CD90DD90ED90FC9020E030E0A90132
:100D7000C701B6010F94FD22882379F088E52FA1E1
:100D800038A5829FF001839FF00D1124ED50F44FA0
:100D9000C586D686E786F08A38C021962CAD3DAD53
:100DA0004EAD5FAD2197CA01B9010F9463236B016A
:100DB0007C012BA13CA14DA15EA1CA01B9010F94F8
:100DC00063239B01AC01C701B6010F94F3296B01AA
:100DD0007C01A5019401C501B4010F9463239B011B
:100DE000AC01C701B6010F94F3290F94A12C28E59B
:100DF0004FA158A5249FF001259FF00D1124ED501F
:100E0000F44F658776878787908B88E5AFA1B8A573
:100E10008A9FF0018B9FF00D1124ED50F44F29A90A
:100E20003AA94BA95CA921A332A343A354A32796B3
:100E30008CAD9DADAEADBFAD27972DA53EA54FA501
:100E400058A982179307A407B50710F4DA01C9015E
:100E500084159505A605B70510F4D301C20129A98B
:100E60003AA94BA95CA982179307A407B50710F408
:100E7000DA01C90128E54FA158A5249FF001259F5B
:100E8000F00D1124ED50F44F85A396A3A7A3B0A7AE
:100E90000697A105B10510F40C944491DF01AA5AFC
:100EA000BF4F8091C90B8C93E95AFF4F8091CA0BB9
:100EB000808345284628472809F05F9888E5AFA138
:100EC000B8A58A9FF0018B9FF00D1124ED50F44FCF
:100ED000818D928DA38DB48D892B8A2B8B2B09F05C
:100EE0008A9888E52FA138A5829FF001839FF00D95
:100EF0001124ED50F44F858D968DA78DB0A1892BCF
:100F00008A2B8B2B29F08091080181708093060138
:100F100089A99AA9ABA9BCA9892B8A2B8B2B11F47F
:100F20000C9498908091CE11882319F08150809371
:100F3000CE11129880E28093CE11E090B611F0901D
:100F4000B7110091B8111091B9119701A801632D43
:100F50007DA989AD922D0F94FD2287FF04C03E2C00
:100F6000FDAA09AF212E88E5AFA1B8A58A9FF0019F
:100F70008B9FF00D1124ED50F44F25853685478564
:100F8000508927962CAF3DAF4EAF5FAF279760E0FB
:100F900070E080E89FE30F94ED2A6BA37CA38DA300
:100FA0009EA3232D3DA949AD522D0F9463236B01C0
:100FB0007C018091FE149091FC14891B8F7089AF85
:100FC000A701960160E074E284E799E40F94ED2AAA
:100FD0000F94602C4B015C0189AD82508630B0F5D6
:100FE0008091861190918711A0918811B0918911FB
:100FF00088169906AA06BB0648F588199909AA0910
:10100000BB09BC01CD01660F771F881F991F49AD31
:10101000042F10E020E030E0A90198010F9453293B
:10102000CA01B9010F9402230F94602C680D791D39
:101030008A1D9B1D0F9402239B01AC0160E074E2AA
:1010400084E799E40F94ED2A6B017C01A7019601D6
:1010500027966CAD7DAD8EAD9FAD27970F94632322
:101060009B01AC010F9463236DAB7EAB8FAB98AF4C
:1010700088E5AFA1B8A58A9F80018B9F100D112430
:101080000D50144F2DA93EA94FA958ADD801119666
:101090002D933D934D935C93149795964D905D9051
:1010A0006D907C909897C301B2010F94022369A7B9
:1010B0007AA78BA79CA79B01AC01C701B6010F942F
:1010C00063230F94D12A0F94662B21966CAF7DAFCA
:1010D0008EAF9FAF2197F801EA5BFF4F608371836A
:1010E00082839383FE017196FEA7EDA72AE931E181
:1010F00061963FAF2EAF6197AE014F5D5F4F5AA330
:1011000049A300E010E050E8252E6FE3362EADA590
:10111000BEA52D913D914D915D91BEA7ADA7C70193
:10112000B6010F9463234B015C0120E030E0A9017C
:101130000F94532C87FF04C0B7FAB094B7F8B0945B
:101140006196AEADBFAD61972D913D914D915D9191
:101150006196BFAFAEAF61972F962CAF3DAF4EAF4C
:101160005FAF2F97A50194012F966CAD7DAD8EAD2D
:101170009FAD2F970F94FD2287FF14C0A501940106
:101180002F966CAD7DAD8EAD9FAD2F970F94ED2A50
:101190005B014C019801A1010F94FD2287FF02C061
:1011A00085011401EDA5FEA529A13AA1E217F307D7
:1011B00009F0ADCF20E030E040E85FE3B801C101C5
:1011C0000F94FD2287FF36C028E54FA158A5249F24
:1011D000C001259F900D1124DC01AD50B44F7D015D
:1011E0006D01B6E4CB0ED11C21966CAD7DAD8EADFC
:1011F0009FAD21970F9402239801A1010F946323BF
:101200000F94662BF6016083718382839383980128
:10121000A101B801C1010F9463232DA93EA94FA9D3
:1012200058AD0F946323D70111966D937D938D93E1
:101230009C93149729A53AA54BA55CA56BA17CA10D
:101240008DA19EA10F94632321966CAF7DAF8EAFCD
:101250009FAF219788E52FA138A5829FF001839F3A
:10126000F00D1124ED50F44F85889688A788B08C36
:1012700081149104A104B10419F5818D928DA38D7F
:10128000B48D892B8A2B8B2BD9F4858D968DA78DC8
:10129000B0A1892B8A2B8B2B99F42091AE11309120
:1012A000AF114091B0115091B11121966CAD7DAD4F
:1012B0008EAD9FAD21970F9463230F94D12AFBC16C
:1012C00089A99AA9ABA9BCA9892B8A2B8B2B49F098
:1012D0002091AA113091AB114091AC115091AD11F8
:1012E00008C02091B2113091B3114091B4115091C6
:1012F000B51121966CAD7DAD8EAD9FAD21970F944C
:1013000063230F94D12A0F94662B6B017C0180918B
:10131000C50B9091C60BA091C70BB091C80B23963B
:10132000EEADFFAD2397218D328D438D548D29ABCA
:101330003AAB4BAB5CAB258D368D478D50A12DA7BD
:101340003EA74FA758AB21A132A143A154A12DAB79
:101350003EAB4FAB58AF84159505A605B70508F40D
:10136000AFC081149104A104B10471F16091B50B77
:101370007091B60B8091B70B9091B80B6C157D05F1
:101380008E059F0508F5A30192010F94432969A7D3
:101390007AA78BA79CA7A5019401C701B6010F945A
:1013A000432929A53AA54BA55CA526173707480769
:1013B000590750F469A57AA58BA59CA5A5019401B0
:1013C0000F94532969017A0129A93AA94BA95CA96B
:1013D000232B242B252B51F16091B90B7091BA0B63
:1013E0008091BB0B9091BC0B6C157D058E059F0504
:1013F000E8F4A30192010F9443294B015C0129A950
:101400003AA94BA95CA9C701B6010F9443298616D6
:101410009706A806B90650F4C501B40129A93AA94E
:101420004BA95CA90F94532969017A018DA59EA54A
:10143000AFA5B8A9892B8A2B8B2B51F16091BD0BDD
:101440007091BE0B8091BF0B9091C00B6C157D0508
:101450008E059F05E8F4A30192010F9443294B01E7
:101460005C012DA53EA54FA558A9C701B6010F9453
:10147000432986169706A806B90650F4C501B4019B
:101480002DA53EA54FA558A90F94532969017A01AE
:101490002DA93EA94FA958AD232B242B252B09F4A8
:1014A0000EC16091C10B7091C20B8091C30B9091E2
:1014B000C40B6C157D058E059F0508F443C6FFC05F
:1014C00081149104A104B104B9F16091B50B70913C
:1014D000B60B8091B70B9091B80B6C157D058E05FE
:1014E0009F0550F50F94022329A53AA54BA55CA5AD
:1014F0000F9463232B013C01C501B4010F94022317
:101500004B015C01C701B6010F940223A5019401B0
:101510000F9463239B01AC01C301B2010F94FD2220
:1015200087FF0AC0A5019401C301B2010F94ED2AFF
:101530000F94662B6B017C0189A99AA9ABA9BCA960
:10154000892B8A2B8B2BC9F16091B90B7091BA0B47
:101550008091BB0B9091BC0B6C157D058E059F0592
:1015600060F50F94022329A53AA54BA55CA50F941D
:1015700063234B015C0169A97AA98BA99CA90F94EB
:1015800002232B013C01C701B6010F940223A301E2
:1015900092010F9463239B01AC01C501B4010F9428
:1015A000FD2287FF0AC0A3019201C501B4010F9477
:1015B000ED2A0F94662B6B017C012DA53EA54FA54E
:1015C00058A9232B242B252BC9F16091BD0B7091B9
:1015D000BE0B8091BF0B9091C00B6C157D058E05E5
:1015E0009F0560F50F94022329A53AA54BA55CA59C
:1015F0000F9463234B015C016DA57EA58FA598A96F
:101600000F9402232B013C01C701B6010F94022362
:10161000A30192010F9463239B01AC01C501B401A6
:101620000F94FD2287FF0AC0A3019201C501B401F6
:101630000F94ED2A0F94662B6B017C018DA99EA956
:10164000AFA9B8AD892B8A2B8B2BC9F16091C10B47
:101650007091C20B8091C30B9091C40B6C157D05EA
:101660008E059F0560F50F94022329A53AA54BA589
:101670005CA50F9463234B015C016DA97EA98FA922
:1016800098AD0F9402232B013C01C701B6010F94C2
:101690000223A30192010F9463239B01AC01C501B6
:1016A000B4010F94FD2287FF0AC0A3019201C50176
:1016B000B4010F94ED2A0F94662B6B017C0188E531
:1016C000AFA1B8A58A9F80018B9F100D11240D50EA
:1016D000144FF801EE5AFF4FC082D182E282F382AA
:1016E000C701B6010F94022321962CAD3DAD4EAD3E
:1016F0005FAD21970F94ED2A6DA77EA78FA798ABBA
:10170000F801618B728B838B948B29893A894B8981
:101710005C896BA17CA18DA19EA10F94632321966E
:101720006CAF7DAF8EAF9FAF21972D893E894F89DA
:10173000588D6BA17CA18DA19EA10F9463232F9640
:101740006CAF7DAF8EAF9FAF2F97298D3A8D4B8DAC
:101750005C8D6BA17CA18DA19EA10F9463236396E8
:101760006CAF7DAF8EAF9FAF63972D8D3E8D4F8D4C
:1017700058A16BA17CA18DA19EA10F9463236796B4
:101780006CAF7DAF8EAF9FAF6797F9ADFF2309F4C4
:1017900076C2209100152BA33091011539A7309006
:1017A0000215209003152DEB37E346E855E36BA1B6
:1017B00079A5832D922D0F94FD2287FD60C2809024
:1017C000BE119090BF11A090C011B090C111C090F7
:1017D000C211D090C311E090C411F090C511809156
:1017E000C6119091C711A091C811B091C9118DABCC
:1017F0009EABAFABB8AF2091CA113091CB114091E5
:10180000CC115091CD1129AF3AAF4BAF5CAFC501B0
:10181000B401905821962CAD3DAD4EAD5FAD2197F2
:101820000F9463232B013C01C701B60190582F96FA
:101830002CAD3DAD4EAD5FAD2F970F9463239B0153
:10184000AC01C301B2010F94F3292B013C016DA936
:101850007EA98FA998AD905863962CAD3DAD4EAD45
:101860005FAD63970F9463239B01AC01C301B20189
:101870000F94F3292B013C0169AD7AAD8BAD9CAD82
:10188000905867962CAD3DAD4EAD5FAD67970F9408
:1018900063239B01AC01C301B2010F94F32969AB2F
:1018A0007AAB8BAB9CAB2FEE3FEF4FE75FE30F9430
:1018B000532C18160CF4B2C12FEE3FEF4FE75FEB3D
:1018C00069A97AA98BA99CA90F94FD2287FF08C05A
:1018D0008FEE9FEFAFE7BFEB89AB9AABABABBCAB87
:1018E000A501940121966CAD7DAD8EAD9FAD219784
:1018F0000F94F2292B013C0169837A838B839C83AB
:10190000A70196012F966CAD7DAD8EAD9FAD2F9743
:101910000F94F2296B966CAF7DAF8EAF9FAF6B9734
:101920006D837E838F8398872DA93EA94FA958ADDB
:1019300063966CAD7DAD8EAD9FAD63970F94F2292C
:101940006F966CAF7DAF8EAF9FAF6F9769877A87C9
:101950008B879C8729AD3AAD4BAD5CAD67966CAD7E
:101960007DAD8EAD9FAD67970F94F22969AF7AAFC9
:101970008BAF9CAF6D877E878F87988BDE0111962A
:10198000BEABADABFE017196FAA3E9A38D01C12CEC
:10199000D12C7601D8018D909D90AD90BD908D0198
:1019A00020E030E0A901C501B4010F94FD22882395
:1019B00071F0A5019401C501B4010F9463239B014B
:1019C000AC01C701B6010F94F3296B017C01E9A1B9
:1019D000FAA1E017F107F1F6C701B6010F94A12CA7
:1019E0009B01AC0160E070E080E89FE30F94ED2A7A
:1019F0006B017C019B01AC01C301B2010F94632315
:101A000069837A838B839C83A70196016B966CAD67
:101A10007DAD8EAD9FAD6B970F9463236D837E83F9
:101A20008F839887A70196016F966CAD7DAD8EADC3
:101A30009FAD6F970F94632369877A878B879C8705
:101A4000A701960169AD7AAD8BAD9CAD0F94632370
:101A50006D877E878F87988B06E711E14DA46EA472
:101A60005FA478A8ADA9BEA9CD90DD90ED90FD90C2
:101A7000BEABADAB20E030E0A901C701B6010F94C9
:101A8000FD22882331F1F801608171818281938187
:101A90000F940223A70196010F94ED2A6B017C019C
:101AA00020E030E0A9010F94532C87FF04C0F7FA1F
:101AB000F094F7F8F094242D362D452D572DC701BD
:101AC000B6010F94FD2287FF04C04C2C6D2C5E2CB8
:101AD0007F2C0C5F1F4F29A13AA14DA95EA92417A5
:101AE000350709F0BFCF29A93AA94BA95CA960E045
:101AF00070E080E89FE30F94F22920E030E040E0BE
:101B00005FE30F9463230F94A12C6B017C01209160
:101B1000B10B3091B20B4091B30B5091B40B642DCB
:101B2000762D852D972D0F946323A70196010F9491
:101B300063234B015C01A701960160E070E080E83F
:101B40009FE30F94F2299B01AC01C501B4010F94EE
:101B5000ED2A7B018C0120E030E040E85FE327962E
:101B60006CAD7DAD8EAD9FAD27970F94FD2287FFA5
:101B70005BC029A93AA94BA95CA9CA01B9010F9474
:101B8000632323EC38EB42E35FEB0F94632323EFF3
:101B900036E64FE55FE30F94F22929A93AA94BA94C
:101BA0005CA90F9463232BED3FE049EC5FE30F94B6
:101BB000F3292CEE31E548E35EE30F94F2294B0163
:101BC0005C0124EE3BEC46E150E40F94532C1816D4
:101BD0005CF5A50194016BED7FE089E490E40F943E
:101BE000F2299B01AC0127966CAD7DAD8EAD9FAD0A
:101BF00027970F94ED2A242D362D452D572D0F9420
:101C000063235B016C019B01AC01B701C8010F9418
